:020000022000DC
:1060000000000420F9D7070039D807003BD8070063
:106010003DD807003FD8070041D807000000000026
:10602000000000000000000000000000E5D60700AE
:1060300045D807000000000005D7070049D8070031
:106040002DDA07004BD80700E1AB07003534040018
:10605000E53404004BD8070029B007004BD80700EF
:106060004BD807004BD807004BD807004BD8070088
:106070004BD807004BD807004BD807004BD8070078
:106080004BD8070069D407004BD807004BD807004E
:106090004BD807004BD80700F98C07004BD80700F6
:1060A0004BD807004BD807004BD807004BD8070048
:1060B0004BD807004BD8070000000000000000008C
:1060C0004BD807004BD807004BD8070019E0070052
:1060D0004BD807004BD807004BD80700C96C02000B
:1060E0002DAC07004BD807004BD80700000000007C
:1060F000000000004BD807000000000091E00700FE
:10610000000000000000000000000000000000008F
:10611000000000000000000000000000000000007F
:10612000000000000000000000000000000000006F
:10613000000000000000000000000000000000005F
:10614000000000000000000000000000000000004F
:10615000000000000000000000000000000000003F
:10616000000000000000000000000000000000002F
:10617000000000000000000000000000000000001F
:10618000000000000000000000000000000000000F
:1061900000000000000000000000000000000000FF
:1061A00000000000000000000000000000000000EF
:1061B00000000000000000000000000000000000DF
:1061C00000000000000000000000000000000000CF
:1061D00000000000000000000000000000000000BF
:1061E00000000000000000000000000000000000AF
:1061F000000000000000000000000000000000009F
:10620000F1EE103A43F08073E1EE103A704700BFB0
:1062100010B5054C237833B9044B13B10448AFF3E0
:1062200000800123237010BD946500200000000051
:10623000600A0A0008B5034B1BB103490348AFF3DA
:10624000008008BD0000000098650020600A0A0078
:10625000154B002B08BF134B9D46A3F5803A002138
:106260008B460F461348144A121A62F00EF90F4B70
:10627000002B00D098470E4B002B00D098470020F1
:10628000002104000D000D48002802D00C48AFF397
:10629000008062F067F82000290057F0FFFA61F0F3
:1062A0008DFF00BF00000800000004200000000077
:1062B0000000000094650020BCD700200000000012
:1062C000000000000146014800F07ABACC650020C9
:1062D00038B5064B1D783DB100242046013400F04E
:1062E00035FEE0B28542F9D838BD00BFC865002050
:1062F000407DFF2806D010B500F074FD044618B1AB
:10630000204610BD0020704758F03EF8204610BDD2
:10631000407DFF280ED000B583B00DF1070100F0DD
:10632000B5FD20B19DF8070003B05DF804FB4FF008
:10633000FF30F9E74FF0FF30704700BF407DFF2886
:1063400011D000B583B001220DF1070100F056FD18
:1063500020B94FF0FF3003B05DF804FB9DF8070053
:1063600003B05DF804FB4FF0FF307047407DFF281D
:1063700001D000F0EBBD7047407DFF2801D000F058
:106380002BBE0020704700BFF8B50646407DFF28B1
:106390001CD017465AB10D46144600F0FDFC2946A4
:1063A000224680B1707D00F07BFD241A01D1384671
:1063B000F8BD054457F0E8FF707D00F0EDFC29467C
:1063C00022460028EED13F1B3846F1E70020F8BDF9
:1063D0000AB32DE9F043524991F81C6191F81D511F
:1063E00091F81E7193B0994614467B1CAA1C8046F6
:1063F000B01C81F81C0181F81D2181F81E3101A813
:106400004222002162F041F8B9F1410F05D8002085
:1064100013B0BDE8F083422070478DF806608DF818
:106420000E608DF82660721C40F20126D2B2ADF8E3
:106430001060DFF8F0C08DF81E20242640F6083EDC
:106440006B1C8DF827208DF83120ADF804E08DF815
:1064500016608DF820608DF82460CDF818C00426F1
:106460004FF0060C65F07F0540F209424FF0010E37
:1064700098F81410ADF80C208DF81CE005228DF86A
:106480001F608DF830608DF822C040F207568DF8FD
:1064900025C08DF82A5020464FF0030E63F07F048C
:1064A0004FF0080C02234FF411658DF814108DF88D
:1064B00007308DF808308DF809308DF812308DF8DE
:1064C00021308DF815208DF823208DF82BE08DF8E4
:1064D0002CC04FF00A0EADF82E504FF0400C01A921
:1064E000ADF8286007258DF833308DF840208DF801
:1064F0004140422244F20204ADF838608DF83B304E
:106500008DF83A708DF834E08DF83CC08DF83F502E
:10651000ADF8424061F095FF422013B0BDE8F08332
:10652000CC65002020010524A0F11000FFF750BF2A
:1065300070B50368184A5B6882B093428DF8071003
:1065400024D10546407DFF281DD000F025FC0DF12B
:10655000070601243146224688B1687D00F0A0FC80
:10656000241A02D1012002B070BD064457F00CFF7E
:10657000687D00F011FC314622460028EDD1C4F1BF
:10658000010002B070BD002002B070BD01220DF10B
:106590000701984702B070BD89630200437DFF2B5D
:1065A00000D07047094B1A78002AFAD110B500F1D3
:1065B000100442750649204601221A7000F0CCF9F9
:1065C00021460448BDE8104000F0DCB8C865002052
:1065D00010D30800CC65002001B900B1704700B5A8
:1065E00083B0694600F0EEFB009BB3F5966F02D0D6
:1065F00003B05DF804FB00F07DFBF9E730B4084B15
:10660000084A4FF47F4102F10805002430324FF46C
:106610007A7099821D60C3E901401A6130BC7047ED
:10662000B065002020D308002DE9F0410024484E39
:106630002546435D4719A3B103F14002D2B2012AB6
:106640000AD9F42B08D81A060ED44FF0010EA3F580
:106650005842B2F5006F56D201354719435D002B01
:10666000EAD12046BDE8F08103F0E002C02A57D00D
:1066700003F0F002E02A66D003F0F802F02AEBD132
:1066800003F007024FF0040E7B7803F0C00CBCF15E
:10669000800FE1D197F802C00CF0C00803F03F036F
:1066A000B8F1800F43EA8213D6D10CF03F0CBEF153
:1066B000030F4CEA83132DD0FA7802F0C007802F25
:1066C000CAD102F03F0242EA8313A3F58032B242FC
:1066D000C2D8A3F55847B7F5006FBDD3B3F5803FD7
:1066E00005F1040510D31E2CBBDC6300970A0B4494
:1066F000C2F30902A7F52057A2F5105221F8147031
:106700005A80023495E77544202CAAD021F8143021
:1067100001348EE7A3F50062B2F5784F97D39BE77B
:106720007A7802F0C007802F03F01F0394D102F0A3
:106730003F0242EA8313A3F18002B2F5F06F8BD2DD
:106740004FF0020E83E703F00F024FF0030E9BE7BA
:10675000FFFF0F0090F850310B2B0CD871B103F1F3
:10676000480210B45C1C80F8504140F822105DF8DB
:10677000044B184670470023184670470B461846CE
:10678000704700BF70B504460E68B4F81821B4F81D
:106790001A31656936689B1A08469BB294F81C1139
:1067A0002A44B04758B1B4F818216369104480B244
:1067B000A4F81801588094F81C211A71012070BDAA
:1067C0002DE9F043284DDFF8B090AC4604468846EA
:1067D000BCE80F0089B003AF0FC703AE0FCE05F1C1
:1067E000140E25460FC59EE80700DCF800303B80FC
:1067F0006B4636682E8003C36B4603CB012504F13C
:1068000018034FF480766361A061E16184F8202071
:1068100004F59870C4F818912022A4F81C61002196
:1068200084F81E5161F031FE40F20947042240F223
:10683000EF230E4E0E48C4F828010021C4F82C1195
:1068400084F85021A3804FF4E131A571C4F8207180
:10685000C4F824610748FFF7A1FE404600F038FA6B
:10686000284609B0BDE8F08354D3080084D308005B
:106870008CD30800B0650020090000010048704773
:10688000CC650020014B5869704700BFCC650020E3
:106890002DE9F04F89B0F8B1032816D02B4C94F8AD
:1068A000503183424FD9483004F5AA7154F8200082
:1068B000FFF7BAFEC0B20130400040F44070A4F8C7
:1068C0005201234809B0BDE8F08F204CD4F82C01C8
:1068D00050B104F5AA71EBE71C4CD4F82031A4F8B0
:1068E00054314FF44170EAE7684600F005FA054676
:1068F00010B300F1FF3A0DF10103164FE94653FAC8
:106900008AFAA64604AE97E80F0019F801CB86E88C
:106910000F000CF00F080DF1200BD8440BEB1C1CE2
:1069200018F8108C1CF8103CAEF85681D145AEF822
:1069300054310EF1040EE6D16800C0B201304000BF
:1069400040F44070BBE70020BCE700BFCC650020EE
:106950001E67002074D3080010B504460248FFF7F4
:10696000F9FE207110BD00BFCC65002030B5144C7D
:10697000236883B013B3186851B91CF0F5F9236884
:1069800093F90400012103B0BDE8304058F03CB851
:106990000C4B0093002501238DF805308DF8045031
:1069A00002AB13E906001CF07BF9236893F904009D
:1069B000294603B0BDE8304058F026B803B030BDDA
:1069C0006067002080BA8C010448006828B108B5CF
:1069D00000681CF017FA012008BD704760670020AE
:1069E000084B1B6843B141B9074B4022C3F88020D4
:1069F000BFF34F8FBFF36F8F7047034B40221A6076
:106A0000704700BF6067002000E100E0024B53F8D0
:106A1000200000B1C06870476467002030B4094CA2
:106A2000BDF8085054F8204044B1246934B10846F8
:106A3000A44611461A462B4630BC6047002030BCA5
:106A4000704700BF6467002030B4084CBDF80850A0
:106A500054F8204044B1646934B10846A446114654
:106A60001A462B4630BC604730BC70476467002034
:106A700000207047024B186808B190F8600070471A
:106A80006C6700202DE9F843234C2568002D3CD08D
:106A90001E462C2303FB00531746D3F8209088464C
:106AA0000446B9F1000F32D0484662F0E4FD2C23D1
:106AB00003FB0454D4E90954DFF864C0174B0828D9
:106AC0000246494628BF08224046002D08BF6546B9
:106AD000002C08BF1C4661F0B4FC284662F0CBFDD8
:106AE00010280246294628BF1022384661F0A9FC2A
:106AF000204662F0C0FD042802462146304628BFE9
:106B00000422BDE8F84361F09CBCBDE8F883DFF8DF
:106B100014900820CBE700BF6C670020B4D30800B6
:106B2000A4D3080098D3080070B5104E3368D3B1D1
:106B30002C2404FB0034054662691AB1904733687F
:106B400084F832002C2202FB053393F8324014B152
:106B50000124204670BD284623463A22022101F036
:106B6000E7F8204670BD1C46204670BD6C670020CB
:106B7000074B1B6853B110B42C2404FB0030C46ACB
:106B8000038E0C6013805DF8044B7047704700BFA4
:106B90006C67002008B520220023052101F0C8F809
:106BA0004FF0FF3008BD00BF30B4094C24685CB121
:106BB0000D4611462C2202FB0044E46924B11A461A
:106BC0002846234630BC1847012030BC704700BF20
:106BD0006C67002030B4094C029A246854B10D4609
:106BE0002C2101FB0044A46824B119462846234601
:106BF00030BC18474FF0FF3030BC70476C67002046
:106C000030B4094C029A246854B10D462C2101FB82
:106C10000044E46824B119462846234630BC18478E
:106C20004FF0FF3030BC70476C670020044B1B688E
:106C30002BB12C2202FB0030036903B118477047C7
:106C40006C670020054B1B682BB12C2202FB003027
:106C5000836903B118470120704700BF6C670020AB
:106C600005F0DCBB00B5164B83B04022002483F84E
:106C7000272301A9012320468DF804308DF8054013
:106C800002F0DAFE4FF0804302A8D3F8385400F83F
:106C9000084D56F04DFE0B4B019301A856F098FE9F
:106CA00056F0A8FEEB0707D400214FF0FF3002F0AA
:106CB0004DFFFFF70DFBF7E7204605F0AFFBF3E7CD
:106CC00000E100E0616C0200002005F01DB800BF8B
:106CD00000B5002383B00322CDE900230349044813
:106CE000C82255F0F1FA03B05DF804FBB8D30800F0
:106CF000656C020057F0F4BC4FF08052536E1BBA23
:106D00000360136E1BBA4360082070470048704749
:106D1000C0D3080070B51E4C2368D3B1012901D03F
:106D2000012070BD1578C5F34115012D13D0022D3A
:106D30000FD15478012C21D0022CF1D19388072B4C
:106D400007D1144C114623892246BDE8704003F058
:106D500035BE002070BD51782229E1D111465288FC
:106D6000003218BF01225A7503F010FE2268D36961
:106D7000002BD5D0507D9847284670BD9C69002CCB
:106D8000E7D0114623782246BDE8704003F016BED6
:106D9000706700200460002010B5044602F034FE45
:106DA00008B9002010BD02F037FE0028F9D1044BCD
:106DB0004FF4367202FB0434207900F0010010BD5C
:106DC000F4670020064A4FF4367303FB00230833B0
:106DD000186808609A889B798B718A80704700BF19
:106DE000F467002008B5044A4FF4367303FB002013
:106DF000103002F055FC08BDF46700202DE9F8437F
:106E00004FF4367404FB00F41E4E4FF6FF73074632
:106E100004F110054FF6FE70824288BF1A463544D1
:106E2000284692B202F066FC804602F0EDFD10B9F1
:106E30004046BDE8F88302F0EFFD81460028F7D117
:106E40003444E378002BF3D0284602F041FC3F287D
:106E5000EED9E178484603F0E7FC0028E8D0284660
:106E600002F036FC3F2804D8E178484603F0ECFCF9
:106E7000DEE7054AE178484602EBC712402303F0FB
:106E8000F3FCD5E7F467002074670020034A4FF451
:106E9000367303FB0020103002F096BCF46700202C
:106EA0002DE9F8434FF4367505FB00F5244F4FF6F6
:106EB000FF73064605F124044FF6FE70824288BF38
:106EC0001A463C4492B2204602F0B8FC8046204666
:106ED00002F0E6FB3F2802D84046BDE8F88302F006
:106EE00093FD0028F8D002F097FD81460028F3D1E9
:106EF000204602F0D5FB0028EED03D444846A97854
:106F000003F092FC0028E7D00E4B402202EBC6169D
:106F10001E442046314602F0EDFB034660B1324686
:106F2000A978484603F0A0FC0028D5D1064B1B6881
:106F3000DB07D1D500BECFE7A97803F085FCCBE70E
:106F4000F467002074670020F0ED00E02DE9F041C7
:106F5000804602F059FD10B90020BDE8F08102F032
:106F60005BFD07460028F7D14FF4367404FB08F4A4
:106F7000164E04F124053544284602F091FB002802
:106F8000EAD026443846B17803F04EFC0028E3D01E
:106F900040220F4B02EBC81898442846414602F0A5
:106FA000A9FB044660B14246B1783846234603F057
:106FB0005BFC40B9074B1B68DB07CDD500BECCE7B7
:106FC000B17803F041FC2046C7E700BFF46700201A
:106FD00074670020F0ED00E008B5044A4FF4367302
:106FE00003FB0020243002F073FB08BDF46700208F
:106FF00070B5204C82B000214FF4367220460D4609
:1070000061F043FAFF234FF4E132082604F138011E
:107010006371A26001234FF48072009504F11000A7
:10702000A67302F001FB144B1B78C3F3800300939B
:1070300004F59C7101234FF4807204F1240002F0E6
:10704000F3FA04F50E71012054F082FB04F522716D
:107050000646012054F07CFB06B130B9074B1B6893
:10706000DB0700D500BE02B070BDC4E90756C4E915
:107070000C05F8E7F4670020B8600020F0ED00E0B0
:1070800038B5094C206A256B20B154F085FF0023E8
:10709000C4E907332DB1284654F07EFF0023C4E92C
:1070A0000C33012038BD00BFF467002010B50E4C32
:1070B0000E482378002202600271DA0709D59B0787
:1070C0000DD521780A48C1F38001BDE8104002F0D7
:1070D00063BC103002F040FC23789B07F1D40448D5
:1070E00002F03AFCEDE700BFB8600020F467002032
:1070F000186800202DE9F0414B79022B82B004D0B2
:107100000025284602B0BDE8F0818B79022BF7D12B
:10711000364EB3782BB1364B1B68DB07F0D500BE7B
:10712000EEE78B7833700C780C4407466378242B99
:107130004FF009050BD1082A02D822E0AA4220D339
:1071400023781C441D446378242BADB2F6D0052B64
:1071500038D0042B15D163790A2B12D1254A94F823
:1071600000800192022301320092384604EB0801AC
:107170001A4603F095FA0028CDD00E3518FA85F599
:10718000ADB202F041FC0028BBD002F045FC044641
:107190000028B6D1F378002BB3D0174802F098FA44
:1071A0003F28AED9F178204603F03EFB0028A8D056
:1071B000114802F08DFA3F28F17811D8204603F0EB
:1071C00043FB9EE72146384603F00AFB0028A2D085
:1071D000A378737023781C441D44ADB26378B8E77C
:1071E000064A2046402303F03FFB8AE7F46700206D
:1071F000F0ED00E0F66700200468002074670020CE
:1072000038B5137803F06003202B01D0002038BD7F
:10721000294C938825789D42F8D15378203B032B45
:10722000F4D8DFE803F008151E02012936D003293F
:1072300039D0012038BD01290CD00329F9D11F4BC9
:10724000002BF6D01E490020AFF30080012038BD8E
:107250000129EED111460723194A03F0AFFB0120A3
:1072600038BD01291AD00329E3D1164B55881B7864
:107270001548257113F004011CBFE94301F0010119
:1072800002F08AFB114B002BD3D0C5F3400205F06E
:1072900001010020FFF7A0F9012038BD114603F0DD
:1072A00075FB012038BD0A4B002BC2D0518800204D
:1072B000AFF30080BDE700BFF467002000000000CE
:1072C000FC670020B860002018680020D965020023
:1072D000000000002DE9F0475F4CE2788A420D463D
:1072E00080461F4659D15D4E9AB2314604F11000D6
:1072F00002F0A4FA5A4BC3B16379FF2B15D0A7B1A2
:1073000006EB070A04F1100902E056450DD0637937
:1073100016F8012B9A42F8D1484602F0D1F900281C
:10732000F3D16179AFF30080EFE74E4B23B14E48C4
:1073300002F0C6F9002863D002F066FB002862D193
:10734000A3789D4202D00120BDE8F087474B13B1DE
:107350000020AFF3008002F057FB00282BD14448F7
:1073600002F09EF90028EED1002FECD017F03F0775
:10737000E9D1A178404603F057FA0028E3D0A1787C
:1073800040463B463A4603F06FFA0028DBD1394BC2
:107390001B68DA070CD500BED6E7A3788B42D5D0A0
:1073A000344B1B68DB0703D500BE0020BDE8F08727
:1073B0000020BDE8F08702F02FFB05460028CED163
:1073C0002B4802F06DF90028C9D0A178284603F0B7
:1073D0002BFA0028C3D040222749254802F08AF919
:1073E000034600282CD02846234AA17803F03CFA13
:1073F0000028A8D11F4B1B68D907B0D500BEAEE747
:10740000AFF3008098E702F007FB0646002897D10B
:10741000E378002B94D0144802F05AF93F288FD912
:10742000E178304603F000FA002889D00E4802F0D7
:107430004FF93F28304607D8E17803F005FA7FE797
:10744000A17803F001FA8AE74023044AE17803F0C7
:107450000BFAA37875E700BFF4670020746700207B
:107460000000000000000000046800200000000090
:1074700018680020F0ED00E0B4670020704700BFFE
:1074800001207047704700BF704700BF044B0022C7
:10749000C3E90022C3E90222C3E90422704700BF06
:1074A0004C6C002001207047044B0022C3E90022ED
:1074B000C3E90222C3E90422704700BF4C6C0020DC
:1074C0002DE9F0434B79032B83B004D000242046F0
:1074D00003B0BDE8F0830B79C3EBC3041234A4B24C
:1074E000944205D9254B1B68DA07EFD500BEEDE7BE
:1074F000234A5578002D3ED0557B002DF2D102F164
:107500000C054FF4A0770E788A1992F801C0BCF1EF
:10751000210FE7D1AA608946895D80466E1CA81CB0
:107520001144CDE900061A464046032303F0B8F89B
:107530000028D7D099F80630A978012B04BF99F814
:107540000730EB700123AB7199F80220AB682A7009
:10755000B3F80730AB800029B9D00A4A40463A4414
:10756000402303F081F90028B1D1044B1B68DB07ED
:10757000ADD500BEABE715468027C4E7F0ED00E0CF
:107580004C6C0020CC6A00202DE9F047137803F002
:107590001F06012E82B003D0002002B0BDE8F087A4
:1075A000DFF80882978898F80040FFB2BC4200F0EC
:1075B000B08098F80C40BC42EED13746B4464FF04C
:1075C000C00E4FF0130A4FF0120913F060030C467F
:1075D0000546164604D1012900F0A4800120DCE70D
:1075E000202BD9D15378013B0A2BD5D801A252F8D0
:1075F00023F000BFC9760200BF760200A976020020
:10760000997502009975020099750200997502003A
:107610009975020069760200417602002176020027
:1076200001291BD00329D9D173880C2606FB0786B4
:10763000DBB260461946B371FFF720FF0120ACE7CB
:107640000129CBD173880C2202FB07871B0A6046F5
:107650001946FB71FFF714FF00289DD031462846DC
:1076600003F094F9012098E7012900F086800329AE
:10767000B4D1F48871884B4B402C4FEA112220463C
:1076800028BF402011F0FF01734407D0012C05D919
:107690001C788C4202D1013880B2013300906046E0
:1076A000FFF7D2F9012078E7012997D108EB090209
:1076B00031462846234603F081F920466DE701292B
:1076C0008CD108EB0A02F3E7012987D1F38871888E
:1076D000344F402B4FEA1122184628BF402011F0AA
:1076E000FF01774454D0012B52D9013880B2397050
:1076F0007B1C00906046FFF791F90444A3B2002B75
:1077000049D1294A1268D2077FF546AF00BE184614
:1077100043E74FF0000E7746F4464FF0070A4FF06C
:10772000060952E75378062B7FF436AF53881B0ABD
:10773000212B12D0222B7FF42FAF6046FFF766F982
:107740007B001F4408EB8708024631462846B8F8FC
:10775000043003F033F920461FE77B001F4408EB99
:107760008708D8F80820002A3FF416AF137831466E
:1077700002B0BDE8F04703F021B9F388402B3FF693
:107780000BAF084A3146724403F018F9204604E76B
:107790003B460024ADE73A463146284603F00EF951
:1077A0000120FAE6CC6A0020F0ED00E04C6C0020ED
:1077B000F0B52C4CA67865788E4283B0074610D081
:1077C000A9422CD0A07B657B88423FD0A94244D0FF
:1077D000254B1B68DA0702D4002003B0F0BD00BEC1
:1077E000FAE780264FF0400C0020A9429BB21AD045
:1077F0001E4D3544FAB9009311462B460222FFF77D
:1078000023F92A46A1783846402303F02DF80028B2
:10781000E3D1154B1B68DB07DED500BEDDE74FF07B
:10782000400C00209BB2114961444AB91A46FFF747
:1078300029FE0120D1E72A460221FFF725FEE0E7D5
:107840000A460121FFF720FE0120C6E70C344FF461
:10785000A0764FF4807C0120C7E74FF4807C0120A4
:10786000E0E700BF4C6C0020F0ED00E0CC6A0020A7
:1078700070B5194C82B000210D464FF4EC722046D1
:1078800060F003FE04F138010123802204F11000AE
:10789000009501F0C9FE04F1B80101238022009592
:1078A00004F1240001F0C0FE04F59C71012053F0A6
:1078B0004FFF04F5C4710646012053F049FF30B96B
:1078C000064B1B68DB0700D500BE02B070BDC4E9E3
:1078D0000756C4E90C05F8E7E46C0020F0ED00E081
:1078E00038B5094C206A256B20B154F055FB0023B4
:1078F000C4E907332DB1284654F04EFB0023C4E9F8
:107900000C33012038BD00BFE46C002010B5084CDA
:10791000002304F11000C4E90033C4E9023302F08B
:107920001BF804F12400BDE8104002F015B800BFB8
:10793000E46C00202DE9F0434B79012B83B004D097
:107940000025284603B0BDE8F0838B79012B0C4657
:10795000064616D049780429F2D10025032BEFD131
:10796000E379002BECD1DFF8FC8098F8013013B9F3
:1079700098F802700FB3384B1B68DB07E0D500BEE8
:10798000DEE7CB79002BDBD10B781C449DB261780C
:1079900024290BD1954202D9D2E7AA42D0D3237829
:1079A0001C442B44617824299DB2F6D00429C7D108
:1079B0006379012BC4D1A379D0E7A37888F800308C
:1079C00094F8009021794D44ADB2A14439B925E035
:1079D00099F800308F421D44ADB299441ED2AA429C
:1079E0001CD399F80130052BF2D14946304601925B
:1079F00002F0F6FE019A0028BDD099F80230D909AC
:107A000014BF88F8013088F8023099F800302179E5
:107A100001371D44FFB2ADB29944D9E70F4801F0D8
:107A200057FE3F288DD998F80210002002F0FCFE86
:107A3000002886D0094801F04BFE3F2898F8021034
:107A400003D8002002F000FF7BE7054A4023002016
:107A500002F00AFF75E700BFF0ED00E0F46C0020D3
:107A6000A46C0020E46C002000207047F8B53C4D69
:107A7000AA788A421F4612D19AB23A4905F11000FB
:107A800001F0DCFE384B13B10020AFF30080374823
:107A900001F01EFE3F282CD801242046F8BD6B784B
:107AA0008B4208D0324B1C6814F00104F5D000BEA4
:107AB00000242046F8BD064605F1240001F0F0FD43
:107AC00040BB2C4801F0ECFD0028E5D1002FE3D0AD
:107AD00017F03F07E0D16978304602F0A5FE044672
:107AE0000028D9D0697830463B463A4602F0BCFEC1
:107AF000D3E7A978002002F097FE04460028CBD0F7
:107B00001A4801F0E5FD3F28A9781ED8002002F0B0
:107B10009BFEC2E76978002002F086FE0028D0D0E4
:107B20004022154905F1240001F0E4FD034690B11F
:107B3000114A6978002002F097FE0028ACD10C4B66
:107B40001B68DB07BDD500BEBBE7064A402300200B
:107B500002F08AFEA1E7697802F076FEB1E700BF85
:107B6000E46C0020A46C002000000000F46C0020F5
:107B7000F0ED00E0086D0020646C002030B4114B83
:107B80009C689A6B93F83C5083F82C10A21A02213F
:107B900083F830109A6225B942F2050183F83E500D
:107BA000998744B13AB11A7BD20906D193F82F10C4
:107BB00030BC02F099BE30BC704793F82E1030BC38
:107BC00002F092BEBC70002038B5214B214C054616
:107BD0001BB1607BFFF736F8A8B1A06BA36894F8DF
:107BE0002F101D4A1B1AB3F5007F28BF4FF40073F6
:107BF00028469BB202F038FE20B9184B1B68DB0701
:107C000000D500BE38BDA268A36B84F83E0042F2E6
:107C10000771D31A0120A1870221A36284F82C00E6
:107C200084F83010002AEDD0002BEBD0237BDB0949
:107C300006D194F82F102846BDE8384002F054BE13
:107C400094F82E102846BDE8384002F04DBE00BF23
:107C5000456C0200BC700020BC6E0020F0ED00E01E
:107C600070B5304CE28AA36852BA92B286B005462B
:107C700012B1B3FBF2F292B2A66BD4F81110607B92
:107C80009B1BB3F5007F28BF4FF4007309BA009324
:107C9000B6FBF2F302FB13621944234BFEF79AFF83
:107CA000031E20DB94F82E200DD011469BB22846EF
:107CB0001D4A02F0D9FDA0B91C4B1B68DB0710D58B
:107CC00000BE06B070BD0724194603A88DF80C50FD
:107CD0008DF8102005938DF811308DF80D4002F0CD
:107CE000B7FB06B070BDA268A36B43F6022000216B
:107CF000D31AA08784F83E1001200221A36284F8E1
:107D00002C0084F83010002AEBD0002BE9D0237B24
:107D1000DB0914BF94F82E1094F82F10284602F0B7
:107D2000E3FDDEE7BC700020BC6E0020F0ED00E05B
:107D300010B4054C012084F83C1084F83D2084F8F0
:107D40003E305DF8044B7047BC700020402200219B
:107D5000014860F09ABB00BFBC70002040220021A7
:107D6000014860F092BB00BFBC7000204B79082B2B
:107D700001D0002070478B79062BFAD1CB79502B9C
:107D8000F7D1162A06D81C4B1B68D907F1D500BEBF
:107D90000020704770B5194D8B7885F82D300B7821
:107DA00082B005F12F0205F12E0619440223CDE918
:107DB00000261A46044602F073FC48B90E4B1B68B5
:107DC000DA0702D500BE02B070BD002002B070BD5F
:107DD000204695F82F100A4A00241F2385F83040CA
:107DE00002F042FD30B9044B1B68DB0702D500BE30
:107DF0001720E8E71720E6E7F0ED00E0BC70002070
:107E0000BC6E0020012901D001207047F0B5137825
:107E100003F07F01022985B0054606D003F0600318
:107E2000202B1AD0002005B0F0BD5478012CF5D1DC
:107E30005388002BF6D1434E918896F83030042BAE
:107E4000C9B279D096F82E408C423DD096F82F409A
:107E50008C4257D0012005B0F0BD5378FE2B16D0D0
:107E6000FF2BDFD15388002BDCD1D488A3B2002BA9
:107E7000D8D1344E1146284686F83030C6E90D3345
:107E8000B48786F83E3002F081FD0120CBE75388AD
:107E9000002BC7D1D388012BC4D12B498DF80F30CB
:107EA00000294DD00192FEF7E5FD019A0028B9D0D6
:107EB000431EDBB204AC114604F8013D28462246BD
:107EC000012302F07BFDC5E7022BC3D1B26BB3687F
:107ED0001E4F9B1AB36206F120030FCB07C73A4629
:107EE000214602F80C39032428460D2386F8304039
:107EF00002F0BAFC0028ADD1154B1B68DB0791D509
:107F000000BE90E7002BA5D1214602F0DFFC00283F
:107F1000A0D12146284602F005FD00289AD1002470
:107F200096F82F10094A86F8304028461F2302F0A1
:107F30009BFC0028E0D08DE702F0D6FC204672E7DB
:107F40000B46B7E7BC700020756A0200BC6E0020CB
:107F5000F0ED00E02DE9F041B44C94F83050012DE3
:107F60008EB01E46074645D028D3032D05D0022DDE
:107F70005FD001200EB0BDE8F08194F82E308B4226
:107F8000F7D10D2EF5D1E37B282B00F01A812A2B97
:107F900040F00D81A64B13B1607BFEF747FE002534
:107FA00094F82F10A34A84F830501F23384602F06B
:107FB0005BFC002861D094F83050D8E794F82F503B
:107FC0008D42D6D11F2B06D1DFF868829A4BD8F8A4
:107FD00000209A4271D0042394F82E1084F8303097
:107FE000384602F081FC384694F82F1002F07CFCF1
:107FF0000020BFE7B3F5007F08D9904B1B68D90775
:1080000000D500BE00200EB0BDE8F081E27BA36B7E
:10801000282A00F087802A2A00F08F80217B626B5B
:108020001E44CB09A66336D096422CD3022384F893
:10803000303094F82E10384602F074FC002898D1A5
:10804000A368A26B94F82E60934202D9217BC909E0
:108050002ED19B1A7A4AA3620FCA764D07C52A46CB
:10806000314602F80C39032538460D2384F8305088
:1080700002F0FAFB00287FF47CAF704B1B68DB0733
:10808000C0D500BE76E76D4B1B68DA0793D500BEFE
:1080900094F830506BE793B2607B664A04F10F01AD
:1080A000FEF778FD0028C0F29F80A66B626BBBE7ED
:1080B0003146384602F018FC5BE7C446BCE80F00C6
:1080C00026460FC69CE80F0007C626F8023B1B0C8D
:1080D0003370D4E90123E17B5A4E62620120002211
:1080E000282963632662A26284F82C20A26384F8A4
:1080F000300000F0AD802A2900F0DF80002B00F076
:10810000EF80227BD20940F0EB80B3F5007F00F2D4
:108110006F819BB22946474A384602F0A5FB0028EA
:10812000ABD048E7626B1E449642A663BFF47EAFB5
:10813000FFF796FD94F8305019E7E28A52BA92B2EE
:108140001AB1A168B1FBF2F292B2D4F81110394D14
:10815000B3FBF2FC09BA02FB1C32607B009661445F
:108160002B46FEF74DFD0028C0F2FB81864230D938
:10817000361A40B1A36B291813FA80F33246284609
:10818000A36360F069F9002394F82F508DF818501C
:108190000722194605A88DF8147007968DF8193036
:1081A0008DF8152002F054F994F83050DFE6264B94
:1081B000002B3FF4F4AE04F10F01607BAFF30080BD
:1081C000EDE6224B002B3FF4EAAE607BAFF300807C
:1081D000E5E6D4E90D231E449642A663BFF426AF1C
:1081E0003846FFF7F1FCE6E6A368A66B94F83C106E
:1081F00084F82C509A1B0220A26284F8300021B926
:1082000042F2050084F83E10A087002B3FF44EAFE9
:10821000002A3FF44BAF237BDB0940F0E58194F863
:108220002F10384602F060FB3FE700BFBC70002013
:108230002D6C0200BC6E002055534243F0ED00E06F
:10824000DC70002055534253000000000000000085
:10825000E28A52BA92B20BBB002A3FF4E7AE94F81E
:108260003C10A362022284F82C2084F830200029DC
:108270007FF4DFAE42F205010022A18784F83E20A0
:10828000002B3FF4D6AE237BDB0940F09A812946D0
:10829000384602F029FB94F8305068E6207BC0098C
:1082A00013D0002A00F08081B3FBF2F2002A00F024
:1082B000A3812829384694D13AE7E28A52BA92B289
:1082C000002BC9D0207BC009EBD094F83C10A362EE
:1082D000022284F82C2084F830200029CAD0D2E76A
:1082E000667B252900F22B81DFE811F022012901AC
:1082F0002901E50029012901290129012901290173
:10830000290129012901290129012901290129011D
:10831000BD0029012901290129012901290129017A
:1083200099008700290129017100290129012901EA
:1083300029014C0029012600304604AA05A9FEF7B0
:1083400017FC059B002B00F04481BDF81020002A8B
:1083500000F03F81013B1BBA12BAC8E90032082085
:10836000A368002B44D0984228BF184683B26063AC
:10837000A64A94F82E10384602F076FA00283FF408
:108380007CAE18E605AD00230DF10E02304604A9BF
:108390006B600593AB60FEF7EBFB049A002A00F0DC
:1083A0001881BDF80E30002B00F0138112BA08219D
:1083B00006925BBA0222ADF81E308DF817108DF8C8
:1083C0001C2095E8070088E807000C20C8E7904BC0
:1083D00003B33046227DE17CAFF30080D0B994F83E
:1083E0003C302BB943F602220023A28784F83E30AA
:1083F00001213846FFF7C2FBDDE5864B53B1E17C36
:108400003046C1F3400301F001020909FEF7CCFB3D
:108410000028E4D0A368002B3FF408AEE8E79DF8FD
:1084200016307D49002203F0800362F3C7138DF8F4
:10843000163003238DF815208DF817208DF8143091
:10844000002900F0E1803046FEF7FCFB9DF8163075
:1084500080F0010060F3C7138DF81630059BC8F853
:10846000003004207CE74FF0203302250022CDE9C4
:108470000522304607A909AA08934FF0800C0793FC
:1084800009930D93CDE90A330C931F260DAB8DF89C
:1084900016508DF8175005AD8DF818608DF815C081
:1084A000FEF7F0FA0FCD594E0FC60FCD0FC62B6851
:1084B0003360242054E794F83C2094F83D0094F86D
:1084C0003E10DFF848C1DFF858E14FF000084FF0E8
:1084D0000003CDE90588CDE9078862F303038DF831
:1084E0001630F0220A23ADF824808DF820008DF894
:1084F00021108DF814208DF81B3005AD0FCDACE8A0
:108500000F002B68ACF80030BEF1000F76D0ACF154
:10851000100130464FF40072AFF300800028A4F839
:108520003C8084F83E800FDB00283FF473AF17E7F0
:108530003046FEF7F9FA00283FF451AF6AE794F8A5
:108540003C30002B7FF454AFA38E304A3349607B1C
:10855000FEF720FB0028FFF64BAF00283FF45AAF90
:10856000FEE6A36BA2681E4443F602200021931B83
:10857000A08784F83E1001200221A663A36284F83C
:108580002C0084F83010002A3FF453AD002B3FF448
:1085900050AD237BDB0914D194F82F10384602F03C
:1085A000A3F994F83050E2E4012294F83C1084F8E6
:1085B0002C200222A36284F8302000293FF45AAE16
:1085C0005EE694F82E10384602F08EF994F830509A
:1085D000CDE494F83C30002B7FF40AAF43F602223E
:1085E00084F83E30A28703E794F82E10384602F054
:1085F0007BF9D4E90D2617E50222D6E7A4F83CE082
:1086000084F83EE01220ABE601201FE7BC6E00209C
:1086100000000000A96B0200456C0200CB70002036
:108620000000000070B5134C134E84B020464FF488
:10863000AE7200215FF029FF4025002304F58E7201
:108640000092CDE901561A46194604F1B00003958F
:1086500004F068F92E4404F170020023CDE90025EE
:10866000CDE90265201D1946012204F05BF904B032
:1086700070BD00BF7C710020FC70002010B5054C5F
:1086800004F1B00004F07AF9201D04F077F901201C
:1086900010BD00BF7C71002038B5074C2046002576
:1086A00000F8B85B01F058F904F10C0001F054F93E
:1086B00084F8B150657138BD7C7100204B79FF2B77
:1086C00001D0002070472DE9F04FDFF824B19BF86E
:1086D000B13083B04BBB9BF8053033BB0B788A4677
:1086E0000AEB02050AEB030489788BF80010A54217
:1086F000064614D91AF80320A3189D420FD36278B6
:10870000042A0CD00B2A0AD0052A0BF1B8080BF169
:10871000B0070BF10C0917D09D421C4609D8A4EBF9
:108720000A0080B203B0BDE8F08F002003B0BDE8BE
:10873000F08F1A7813449D42F1D36278042AEED068
:108740000B2AECD0052AE7D12146304602F048F842
:10875000002843D0A378DB0905D19BF8B1301BB3C7
:108760002278A318D8E79BF80530002BF8D14846AB
:10877000019301F0F1F8A2788BF80520A2889BF80C
:1087800004C0019B1849C2F30A02A2F50072B2FAB2
:1087900082F2520962F3410C18468BF804C004F0CF
:1087A00037F92278A318B7E7404601F0D5F8A37847
:1087B0008BF8B130A3889BF8B020C3F30A03A3F56C
:1087C0000073B3FA83F35B0963F341023946304621
:1087D0008BF8B02004F064F90028C1D1034B1B686A
:1087E000DB07A2D500BEA1E780710020F0ED00E01C
:1087F0007C71002070B51C4C94F8B1208A4205466B
:108800001E460FD1B4F8BC20F2B9184B23B1B2B256
:1088100017490020AFF300802846164904F040F9BC
:10882000012070BD63798B4201D0002070BD124BD6
:108830001BB1B1B20020AFF300801049284604F00C
:10884000E7F848B1012070BDB2B2D4F8B41004F119
:10885000B80000F0F3FFD8E732462846074904F095
:1088600099F8012070BD00BF7C710020000000005D
:10887000FC7000202C72002000000000807100209D
:10888000F8B50E688D88B7783544AE420BD23B46BA
:108890009F42344603D10BE06378042B05D0237844
:1088A0001C44A542F8D80020F8BDA3789F42F6D119
:1088B000E3789A42F3D1A542F5D9237D012B06D95D
:1088C000144B1B68DA07EED500BE0020ECE72379D5
:1088D0000D46DBB1012BE6D12278E389617A13449E
:1088E000114423442144994204D3DCE70A7811441B
:1088F0008B42D8D94A78052AF8D101F071FF28B9FE
:10890000044B1B68DB07CED500BEF8BDA41BEC8072
:108910000120F8BDF0ED00E0C28832B9654B1B685C
:10892000DB0700D500BE00207047F0B40378624832
:1089300003EB830403EB4403C058831803D08E7801
:108940001C7BA64207D95B4B1B68D90700D500BE2C
:108950000020F0BC70472EB9012C01D90120F8E7A6
:1089600001268E7001248C60C1F80E404C770025E2
:108970006FF03F0481F822508C766FF003056FF0A2
:108980006404CD760C774D4DC1F81E50082481F853
:108990002340825CB3F80D4014441C441344A342AA
:1089A000D1D2474F9D78102D0CD827FA05F0C0433F
:1089B00010F0010006D1DA78964203D107E05A7828
:1089C000242AEFD01A7813449C42F8D8BBE79C4283
:1089D000B9D0062D06D0102D04D0042DB9D1012216
:1089E00048730A73CF781A79974218D81FB9012AA9
:1089F000B4D80127CF701A781A44A2420FD29678C1
:108A000006F0FD0CBCF1050F0FD0112E03D10CE0C8
:108A10005678242EF3D0167832449442F8D8254B59
:108A20001B68DA0794D500BE93E7D678B742F2D137
:108A30009442F4D0D1F812408CB9062D30D0102DCC
:108A40002ED0042D09D1B2F80560B2F807505C7D34
:108A500005FB06F304FB03F4E408C1F812404B687D
:108A600063B9557E012D3FF679AFD2F81A3025B99A
:108A7000D2F81E209A427FF471AF4B60114AA2FBDC
:108A800003235A0BCBD0631E1344B3FBF2F3023320
:108A9000B3F5807F28BF4FF48073C1F816305DE7CF
:108AA000B2F80530B2F8074004FB03F42401E408EF
:108AB000D3E700BFF0ED00E0D87200200301010110
:108AC000501001005917B7D12DE9F84F0B785D4CC4
:108AD00003EB83050E4603EB45030989E7589146EE
:108AE000804679B13944CB7803F00303012B00F0C1
:108AF0009480738933B13B44DA7802F00302012A8F
:108B000000F091807488B58800233C44B381F381E0
:108B100033827382B382F3823D44A278AC4238BF81
:108B2000134609D29A4203D10CE06378042B06D095
:108B300023781C44A542F8D80020BDE8F88FA3781C
:108B40009A42F5D1E3789945F2D1A542F4D994F847
:108B500004A0BAF1020F15D8E31BF380B9F1000F9E
:108B600016D023781C44BAF1000F4CD04FF0000B04
:108B700006E06378052B28D0042B03D023781C440F
:108B8000A542F6D8304B1B68DA07D5D500BED3E72F
:108B9000737F012B12D006F11E03494686F81D9003
:108BA000A6F81890A6F81A90184630225FF06DFCCF
:108BB00001463046FFF7B0FE0028BDD023781C44A4
:108BC000BAF1000FD2D10120B7E7E37803F0030335
:108BD000B9F1000F01D0012B18D0022BACD12146E6
:108BE000404601F0FDFD28B306EB4B03E21B1A8162
:108BF00022780BF101039A4514444FF0010BBFD8C2
:108C0000B9F1000FDFD002237377DCE7A388B269E4
:108C1000C3F30A039342E2D28EE7002333818978BB
:108C200001F08EFE65E7002272819978404601F0DE
:108C300087FE67E7044B1B68DB077FF57DAF00BE4F
:108C40007BE700BFD8720020F0ED00E010B4064CC6
:108C500006480023C4E900331946C4F807304E2201
:108C60005DF8044B5FF011BCD8720020E473002063
:108C70000120704710B4064C06480023C4E90033B5
:108C80001946C4F807304E225DF8044B5FF0FDBB77
:108C9000D8720020E47300202DE9F0414B790E2BAF
:108CA00004D04FF000084046BDE8F0818B79012BDD
:108CB000F7D1CB79012BF4D13E4E33682BB13E4B2B
:108CC0001B68DB07EDD500BEEBE714460F461A46DE
:108CD000314605463760B480FFF7D2FD0028E0D06A
:108CE000F2883368B97813443C44A74293F814C01F
:108CF0003B4605D308E05A78042A4DD00B2A4BD0C6
:108D00001A7813449C42F6D8BCF1000F4ED02B4980
:108D10004A88002AD3D1D81B1FFA80F83272A1F8F2
:108D200002809C4293F802E00A8098BF034605D86F
:108D30000BE05A78042A2BD00B2A29D01A78134436
:108D40009C42F6D8DB1B1FFA83F80022BCF1010F0E
:108D5000A1F804804A77B2D117FA80F017FA83F3AA
:108D6000984281780AD282788A4203D118E0427808
:108D7000042AF8D0027810448342F8D8284600220A
:108D80000E49FFF7A1FE00288BD0A6F804808AE7E1
:108D90009A787245D2D0D5E79A788A42B0D0B3E7B4
:108DA000C278012AE6D18342EFD1E7E7DB1B1FFA45
:108DB00083F8EAE7D8720020F0ED00E0E4730020C9
:108DC0002DE9F047167806F01F04012C8CB004D072
:108DD000002420460CB0BDE8F087DFF8F892B2F826
:108DE00004C0D9F80070804615465FFA8CF317B1BD
:108DF000BA789A422CD0B44F7C88002CE9D03A78CB
:108E000002EB820002EB400259F802E07444A278BF
:108E10009A42DDD1C6F34116F3B2002B00F09C80DC
:108E2000012B12D15FEA1C2C0FD16B881B0A022B7D
:108E300000F02E81062B00F01781012B00F0F58049
:108E4000A24B1B68DB0700D500BE07233B77BFE7BB
:108E5000C6F34116F4B2002C47D0012C25D15FEAAD
:108E60001C2C26D0B9F80620BB18B95CDA8911444D
:108E700019448B420ED29A78023A052A06D8DA783B
:108E8000624503D107E05A78242AF4D01A781344B3
:108E90009942F8D849B1002389F80930012498E7AC
:108EA0008A4B1B68D90700D500BE072389F8093013
:108EB0008EE76B881B0A012B00F09580022BEFD107
:108EC0006B78812B00F04781862BE9D10129E2D113
:108ED0000B46404629467E4A01F070FD0028DAD153
:108EE000FF2389F80930002473E76B780A2B4AD0F6
:108EF0000B2B3ED10129CED1EB88002BF0D1B9F854
:108F00000630FA181179A9B1F85CD189537A014475
:108F1000034413440A44934205D395E119780B4462
:108F20009A4240F2918159780529F7D199784046C3
:108F300001F006FD0026A9F806606A8865494046EA
:108F4000FFF79EFC04460028CAD02946404601F09F
:108F50001DFD89F809603CE76B780A2B27D00B2BA5
:108F60007FF46EAF012900F0BD8000233B77012420
:108F70002FE7564B1B6813F001032FD107221C4625
:108F800089F8092025E7012985D1EB88012BA7D194
:108F9000B9F80620BF18A3D00CAAF97802F8301D42
:108FA000294601F00BFD04460028D2D198E701299B
:108FB000DBD1EB88012B35D1FB889BB31EEB030380
:108FC00030D00CAADB7802F8303D40460B462946EB
:108FD00001F0F4FC044628B33E77FAE600BE07230E
:108FE00089F80930F5E66B78812B00F0D180862B6B
:108FF00000F0BE80012B7FF453AF012900F0CB803D
:1090000002297FF448AF344B002B3FF444AF99F86A
:109010000A100020AFF30080B0FA80F489F809004C
:109020006409D6E6FF233B77D2E67B7F0BB187F856
:109030001DC06C78842C61D8822C65D2012C00F084
:109040000A81812C7FF4FCAE01298ED1EB883BB1E3
:10905000294640463023214A01F0B0FC002884D143
:10906000FF233B770024B4E66B78812B00F0A180CE
:10907000862B7FF4E5AE01297FF477AF2946404681
:109080000123134A01F09AFC00287FF46EAFE7E752
:109090006B78812BD8D040F2B080852B00F0978080
:1090A000862B7FF4CDAE01297FF45FAFEB88012BD7
:1090B000D6D10B4640462946094A01F07FFC0028DC
:1090C0007FF453AFCCE700BFE4730020F0ED00E085
:1090D000F9D30800D87200200000000002740020BC
:1090E000FAD308006A8839464046FFF7EDFC0028AD
:1090F00098D02946404601F049FC36E7862CD2D06C
:1091000065D3872C7FF49CAE01297FF42EAFEB88CA
:10911000002BA5D0B64EE94606F1300A30687168DA
:10912000B268F368CC46ACE80F0010365645E1460D
:10913000F4D19DF80210002940F09F80832C00F0AC
:109140008381872C00F06481822C00F061810823E8
:109150003B7700243DE601297FF49DAE2946404639
:109160000123A44A01F02AFC00287FF494AEB7E65C
:1091700001297FF490AEEB88012B7FF4B1AE294634
:1091800040469D4A01F01AFC00287FF484AEA7E611
:1091900001297FF480AEEB88012B7FF4A1AE294634
:1091A00040460123954A01F009FC00287FF473AE84
:1091B00096E601297FF4D9AE0B464046294607F1D1
:1091C0001C0201F0FBFB00287FF4CFAE48E7012929
:1091D0007FF4CBAEEB88022B7FF442AF0CAA302198
:1091E00022F8301D4046294601F0E8FB04460028DD
:1091F0003FF436AF00233B77EBE5012B7FF420AE45
:1092000001293FF425AF02297FF4AFAE7849A1F1DF
:109210001E00FFF781FB044660B3794B7A6BBA619D
:109220003BB1734A79783878AFF3008000287FF437
:109230009CAE7449002302204FF480720880C7E975
:1092400003337B61BA83C4E56F4B1B68D8077FF596
:1092500047AE00BE44E601293FF4FAAE02297FF48E
:1092600084AE6349A1F11E00FFF756FB04460028B7
:109270007FF47BAE08233B77ABE59DF80300002825
:109280007FD1FA88002A3AD01EEB020337D01EF8AD
:109290000220B3F80D005D4E104418441344984268
:1092A0000FD99A78102A04D826FA02F2D20700F1D0
:1092B000D5801A7813449842F1D95A78242AF8D1E3
:1092C000EDE70346832C5AD0872C4CD0822C7FF4B8
:1092D0003EAF01218DF803101A781A44904237D915
:1092E000947804F0FD06052E10D0112C0ED01478C1
:1092F00022449042F2D95478242CF8D1EEE7424B24
:109300001B68D9077FF523AF00BE20E7D478A142C0
:10931000EDD1997806291DD010291BD004297FF49E
:1093200016AFB2F80510B2F807205B7D02FB01F220
:1093300003FB02F3DB08CDF812306A4629464046AB
:10934000302301F03BFB044600283FF489AE51E78F
:109350000246DEE7B2F80510B2F8073003FB01F36E
:109360001B01DB08E7E79A78062A06D0102A02D00C
:10937000042A7FF4ECAE997DACE79979AAE71979D4
:10938000A8E7019B002BD8D1FA88002AB7D01EEBA2
:109390000203B4D01EF802E0B3F80D20DFF86CC071
:1093A00072449E1873449E420ED99A78102A03D8AC
:1093B0002CFA02F2D20756D41A7813449E42F2D9FC
:1093C0005A78242AF8D1EEE733461A7813449E429D
:1093D00064D99A7802F0FD01052948D0112A46D0B7
:1093E0001A7813449E42F2D95A78242AF8D1EEE72B
:1093F00002740020E1720020FAD30800E27200201B
:1094000000000000E4720020F0ED00E050100100C8
:1094100001238DF8023001234FF001120293002343
:109420000392ADF810304FF6C0428DF8223040F272
:109430009B13ADF81A20ADF81C30404ACDF81E2021
:1094400008238DF8233078E7FB88002BE3D01EEB50
:109450000303E0D01B7B8DF80230DCE7DA78914221
:109460007FF427AF2EE7DA789142A5D1ADE7DA781D
:109470009042B5D1823C052C3FF669AE01A252F86C
:1094800024F000BF05950200E9940200CB9402008D
:109490004F9102004F910200A19402003346E9E788
:1094A000D3F8151042F21073B1FBF3F301910029C8
:1094B0003ED0DDF812208BB9931CB3F5807F28BF16
:1094C0004FF48073CDF8163037E75A7E72BBD3F86D
:1094D000221042F21073B1FBF3F3E7E7013A1A44AA
:1094E000B2FBF3F30233E8E75A7ECAB1053203EB6D
:1094F0008202D2F80210D3F81A3042F21072B3FB93
:10950000F2F3D3E75A7E72B1053203EB8202D2F84E
:109510000220D3F81A1042F21073B2FBF3F3C5E73E
:10952000D3F81E10E7E7D3F81E20F2E700230193DB
:109530000023ADF81630ADF81830FEE60301010146
:109540002DE9F84F334C238953B12278324F02EB87
:10955000820502EB45057D592B449F788F420AD046
:109560002E4B1B68DB0703D500BE0020BDE8F88F3B
:109570000020BDE8F88FD4E904369E4205460BD39F
:1095800027490023C4E90333636119B161781046A8
:10959000AFF300800120E9E701F046F90028E7D0A9
:1095A000DFF88090A36999F80000D4E9042BA2EBBE
:1095B0000B0808EB00069E4228BF1E46B04213D996
:1095C000164B1B6813F0010301D000BE002339467F
:1095D0002846144A01F048F90028DBD10F4B1B68DC
:1095E000DA07C5D500BEC1E7E168A6EB000A594419
:1095F000484452465EF025FF0BEB0A03D0456361F9
:10960000B3B2E4D199F8012042F0020289F80120B6
:10961000DDE700BFE4730020D8720020F0ED00E029
:1096200000000000E47200202DE9F041B2F5004F87
:109630009DF8188030D80446C0681E460F4615466F
:1096400018B14FF0FF3152F0F1FA206918B14FF024
:10965000FF3152F0EBFAE288E068276066F30E0211
:10966000C2F30721002368F3C711E2806381A5805C
:10967000E171238118B11A46194651F08FFE206915
:1096800038B100231A46194651F088FE0120BDE882
:10969000F0810120BDE8F0810020BDE8F08100BF2D
:1096A00003894289808892B29BB2934236BFC2EB53
:1096B00040029B1A9B189BB2984228BF18467047DD
:1096C000028943899BB2981AB0FA80F0400970472A
:1096D00003894289808892B29BB2934236BFC2EB23
:1096E00040029B1A9B189BB2984286BFC01A80B258
:1096F000002070472DE9F843054600690E461746DD
:1097000018B14FF0FF3152F091FA2B896989A8887E
:109710009BB289B28B4236BFC1EB40045C1AE4189D
:10972000A4B2002C4AD0A04206D283422CBF191A00
:10973000191889B269810446BC4228BF3C46884258
:10974000A4B203D8091A89B28842FBD9EA882B68E7
:10975000401AC2F30E0887B21FFA88F2BC4202FB1D
:10976000013125D917FB08F91FFA89F94A46304615
:109770005EF067FEE21B12FB08F206EB090092B2F4
:1097800029685EF05EFE6A89A88892B211198BB2D0
:109790009A4215D940001B1A9BB228696B8120B1EF
:1097A00000231A46194651F0F9FD2046BDE8F8831A
:1097B00002FB04F230465EF044FEE4E769898BB2B6
:1097C00040008342E9DBE6E738B5054600690C4610
:1097D00018B14FF0FF3152F029FA29896B89AA8814
:1097E00089B29BB2994236BFC3EB4200C81A4018F7
:1097F00080B200B3824209D291422CBF8B1A8B18DF
:109800009BB29A426B8103D89B1A9BB29A42FBD9B6
:10981000EA882968C2F30E02204602FB03115EF0BB
:1098200010FE0124286920B100231A46194651F080
:10983000B5FD204638BD0446F4E700BF2DE9F047EA
:109840001446002A4FD00546C0680F4618B14FF0A5
:10985000FF3152F0EBF9EA792E896989AB88D20998
:10986000B6B289B242D18E4236BFC1EB4301711A02
:10987000891989B2994252D2591A89B28C42E88820
:1098800028BF0C46C0F30E08B342304603D8C01AB6
:1098900080B29842FBD21B1A2A681FFA83F9A145AD
:1098A00008FB002047D219FB08FA1FFA8AFA524631
:1098B00039465EF0C6FDA4EB090212FB08F207EB85
:1098C0000A0192B228685EF0BCFDA3199BB2AA8877
:1098D000B3424FEA420201D3934201DB9B1A9BB28F
:1098E000E8682B81F8B92046BDE8F087E8889C42FB
:1098F000C0F30E080FD28E4223D3721A92B25800D0
:1099000022448242C0DBCE18361BB6B2B14220D907
:10991000361AB6B2B8E7E41A08FB0477B3B9E868B8
:1099200000240028DFD000231A46194651F036FDE6
:109930002046BDE8F08708FB04F239465EF081FD61
:10994000C3E75800421A324492B2D9E70E461C4689
:1099500098E7B04298DCDBE710B50446C06818B160
:109960004FF0FF3152F062F9206918B14FF0FF312A
:1099700052F05CF9E06800236381238118B11A4634
:10998000194651F00BFD206920B100231A461946F3
:1099900051F004FD012010BD38B5C379B1EBD31FE0
:1099A0001FD00446C0680D4618B14FF0FF3152F089
:1099B0003DF9206918B14FF0FF3152F037F9E379E2
:1099C000E06865F3C713E37120B100231A46194616
:1099D00051F0E4FC206920B100231A46194651F0E9
:1099E000DDFC012038BD00BF704700BF704700BFDD
:1099F0000020704700207047704700BF704700BFCD
:109A0000704700BF704700BF024B5878003018BF46
:109A1000012070478C740020024B1878C0F380003E
:109A2000704700BF8C740020024B1878FF3818BFB5
:109A300001207047186100202DE9F047374E337838
:109A4000FF2B82B004D00125284602B0BDE8F08784
:109A5000002946D0382288460746002130485EF06B
:109A600014FD304B3049002501201D7051F070FE6F
:109A70002E4B1860002834D02D4C2346626833F8F2
:109A80000C0B6188009551F0E5FBA168054652F08A
:109A9000A7FA284B1D6075B3274B23B12748AFF3B6
:109AA0000080274B1860254CDFF89CA02278DFF857
:109AB000909000252B460EE0D9F8003013EB4513AB
:109AC0000FD05B686BB1984722780135EDB2511D1C
:109AD000A9422B4615DBAA42EED89B1A0AEB431388
:109AE000EFE7184B1B68DA0700D500BE00252846B3
:109AF00002B0BDE8F087134B1B68DB07F6D500BE4C
:109B0000A2E741463846377001F050FE054600286E
:109B1000F1D0384601F04CFE96E700BF18610020F6
:109B20008C7400208C7500203C740020C4740020CC
:109B3000BC600020C87400200000000038740020C1
:109B400034740020F0ED00E0FCD30800B94B1B7822
:109B5000FF2B00F0A1812DE9F04F04468BB04FF4AC
:109B60007A7200238002A10D5EF078F9B24DDFF821
:109B7000E4B2B24E8246671C286800F02481002CB3
:109B800000F02181BAF1000F14BF5246012207A94B
:109B900051F0BAFEC0B19DF81D30013B072B00F219
:109BA0001481DFE813F0F200D300CA00BF00B70051
:109BB000410014000800089B0BB1099898472868D9
:109BC00052F0E0F90028D6D10BB0BDE8F08F9DF837
:109BD00020109B4B01F07F0703EB470303EBD113EE
:109BE00093F826006FF3000083F8260093F8260010
:109BF0006FF3820083F82600002F00F04581914A20
:109C00001B7D12789342C0F03381501D9842C0F200
:109C100034819B1A0BEB43139F699DF82120099B0C
:109C20009DF81C00B847CAE7874A1378002B00F05C
:109C300024811378013BDBB21370137803F0FF002B
:109C4000002BBCD1DFF8F8919DF81C8099F800300A
:109C500043F0010389F8003099F8263060F30003DF
:109C600089F8263099F8263060F3820389F8263087
:109C700099F8273060F3000389F8273099F82730E6
:109C800060F3820389F8273000F002FF9DF820304E
:109C900003F06002602A00F00681402A00F00A8189
:109CA00003F01F03012B00F0D581C0F01281022BBD
:109CB00040F0F9809DF8241001F07F07082F00F292
:109CC000F2807B00C80901934B44034400905D4837
:109CD0001F7D03789F4280F00F82336803EB4717A4
:109CE000002A00F0108257B1786900F0D1FE7B693C
:109CF000404608AA0121984700287FF460AF9DF8EC
:109D00001C00002101F0BEFF80219DF81C0001F025
:109D1000B9FF54E74A4B1B78D8077FF550AFFFF7E0
:109D200071FE4CE7464B1A78D7077FF548AF187895
:109D3000C0F3C000FFF764FE41E7414BDB78D90771
:109D40007FF53DAF0898FFF751FE38E73D4F9DF88E
:109D50001C903A780023984610E0336813EB4813C0
:109D600000F08080DB68484698473A7808F101089F
:109D70005FFA88F8511D8845434645DC9045A3EBC2
:109D80000203EAD30BEB4313ECE72E4F9DF81C9034
:109D90003A78002398460FE0336813EB48135BD002
:109DA000DB68484698473A7808F101085FFA88F876
:109DB000511D884543460FDC9045A3EB0203EBD3CE
:109DC0000BEB4313ECE72246E1E6204B1B68DA0776
:109DD0007FF5F5AE00BEF2E63822002118485EF0AD
:109DE00054FB1B4A4FF0FF33C2E90533C2E900338D
:109DF000C2E90233D3611384136100F03FFE104BBC
:109E00009DF820209A70DAE6382200210C485EF096
:109E10003CFB0F4A4FF0FF33C2E90533C2E9003380
:109E2000C2E90233D3611384136100F027FEFFF708
:109E3000E5FDC4E618610020C874002034740020D9
:109E40008C740020387400208C750020F0ED00E048
:109E500090740020FCD30800A44B1B68D907CCD514
:109E600000BECAE7A14B1B68DA07DED500BEDCE7FF
:109E7000326812EB43137FF4CFAE9C4B1B68DB07B9
:109E80007FF5A2AE00BE9FE6099B9DF821209DF8BC
:109E90001C0000F013FE92E67047FCF7F3FC02464C
:109EA000002840F0E981914B1B68DA077FF527AF66
:109EB00000BE24E78E4800283FF421AF00F0E8FD03
:109EC000404608AA0121FCF725FF00287FF477AE61
:109ED00015E7202A00F0F180002AE4D19DF8213016
:109EE000092BE0D801A252F823F000BF13A0020012
:109EF000F39F0200A79E020035A00200A79E020069
:109F0000D59F0200819F0200A79E02006B9F020066
:109F1000159F02009DF8223001931A4699F80130EE
:109F20009A4200F0548199F80130002B40F054819E
:109F3000019B89F80130002B00F04781581EC0B208
:109F4000FCF7A0FC18B14378022B00F0C181674BED
:109F50001B68DB0700D500BE644B1B68D80700D523
:109F600000BE002389F80130C9E60AAA99F8013039
:109F700002F80E3D4046012308A900F01FFD1EE631
:109F8000BDF82200030A5A1EC0B20E2A3FF6B7AE31
:109F900001A151F822F000BF8BA2020067A20200CB
:109FA00057A20200FF9C0200FF9C020039A202009F
:109FB00067A20200FF9C0200FF9C0200FF9C0200BF
:109FC000FF9C0200FF9C0200FF9C0200FF9C02001D
:109FD000BBA2020008A800F061FD40469DF82210D7
:109FE00001F0ECFB99F8003043F0020389F80030EF
:109FF000E5E5BDF82230012B7FF481AE99F8003001
:10A0000040466FF3C30308A989F8003000F0BEFC96
:10A01000D5E599F80030990801F00201C3F3401327
:10A020000AAA0B4322F80E3D4046022308A900F07D
:10A03000C5FCC4E5BDF82230012B7FF460AE99F871
:10A040000030404643F0080308A989F8003000F0CA
:10A050009DFCB4E59DF824300F2B3FF650AE4B44E9
:10A06000244A1B791778BB4238D2376817EB43175D
:10A070003FF445AE786900F00BFD7B6908AA012129
:10A080004046984700287FF49AAD9DF8203013F0A1
:10A0900060077FF434AE9DF821300A3B012B3FF678
:10A0A0002EAE00F0F5FC9DF821300A2B00F0FC806C
:10A0B00008A9404600F06AFC81E59DF824300F2B8A
:10A0C0003FF61DAE4B440B4A1B791778BB4260D25A
:10A0D000376817EB43173FF412AE05E67A1D9A4234
:10A0E000FFF60DAEDB1B0BEB4317C3E7F0ED00E013
:10A0F000156D020038740020581DB84239DA002A64
:10A100007FF4FDAD17469DF82130012B03D036D3E7
:10A11000032B7FF4C8AEBDF822200292AAB9B84A38
:10A12000012B10783DD001F0ADFD019B009A4B440E
:10A13000134493F8262042F0020283F8262093F875
:10A14000262042F0010283F82620002F3FF437AD8D
:10A15000786900F09DFC7B69012108AA4046984778
:10A16000002000F095FC99F82730D9073FF527AD7E
:10A170009EE7FB1A0BEB4317002AC4D0B4E5019B02
:10A18000009A4B44134420330AAA9B79C3F340033B
:10A1900048E77A1D9A42FFF6B2ADDB1B0BEB431783
:10A1A000A2E501F097FD019B009A02994B441344EC
:10A1B00093F8262061F3410283F8262093F82620A5
:10A1C00061F3000283F82620BFE7FFF717FC404643
:10A1D00008A900F0DBFBF2E40021404601F000FB9F
:10A1E000404601F09FFB874F99F80230029300230D
:10A1F00000943A781C460CE00BEB4313DB684046B6
:10A2000098473A780134E4B2501D8442234600F363
:10A21000CE809442A3EB0203EED2336813EB4413D7
:10A22000ECD1794B009C1B68DB0700D500BE9DF884
:10A23000083089F802307BE6FFF7DAFB0246002897
:10A240003FF45DAD4046137808A900F0B7FB002845
:10A250007FF4B5AC53E5BDF82410FCF719FB0246BA
:10A260000028EFD14BE5022B3FF417AEFFF7C2FBFE
:10A27000024600283FF443AD4046538808A900F049
:10A280009DFB00287FF49BAC39E5FCF7F7FA02460A
:10A2900000283FF408AE4046122308A900F08EFBC8
:10A2A00000287FF48CAC2AE50AAA08A902F80E7DE2
:10A2B0004046012300F082FB81E4544B002B3FF425
:10A2C0001EADFCF723FD024600283FF418ADD3E78E
:10A2D000C27999F80030511161F30413921162F3BD
:10A2E000451389F800304388CDF81080CDE900A4EB
:10A2F000C318039300F10907039BBB4237D97B784E
:10A300000B2B03BF3B7897F803A0FF184FF0010A0F
:10A310007B78042B43D1039B3A4ACDF814A0DB1B76
:10A3200000219BB20291127888469A4617E0346861
:10A3300014EB481433D052463946049823699847A1
:10A34000082808F1010201D9824543D22D4B5FFA5A
:10A3500082F81A78CDF80880511D88451CDC029BD4
:10A360009045A3EB0202E2D30BEB4214E3E7DDF8E6
:10A370001080DDE900A4FFF73FFB28E702464346D3
:10A3800004463946224802F0B1FA1E4B029A1B7865
:10A39000053393422744AFDADDE900A4D7E51A4B31
:10A3A0001B68DF07DDE900A47FF5D6ADD3E53822D1
:10A3B00000211848009C5EF068F8174A4FF0FF3300
:10A3C000C2E90533D3611384C2E90033C2E9023321
:10A3D00013612CE7DDF814A0BAF1010F1ED00021A3
:10A3E000CBB2534501F10101C8D2BA78134459FAEE
:10A3F00083F31A79FF2AD2D183F80480F0E700BFF3
:10A400001861002038740020F0ED00E00D6D0200AE
:10A41000A07400208C7400209074002023690A4AE4
:10A420000A498B4208BF4FF0020A9342D7D17B7989
:10A43000012BD4D1BB79012BD1D1FB79002B08BFE3
:10A440004FF0020ACBE700BF35790200F570020039
:10A450002DE9F0434378023B85B005460E46042BB8
:10A460000CD8DFE803F0495D037E3F00844B1A7887
:10A47000D70715D51A7842F004021A70814B186874
:10A480008EB933464FF0FF32294650F087FF003037
:10A4900018BF0120F0B97C4B1B68DB0700D500BE5C
:10A4A00005B0BDE8F08304AA002342F80C3D29461C
:10A4B00051F084F9019B43B1744B4FF080525A60C4
:10A4C00040BFBFF34F8FBFF36F8F003018BF012025
:10A4D0000028E0D0324669782878FFF785FA05B081
:10A4E000BDE8F0836A4A13780133DBB21370654B21
:10A4F0001868002ED7D1C4E7614B1A786FF30002B9
:10A500001A701A7800216FF341021A7059701A7884
:10A5100061F382021A705B4B1868002EC3D1B0E75A
:10A520005C4FDFF874913978DFF87081002423469E
:10A530000AE0D8F8003013EB44130AD10134E4B236
:10A540004A1DA242234615DB8C42F2D35B1A09EB6B
:10A550004313DB69002BF1D0696828789847397874
:10A56000ECE7474B1A78D4079AD51A786FF3820232
:10A570001A7083E7424C237858072FD52378414936
:10A580006FF3820323702B788DF8043005220023AB
:10A59000CDF80A30CDF80630ADF80E3008688DF8E9
:10A5A0000520002E59D004AA01A942F8103D51F00F
:10A5B00005F9009B43B1354B4FF080525A6040BFC4
:10A5C000BFF34F8FBFF36F8F003018BF01200028FB
:10A5D0004DD12D4B1B68D90700D500BEE378DA07B3
:10A5E0007FF55EAF274A2B78696810688DF80430D4
:10A5F00003220023CDF80A30CDF80630ADF80E3036
:10A6000002918DF80520F6B104AA01A942F8103D87
:10A6100051F0D4F8009B43B11C4B4FF080525A606C
:10A6200040BFBFF34F8FBFF36F8F003018BF0120C3
:10A6300000283FF430AF32469DF805109DF8040025
:10A64000FFF7D2F92CE733464FF0FF3201A950F063
:10A65000A5FE003018BF0120EAE733464FF0FF3275
:10A6600001A950F09BFE003018BF0120AFE7324631
:10A670009DF805109DF80400FFF7B6F9AEE700BF9E
:10A680008C740020C8740020F0ED00E000ED00E0C4
:10A690008C75002038740020FCD30800347400202E
:10A6A0002DE9F84F0A9F002A4CD090464A78052A97
:10A6B0000C460ED1CE7806F00306B34209D18A7853
:10A6C00002F07F02082A0DD9204B1B68DA0700D55B
:10A6D00000BE1E4B1B68DB0702D40020BDE8F88FCC
:10A6E00000BEFAE7DFF868B0DFF868A09BF80090DA
:10A6F00000250EE06278052AEBD1E27802F0030231
:10A70000B242E6D1A27802F07F02082ADCD89BF898
:10A7100000909AF802100022204602F095F80028D6
:10A72000D2D04846214601F06FF80028D1D0A27857
:10A73000D30916BF0B9B3A701A7022780135454534
:10A740001444D7D10120BDE8F88F00BFF0ED00E040
:10A75000186100208C74002030B51E4D85B008248F
:10A7600000230290019303918DF805402868144658
:10A7700082B9134601A94FF0FF3250F00FFE0030AE
:10A7800018BF0120E0B9144B1B68DB0700D500BEE1
:10A7900005B030BD04AA01A942F8103D51F00EF8F1
:10A7A000009B43B10D4B4FF080525A6040BFBFF346
:10A7B0004F8FBFF36F8F003018BF01200028E2D009
:10A7C00022469DF805109DF80400FFF70DF905B02D
:10A7D00030BD00BFC8740020F0ED00E000ED00E0E7
:10A7E00038B58B7803F07F03082B06D90B4B1B6819
:10A7F000DB0700D500BE002038BD094A094B0C46D6
:10A80000204691781D78002202F01EF80028EDD035
:10A8100021462846BDE8384000F0F6BFF0ED00E0E4
:10A820008C74002018610020CB09263301F07F01D1
:10A830000348044A03EB41010844116801F0BABF20
:10A840008C740020C4740020CB09263301F07F01F2
:10A850000348044A03EB41010844116801F0D6BFE4
:10A860008C740020C474002038B5154C01F07F05AD
:10A8700004EB450404EBD1142034A079C00706D5BD
:10A88000104B1B68DA0700D500BE002038BDA57943
:10A890000D4845F001050078A57101F0F1F8002898
:10A8A000F4D1A379074A60F30003A371A37960F39D
:10A8B0008203A3711368DB07E7D500BE38BD00BF74
:10A8C0008C740020F0ED00E018610020054B01F0D1
:10A8D0007F0203EB420303EBD11191F8260000F055
:10A8E000010070478C74002010B50C4B18780C4692
:10A8F00001F0C8F90A4904F07F0301EB430101EBC1
:10A90000D41191F8263043F0020381F8263091F8F3
:10A91000263043F0010381F8263010BD1861002075
:10A920008C740020054B01F07F0203EB420303EB24
:10A93000D11191F82600C0F3400070478C740020BC
:10A9400010B50F4B18780C4601F036F80D4904F09D
:10A950007F0301EB430101EBD41191F826306FF333
:10A96000410381F8263091F826306FF3000381F817
:10A97000263091F826306FF3820381F8263010BD1F
:10A98000186100208C740020704700BF0A4630B464
:10A99000094C496805461068234603C30023C4E9EF
:10A9A000023392F900209A422846ACBF8021194612
:10A9B0001A4630BCFFF758BFD0750020F0B50E46E0
:10A9C0002B4C496807463068A260254603C5002124
:10A9D000E181F588AB4228BF2B4683B0A381ADB19E
:10A9E0003BB3002A3DD094F90000402B28BF402300
:10A9F00000282CDB1F4A3846FFF736FF98B91E4B5C
:10AA00001B68DB0712D500BE03B0F0BD96F900301D
:10AA1000002BACBF8021002138462B462A46FFF789
:10AA200023FF0028EBD0012003B0F0BD002003B0CD
:10AA3000F0BD94F90020002AACBF194680211A46C7
:10AA40003846FFF711FF0028D9D00120ECE7114666
:10AA5000084801931A465DF0F4FC064A019B8021E8
:10AA6000EEE7054B1B68D907E0D500BE1046CBE7E3
:10AA7000D075002090750020F0ED00E0034B00221F
:10AA8000C3E90022C3E902221A617047D075002091
:10AA9000014B1861704700BFD07500200346064A7D
:10AAA0005968006810B41346002403C3C2E9024485
:10AAB0005DF8044B704700BFD075002070B5404C66
:10AAC0002278C909B1EBD21F82B0064615D03BB13E
:10AAD0003C4B1B68DA0700D500BE002002B070BDF9
:10AAE0002146FFF751FF2369002B40D02246304614
:10AAF00003219847012002B070BD94F90020A0689E
:10AB0000002A08DB0028E8D01A462F4901935DF09F
:10AB100098FCA068019BE589E2881D44ADB2184409
:10AB2000AA42A060E58101D03F2B23D8236923B13D
:10AB3000234A02213046984788B194F90020002327
:10AB40009A42ACBF8021194630461A46FFF78CFE68
:10AB500068B91C4B1B68DB07BFD500BEBEE70146CA
:10AB6000304601F08FF83046802101F08BF801204B
:10AB700002B070BDA28994F90010531B9BB2402B08
:10AB800028BF402300290ADB95424FF0000112D074
:10AB90000D4A3046FFF768FE0028DAD0E7E7954215
:10ABA0000BD001461A46084801935DF04AFC80210B
:10ABB000054A019BEDE70A46EBE780210022E8E722
:10ABC000D0750020F0ED00E09075002000B17047D6
:10ABD00052F032BC00B1704752F038BC0138C3B2F9
:10ABE000042B07D856230D4A03FB00F013181B79DA
:10ABF000DB0706D40A4B1B68DB0700D500BE00202C
:10AC00007047CB09363301F07F0103EB4101054B5F
:10AC100008441044196801F0CDBD00BFE475002060
:10AC2000F0ED00E0947700200138C3B2042B07D880
:10AC300056230A4A03FB00F013181B79DB0701D4E3
:10AC400000207047CB09363301F07F0103EB41014F
:10AC5000034B08441044196801F0D8BDE475002086
:10AC600094770020F0B5441EE5B2042D83B017D8C8
:10AC7000562505FB04F5174E01F07F0405EB44044F
:10AC8000344404EBD1143034A779FF070BD5124BB1
:10AC9000186810F0010001D000BE002003B0F0BD24
:10ACA000002003B0F0BD1F4613460A460146705D02
:10ACB000A579009745F00105A57100F0BDFB0028BE
:10ACC000ECD1A37960F30003A371A37960F382034D
:10ACD000A371E3E7E4750020F0ED00E02DE9F04713
:10ACE000764DAF798F4284B091461E4604465BD0C4
:10ACF000E2234FF0000AA9718DF809108DF8083091
:10AD0000ADF80CA0002E00F0B380012103AF0DF1CF
:10AD10000808FBF72BFE41463A4602232046FBF784
:10AD200053FE51462046FBF721FE9DF80C30EB7098
:10AD30002223D9F800908DF80730002E3ED020460F
:10AD40000121FBF713FE3A460DF1070101232046CE
:10AD5000FBF73AFE9DF80C30EB70494608230022C1
:10AD60002046FBF731FE20460021FBF7FFFD0026C1
:10AD7000102241F2F20320460121EA71ADF80830B9
:10AD8000ADF80C60FBF7F2FD3A464146022320463F
:10AD9000FBF71AFE31462046FBF7E8FD9DF80C3024
:10ADA000EB7004B0BDE8F087222303AF0DF1080873
:10ADB000D9F800908DF80730002EC0D14FF0FF3148
:10ADC000E86D50F033FF31462046FBF709FE204680
:10ADD0000121FBF7CBFD3A460DF107010123204687
:10ADE000FBF7F2FD9DF80C30EB7032460823494624
:10ADF0002046FBF7E9FD31462046FBF7B7FD20462C
:10AE00000121FBF7EDFD334632463146E86D50F047
:10AE1000C5FA102241F2F2034FF0FF31E86DEA71FA
:10AE2000ADF80830ADF80C6050F000FF3146204618
:10AE3000FBF7D6FD20460121FBF798FD3A46022399
:10AE400041462046FBF7C0FD31462046FBF78EFD0C
:10AE500020460121FBF7C4FD334632463146E86DFA
:10AE600050F09CFA9DF80C30EB7004B0BDE8F08710
:10AE70004FF0FF31E86D50F0D9FE31462046FBF728
:10AE8000AFFD03AF204601210DF10808FBF76EFD71
:10AE90003A46022341462046FBF796FD31462046BE
:10AEA000FBF764FD20460121FBF79AFD334632464D
:10AEB0003146E86D50F072FA37E700BF987700200E
:10AEC0002DE9F04F4B781D070E4685B09046097866
:10AED000044662D1DA0600F14881B26812B1B28844
:10AEE000002A5AD1E24D03F02006AB7966F07F06C6
:10AEF0008B42F6B200F06481E2230027A9718DF83D
:10AF000009108DF80830ADF80C70B8F1000F00F0A2
:10AF10006C82012120460DF10C090DF1080AFBF7A6
:10AF200025FD51464A4602232046FBF74DFD394692
:10AF30002046FBF71BFD9DF80C30EB70F223EE7101
:10AF40008DF8096000268DF80830ADF80C60B8F176
:10AF5000000F40F0D980E86D4FF0FF3150F066FEF1
:10AF600041462046FBF73CFD20460121FBF7FEFC55
:10AF70004A46022351462046FBF726FD414620461D
:10AF8000FBF7F4FC20460121FBF72AFD434642462D
:10AF90004146E86D50F002FA45E0B54D13F0200748
:10AFA000AA7946D1914240F0BE800DF10C090DF115
:10AFB000080AB37813F0100F0CBF10222022EA23E6
:10AFC00000278DF809208DF80830ADF80C70B8F125
:10AFD000000F00F0FA8001212046FBF7C7FC022396
:10AFE0004A4651462046FBF7EFFC39462046FBF720
:10AFF000BDFC9DF80C30EB707378EB71F2220121EF
:10B0000020468DF809308DF80820ADF80C70FBF75C
:10B01000ADFC51464A4602232046FBF7D5FC394693
:10B020002046FBF7A3FC9DF80C30EB7005B0BDE8A3
:10B03000F08F914240F0A1800DF10C090DF1080A4A
:10B04000B37813F0100F0CBF40228022EA230027B0
:10B050008DF809208DF80830ADF80C70B8F1000FAC
:10B0600000F0E48001212046FBF780FC51460223DA
:10B070004A462046FBF7A8FC39462046FBF776FCFB
:10B080009DF80C30EB7032882B899A422AD0B78811
:10B09000F2887388BF1ABFB25B099F4228BF1F4660
:10B0A00017F0FF0740F008813A23AF708DF8097060
:10B0B00000278DF80830ADF80C70B8F1000F00F0E3
:10B0C000D98001212046FBF751FC514602234A4614
:10B0D0002046FBF779FC39462046FBF747FC9DF8F4
:10B0E0000C30EB7033782B7273786B727378EB7172
:10B0F000F22200268DF809308DF80820ADF80C609A
:10B10000B8F1000F3FF427AF20460121FBF72EFCDA
:10B1100051464A4602232046FBF756FC314620465C
:10B12000FBF724FC7FE7E223A9718DF80910ADF845
:10B130000C708DF80830B8F1000F00F0DE800121AE
:10B1400020460DF10C090DF1080AFBF70FFC5146E2
:10B150004A4602232046FBF737FC39462046FBF7D8
:10B1600005FC9DF80C30EB7023E7434606F108021E
:10B17000FFF7B4FD05B0BDE8F08FE2230027A97109
:10B180008DF809108DF80830ADF80C70B8F1000F8B
:10B1900000F0D980012120460DF10C090DF1080ABB
:10B1A000FBF7E4FB51464A4602232046FBF70CFC22
:10B1B00039462046FBF7DAFB9DF80C30EB703FE791
:10B1C0000DF10C090DF1080AB8E64FF0FF31E86DFA
:10B1D00050F02CFD41462046FBF702FC01212046A1
:10B1E000FBF7C4FB02234A4651462046FBF7ECFB23
:10B1F00041462046FBF7BAFB01212046FBF7F0FB56
:10B20000434642464146E86D50F0C8F89DF80C3080
:10B21000EB707378E86DEB71F2224FF0FF318DF82F
:10B220000930ADF80C808DF8082097E64FF0FF311B
:10B23000E86D50F0FBFC41462046FBF7D1FB204671
:10B240000121FBF793FB4A46022351462046FBF7B8
:10B25000BBFB41462046FBF789FB20460121FBF75B
:10B26000BFFB434642464146E86D50F097F807E77A
:10B27000987700204FF0FF31E86D50F0D7FC414641
:10B280002046FBF7ADFB20460121FBF76FFB4A464A
:10B29000022351462046FBF797FB41462046FBF729
:10B2A00065FB20460121FBF79BFB43464246414696
:10B2B000E86D50F073F812E712238DF80730D6F8D6
:10B2C00008B0B8F1000F64D020460121FBF74EFB17
:10B2D0004A460DF1070101232046FBF775FB9DF857
:10B2E0000C30EB7059463B4600222046FBF76CFBC6
:10B2F00000212046FBF73AFBD6E64FF0FF31E86D20
:10B3000050F094FC41462046FBF76AFB0DF10C0916
:10B31000204601210DF1080AFBF728FB4A460223CB
:10B3200051462046FBF750FB41462046FBF71EFBEB
:10B3300020460121FBF754FB434642464146E86D57
:10B3400050F02CF80DE74FF0FF31E86D50F06EFC37
:10B3500041462046FBF744FB0DF10C092046012134
:10B360000DF1080AFBF702FB4A460223514620462C
:10B37000FBF72AFB41462046FBF7F8FA204601215D
:10B38000FBF72EFB434642464146E86D50F006F877
:10B3900012E74FF0FF31E86D50F048FC414620467F
:10B3A000FBF71EFB20460121FBF7E0FA4A460DF1B0
:10B3B000070101232046FBF707FB9DF80C30EB70DB
:10B3C00042463B4659462046FBF7FEFA4146204698
:10B3D000FBF7CCFA20460121FBF702FB434642462D
:10B3E0004146E86D4FF0DAFF5EE64FF0FF31E86D61
:10B3F00050F01CFC41462046FBF7F2FA0DF10C0917
:10B40000204601210DF1080AFBF7B0FA4A46022353
:10B4100051462046FBF7D8FA41462046FBF7A6FAEC
:10B4200020460121FBF7DCFA434642464146E86DDF
:10B430004FF0B4FF7FE500BF2DE9F04102F07F0C33
:10B44000BDF818E0D20981BBBCF1000F5ED13E4EC1
:10B45000A6F160077178B47882F0010262F34511B9
:10B460000A466FF3041244F010017270B170B278A2
:10B47000B360032363F3030200258046A6F804E0CB
:10B48000B270F5802846FFF7A1FBBC7AC4BB01254A
:10B490002046BD72FFF79EFB2246404631462C46B1
:10B4A000FFF70EFD2046BDE8F08182F00108BCF1F7
:10B4B000000F2ED0254F01223C4604E00132142A11
:10B4C00004F10C0418D094F86C508D42F6D102EBC4
:10B4D000420507EB850595F8615005F00F066645B6
:10B4E000ECD1C5F34015454504F16C06BFD00132DF
:10B4F000142A04F10C04E6D100242046BDE8F081B2
:10B500002846FFF767FB2046BDE8F08182F001087E
:10B51000D0E70E4F01243D4602E00134142CEBD05D
:10B5200095F86C608E4205F10C05F6D104EB4406EB
:10B53000B60007EB060C9CF861C01CF00F0FECD1B5
:10B5400060363E4486E700BFF877002098770020F9
:10B5500042DF704743DF704744DF704712DF7047B8
:10B56000F0B5334CBFF35B8F014604F590730125B2
:10B57000D3E84F2FC3E8405F0028F9D1BFF35B8FBA
:10B5800012F0FF0F48D1082929D04E01A21954F812
:10B5900006C028489388284F01F5947601EB810E68
:10B5A00050F82660D2889A1A93B2B6B200EB8E0297
:10B5B00009B2B34228BF3346C2F800C707EB810087
:10B5C000C2F8043747F82150BFF36F8FBFF34F8F96
:10B5D0001A4B984218D0043B984215D0F0BD154B39
:10B5E000D3F8C024D1030FD494F80B1161B11449DE
:10B5F000D4F80001C3F8A007C3F8A4270D60BFF377
:10B600006F8FBFF34F8FF0BD0023BFF35B8F84F8C4
:10B610002031BFF35B8FF0BD0A4B0B485A68C2F371
:10B620000802003218BF0122BDE8F040FFF794B8CD
:10B63000E8780020007002402870024050700240FC
:10B640004870024000ED00E0C1B60200174BBFF3A6
:10B650005B8F01460122D3E84F0FC3E84C2FBCF1AA
:10B66000000FF8D1BFF35B8F10F0FF0F14D10A6009
:10B67000BFF36F8FBFF34F8F0D4B994203D0043B45
:10B68000994200D070470B4BBFF35B8F002283F8C9
:10B690002021BFF35B8F7047074B08485A68C2F3FD
:10B6A0000802003218BF0122FFF756B8087A0020BE
:10B6B00050700240E878002000ED00E04DB6020036
:10B6C000F0B5334CBFF35B8FC1B204F59073012624
:10B6D000D3E84F2FC3E8406F0028F9D1BFF35B8F49
:10B6E00012F0FF0F47D1082928D04D01621954F8F4
:10B6F00005E028489388DFF8B0C001F5947550F84C
:10B700002570D2888D009A1A93B2BFB26A1800EBE6
:10B710008202BB4228BF3B46C2F800E76544C2F83C
:10B7200004374CF82160BFF36F8FBFF34F8F1A4B74
:10B730009D4218D0043B9D4215D0F0BD154BD3F867
:10B74000C024D1030FD494F80B1161B11349D4F87C
:10B750000001C3F8A007C3F8A4270E60BFF36F8FE2
:10B76000BFF34F8FF0BD0023BFF35B8F84F8203110
:10B77000BFF35B8FF0BD0A4B0A485A68C2F3080258
:10B78000003218BF0122BDE8F040FEF7E5BF00BF60
:10B79000E87800200070024050700240487002407B
:10B7A00000ED00E0C1B602002870024001207047A1
:10B7B000014B80225A60704700E100E0074BD3F84C
:10B7C0000014D3F8002400200A434FF48001C3F88A
:10B7D0000024C3F85801C3F80413704700700240F6
:10B7E000074B4FF4001229B9C3F80823054B83F81F
:10B7F00021117047C3F80423024B83F821117047CD
:10B8000000700240E878002070B48A788C88414E3D
:10B81000C97802F07F03D50905EB430006EB001061
:10B8200001F00301C4F30A04012904812BD0012192
:10B8300001FA03F4BDB1384802339940C0F804134B
:10B84000D0F810352343C0F81035334B42F48071E3
:10B85000C3F81825C3F80C15BFF36F8FBFF34F8FD4
:10B86000012070BC70472C4803F10C06B140C0F8B1
:10B870000413D0F8141503F594730C43C0F8144561
:10B8800040F82350E1E7082B08D0244B186810F04B
:10B890000100E6D000BE002070BC7047EDB9B6F8DC
:10B8A00018311BB11C4B8022C3F81C251A4A0023F7
:10B8B000C2F85031D2F8003313F4001308BFC2F8B5
:10B8C0005431154B4FF44012C3F80423D3F8142518
:10B8D00042F48072C3F81425BEE7B6F808210E4B77
:10B8E0000021C3F82C1112B18022C3F81C250A4A8A
:10B8F000D2F8003313F4001308BFC2F85431064BDA
:10B90000074AC3F80423D3F8102542F48072C3F821
:10B910001025A1E7E878002000700240F0ED00E07B
:10B92000000820001F4B80222DE9F041C3F884203D
:10B93000BFF34F8FBFF36F8F01241B4D1B4FA046EA
:10B940000026A30004F10C02A11C03F1804303F5BF
:10B950001C3308FA01F108FA02F20A43C7F8082377
:10B9600028465E60013420229E6200215CF08DFD3D
:10B97000082C05F12005E4D10D4BC7F8083320222F
:10B98000C7F81C6500217E620A48BE645CF07DFD3C
:10B99000C7F81485C7F81085024B80225A60BDE8AD
:10B9A000F08100BF00E100E0087900200070024053
:10B9B00000083000E879002001F07F02082A70B406
:10B9C0004FEAD11128D0012303FA02F0C043B1B1EC
:10B9D000294C951CAB40C4F80833D4F81055274BBC
:10B9E0002840C4F8100501EB420103EB01110023CC
:10B9F000CB72BFF36F8FBFF34F8F70BC70471E4C7D
:10BA000002F10C05AB40C4F80833D4F814551B4BB5
:10BA10002840C4F81405E6E7184B03EB0110002496
:10BA2000A0F808411448D1B14FF40064C0F80843AD
:10BA3000D0F8104524F48074C0F81045B3F81841CC
:10BA4000B3F808510C48EC424FF0000608BF4FF421
:10BA50000014C0F81C6508BFC0F80843C3E74FF4E2
:10BA60008014C0F80843D0F8144524F48074C0F85A
:10BA70001445C0F85011E1E700700240E87800205A
:10BA800001F07F004FEAD11CF0B50CEB4005744E7D
:10BA90002D01771985B0FC7A4CB1724B1C6814F0FB
:10BAA000010401D000BE0024204605B0F0BD04F022
:10BAB000FF0E7251BB80A7F806E0002843D1002B8F
:10BAC00057D0BCF1000F00F08E8006EB401100EB68
:10BAD0008003CD8A8A8A0C8B0969521B9B0092B223
:10BAE00003F1804303F51C33A24228BF22465E4D7A
:10BAF000C3F8001600B2C3F804265C4BBFF35B8F9B
:10BB000005EB80010122D3E84F4FC3E8472F002FF8
:10BB1000F9D1BFF35B8FE4B2002C40F0908045F880
:10BB20002020BFF36F8FBFF34F8F514B994202D04C
:10BB3000043B994219D1BFF35B8F002386F8203173
:10BB4000BFF35B8F11E0BCF1000FBED106EB4016D6
:10BB50000123F372BFF36F8FBFF34F8FB37A23B11B
:10BB6000F37A03F0FF04002B74D10124204605B0C2
:10BB7000F0BD404AD2F88024C2F3C0126245A0D082
:10BB80003D4D6A688DF80810C2F3080100314FF48A
:10BB9000E06218BF012101A803938DF80930ADF8C8
:10BBA0000420FEF755FCBFF35B8F06F5907201236E
:10BBB000D2E84F1FC2E8403F0028F9D1BFF35B8FA6
:10BBC000CCB2002C38D12A4A1360BFF36F8FBFF379
:10BBD0004F8F1C46BFF35B8F204686F82011BFF3C2
:10BBE0005B8F05B0F0BD0123204AF372BFF35B8F7A
:10BBF000D2E84F4FC2E8413F0029F9D1BFF35B8F34
:10BC0000E4B26CB91D4A1360BFF36F8FBFF34F8F5F
:10BC1000BFF35B8F86F820C11C46BFF35B8F43E701
:10BC2000154B16495A681648C2F30802003218BF6D
:10BC30000122FEF791FD37E76A680D49F3E70E4BE5
:10BC40000F485A68C2F30802003218BF0122FEF7FB
:10BC500083FD29E786F80AC0FFF782FC24E700BFCE
:10BC6000E8780020F0ED00E004700240087A00203F
:10BC7000507002400070024000ED00E04C70024045
:10BC80004DB6020011F07F0008B512D008280BD085
:10BC90000E4B41F48072C909C3F8182504D10C4B2E
:10BCA00003EB40139A7A62B9BFF36F8FBFF34F8FE4
:10BCB00008BD064B01225A65BFF36F8FBFF34F8F4C
:10BCC00008BD9972FFF74CFCEEE700BF0070024020
:10BCD000E878002011F0770F12D00A4B41F48072FF
:10BCE000C3F80C15C3F80C25CA09C3F8181504BF0E
:10BCF00001F5947143F82120BFF36F8FBFF34F8F8D
:10BD0000704700BF007002402DE9F04FA54BA64CD4
:10BD1000D3F8000300238BB01E461F46012520FAEE
:10BD200003F11A19C9074FEA820209D5116839B11E
:10BD300005FA03F117600E43BFF36F8FBFF34F8F08
:10BD40000133192BEBD1F20700F13582974D330502
:10BD500008D5944BD3F8A83601229BB2A5F816312A
:10BD600085F81C21B70206F4800424D58D4BD3F846
:10BD70001425D00540F1FC81002C00F0A182D3F8FD
:10BD80000024D20740F19C82D3F81035DA0540F147
:10BD9000FB8195F81C3107AF002B40F0BD82814B31
:10BDA000D3F82035089338464FF440730121ADF89D
:10BDB0001C30FEF74DFB04B37A4AD2F8004440F23F
:10BDC00001732340C2F80034E30500F15682670591
:10BDD00010D5744B0122C3F808259A65D3F80023C7
:10BDE00012F4001208BFC3F854216E4B4FF4001236
:10BDF000C3F80423A00500F1358231023DD5694B1B
:10BE0000D3F880C4D3F88414D3F888E4D3F88C74BE
:10BE1000D3F89084D3F89444D3F89804D3F89C24AE
:10BE20005FFA8CF35FFA80FCD0B25A06C9B25FFAAF
:10BE30008EFEFFB25FFA88F85FFA84F901D1052916
:10BE40001BD00024224668F3070263F3070461F362
:10BE50000F2469F30F226EF317446CF3174260F35B
:10BE60001F6267F31F644FF4C063012107A8CDE987
:10BE70000842ADF81C30FEF7EBFA4D4B3340002B77
:10BE800040F09181DFF82491464F4D46CA4609F5AE
:10BE9000907800241DE02B44DA7A002A00F0D78144
:10BEA000DA88AAF804200022DA72D98809914FF4BE
:10BEB000E063012107A88DF820B08DF82120ADF8AE
:10BEC0001C30FEF7C5FABBF1080F47D001340AF168
:10BED000200A04F10C0326FA03F3DB075FFA84FB64
:10BEE000F1D504EB840307EB8303DAF80020D3F8E1
:10BEF0000807630112FA80F2E918CAF80020CA881C
:10BF000080B2024492B2082CCA80C4D0BAF8082089
:10BF10008242C0D1CA88BAF804109142BBD9BBF1A1
:10BF2000000FD0D10122BFF35B8FD8E84F3FC8E8A4
:10BF3000412F0029F9D1BFF35B8F13F0FF0F40F0C1
:10BF400052821C490A60BFF36F8FBFF34F8FBFF35C
:10BF50005B8F85F82031BFF35B8FB7E7164B33401B
:10BF6000002B00F002810F4BD3F86C240192C3F830
:10BF70006C24BFF36F8FBFF34F8F16F4806600F011
:10BF80006E81D3F88024D3F8803483F08003C3F328
:10BF9000C0130593C2F3C0130493DFF808A0002474
:10BFA000A84613E000700240409C0010E878002092
:10BFB000FCFB1F004C70024000040001002C00F04C
:10BFC000F281072E52D0013409F120090199E14094
:10BFD00004EB8403C9070AEB830308EB4412E6B2BF
:10BFE000ECD5D3F80816D9F81070C9B20F44C9F8C7
:10BFF0001070D08A014489B2D182A849D08AB9F898
:10C00000145061188900854202914FF0010C66F0CE
:10C010007F0103914FF4E06B4FF0000E614607A8DB
:10C0200040F2B480D18AB9F81820C3F800766D1AAE
:10C03000ADB2954228BF1546994AC3F80456BFF3DE
:10C040005B8FD2E84F3FC2E841CF0029F9D1BFF35F
:10C050005B8F13F0FF0F40F0ED80029BC3F800C030
:10C06000BFF36F8FBFF34F8F072EACD1019BDB0364
:10C07000454601D4059B43B1EB7A23B1EB88AA88EE
:10C080009A4200F271810123AB72019B9F030BD591
:10C0900095F82B3023B1EB8CAA8C9A4200F2888160
:10C0A000012385F82A30019B5E030DD595F84B30AE
:10C0B00033B1B5F84630B5F844209A4200F27D819C
:10C0C000012385F84A30019B1C030DD595F86B3090
:10C0D00033B1B5F86630B5F864209A4200F27E813B
:10C0E000012385F86A30019BD8020DD595F88B3075
:10C0F00033B1B5F88630B5F884209A4200F2388121
:10C10000012385F88A30019B99020DD595F8AB3053
:10C1100033B1B5F8A630B5F8A4209A4200F22D81CB
:10C12000012385F8AA30019B5A020DD595F8CB3032
:10C1300033B1B5F8C630B5F8C4209A4200F2228176
:10C14000012385F8CA30019B1B020ED595F8EB3010
:10C15000002B00F0F380B5F8E630B5F8E4209A4201
:10C1600040F2EC800720FFF7FBF90BB0BDE8F08F41
:10C17000D3F81025D1053FF50CAE95F821211AB959
:10C180004FF40012C3F8082307AF08E6D38A0993D7
:10C190009DF80C30ADF81CB08DF820308DF821E002
:10C1A000FEF756F90DE70023BFF35B8F85F82031CA
:10C1B000BFF35B8F66E63B4B3B4A3C4D3C4800245B
:10C1C0000127C2F81475C2F81075546094625C605F
:10C1D0009C629C60DC62DC601C631C615C635C6173
:10C1E0009C639C61DC63DC611C6454629464C2F8EF
:10C1F0005841D2F80034D2F800140B43C2F800348E
:10C20000D2F80033C2F808332146C2F804032846A6
:10C210004FF492725CF039F940234FF48072394642
:10C2200007A82B832B818DF82040ADF81C20FEF74A
:10C230000FF98CE51F4B20485A680299C2F3080297
:10C24000B2EB0E0218BF0122FEF786FAB9E61B4BCD
:10C250001B68D80789D500BE0BB0BDE8F08FCDE9CB
:10C2600004669AE600220523012107A88DF81C2008
:10C270008DF81D30FEF7ECF8BFE50121C2F82C1552
:10C280000423002207A88DF81C208DF81D30FEF72E
:10C29000DFF867057FF5AEAD9BE500BF019C0010A0
:10C2A000087A00200470024000700240E878002004
:10C2B0000514C00100ED00E04DB60200F0ED00E015
:10C2C0004F4BBFF35B8F0122D3E84F1FC3E8402FD2
:10C2D0000028F9D1BFF35B8F11F0FF0F32D1494B2A
:10C2E000D3F8C004C70352D495F80B1101F0FF072F
:10C2F000002967D04449D5F80071C3F8A077C3F886
:10C30000A4070A60BFF36F8FBFF34F8FD3F81035C8
:10C31000D8053FF53EAD37E7B5F816310993002251
:10C3200085F81C2188234FF4E06238460121ADF8DE
:10C330001C20ADF82030FEF78BF830E5012385F89E
:10C34000EA3012E7314B32485A68C2F30802003231
:10C3500018BF01220821FEF7FFF92A4BD3F8103548
:10C36000DB053FF516AD0FE70020FFF7F9F88CE687
:10C370000420FFF7F5F8019BC6E60520FFF7F0F86B
:10C38000019BD1E60620FFF7EBF8019BDCE6BFF34B
:10C390005B8F85F82011BFF35B8FD3F81035DF0575
:10C3A0003FF5F7ACF0E6049900293FF40CAE18E62F
:10C3B0000120FFF7D5F8019B76E60220FFF7D0F8C1
:10C3C000019B81E6BFF35B8F85F82071BFF35B8F24
:10C3D000D3F81035D9053FF5DCACD5E60320FFF7DF
:10C3E000BFF8019B80E6094B0A485A680A49C2F324
:10C3F0000802003218BF0122FEF7AEF966E500BF61
:10C40000087A0020007002404870024000ED00E011
:10C41000C1B602004DB602004C70024030B5012892
:10C4200085B000F09F8057D3022840D1BA4BD3F893
:10C430000435002B40F0D780B74AD2F800341C05F1
:10C44000FBD54FF40063C2F80034BFF36F8FBFF326
:10C450004F8FB24AB24B12681B68082A00F0D7808F
:10C46000AD4BB04D80240122C3F81C45C3F8042312
:10C47000C5F88441FDF7D8FA002840F0F880AA4DAD
:10C4800043F204044FF080432268AA4211D0D3F84B
:10C490000C14D3F80C24D003F6D5CA07F4D59E4B60
:10C4A0000122C3F80425BFF36F8FBFF34F8F05B090
:10C4B00030BD04AA002102F80C1D1046FFF74EF80B
:10C4C0009DF804000028E2D010460191FFF744F8DF
:10C4D000019A002AD8D0E2E78F4BD3F80025002A32
:10C4E000E5D14FF480014FF40062C3F80813C3F89C
:10C4F0000024BFF36F8FBFF34F8F884B1B68082B4F
:10C5000000F0B780844B0122C3F80025BFF36F8F82
:10C51000BFF34F8F43F2040203F18D5303F57723EA
:10C52000126803F2DB539A4200F0CA804FF0804356
:10C53000D3F80C24D3F80C34D90301D5D207B6D4E0
:10C5400043F20402784B12689A4200F01881774B4C
:10C5500000221A601B6801934FF080430122019969
:10C560001A60A4E76C4BD3F80025002A9FD0002264
:10C57000C3F80425BFF36F8FBFF34F8F6949802045
:10C58000C1F88400BFF34F8FBFF36F8FD3F8001350
:10C59000C3F80813C3F80025BFF36F8FBFF34F8FA5
:10C5A00043F2040103F18D5303F57723096803F285
:10C5B000DB53994200F0998001AB5D4A0121116083
:10C5C0005C4A5168C1F30801003118464FF000027F
:10C5D0004FF0020318BF01218DF804208DF80530BB
:10C5E000FDF736FF63E743F204024F4B12689A42AD
:10C5F00000F0B0804FF08043D3F80C24D3F80C3413
:10C60000DB037FF519AFD5077FF516AF4FE7032B97
:10C610000AD8494A1168002940F09880474C49F2ED
:10C6200075301060216010605A1E022A10D8424AEC
:10C630001168002967D1424D3848394B00681B68A2
:10C6400049F2753414602960146008287FF408AF3B
:10C65000032B3FF605AF3B493B4B40F2E3704022D2
:10C6600008601A60BFF36F8FBFF34F8FF8E66C60FE
:10C6700005E72B4B1B685A1E022A12D82E4B1A684C
:10C68000002A40F08E802E4949F2753203201A604C
:10C6900008601A60214A224B12681B68082A7FF43E
:10C6A00031AF032B3FF62EAF234B1A68002A74D10B
:10C6B000224949F27532C0201A6008601A6021E7E9
:10C6C00004AB002203F80C2D1846FEF747FF9DF837
:10C6D000041000293FF42AAF18460192FEF73CFFF0
:10C6E000019B002B7FF4E3AE2AE704AB03F80C2D8B
:10C6F0001846FEF733FF9DF80420002A3FF45DAF93
:10C70000FEF728FF5CE70549054B0D4A08681B68E2
:10C710000021116099E700BF007002403001001055
:10C720003401001000E100E0DBE5B1510001004000
:10C730000400004000ED00E000EC064014EC064070
:10C7400014ED06400078024004780240174A0021A8
:10C75000116069E704AB002203F80C2D1846FEF7C0
:10C76000FDFE9DF8041000293FF444AF18460192E5
:10C77000FEF7F2FE019B002B7FF499AE5CE604A865
:10C78000002300F80C3DFEF7E9FE9DF80430002B75
:10C790003FF4DDAEFEF7DCFE89E6044BC0221A60F2
:10C7A000B0E6034B03221A6074E700BF14EC0640A6
:10C7B00014ED0640F8B5037813F0010405D10678AE
:10C7C000C6F3800626B12046F8BD00242046F8BDF9
:10C7D0000F4605464FF0FF3138464FF027FA2A78CA
:10C7E00012F001040FD12B785B0704D42B7843F0AF
:10C7F00004032B700124002338461A4619464EF0D4
:10C80000CDFD2046F8BD3446F5E700BF70B50546BE
:10C810000E4608464FF0FF314FF008FA2878C0F373
:10C82000800444B90024002330461A4619464EF0CD
:10C83000B5FD204670BD2B7813F00102F2D12B78A4
:10C8400062F382032B70EEE710B4C378848803F0A0
:10C850000303022BC4F30A0426D019D8012B04D0F9
:10C86000002318465DF8044B7047022940F2FF325E
:10C8700008BF4FF48062A242F3D21A4B1B6813F038
:10C880000103EED000BE002318465DF8044B70474C
:10C89000022914BF40234FF48063A342EDD3012348
:10C8A00018465DF8044B704702290BD012B1B4F55D
:10C8B000007F11D0A4F108039BB2182B06D9402C9D
:10C8C000EDD0DAE7B4F5007FD7D1E8E7064A22FADF
:10C8D00003F3DB07D1D5E2E700244021134644717E
:10C8E0000171BEE7F0ED00E0010100010A44914250
:10C8F00016D230B44C78052C05D00C7821448A42ED
:10C90000F8D830BC70478C7804F07F0500EB450503
:10C91000E4092B550C7821448A42EBD830BC70478F
:10C92000704700BF2DE9F04182B00678089DBDF840
:10C930002470009361F300060446294600F8086B52
:10C94000012316463A46BDF82C80FCF76DFE05B172
:10C950003FB90A9B63600120A4F8028002B0BDE8E1
:10C96000F08104F11C0101204EF0F2FE26B90346CD
:10C970003046C4E90503ECE70023FAE710B50446A6
:10C98000406908B14FF008FBA06908B14FF004FB03
:10C99000012010BDF0B50B460D4613F8081B83B0FF
:10C9A00011F0020F0746184640F2FF130CBF3F2458
:10C9B0001C461646FCF774FEE8B9E6B126421AD1C9
:10C9C0002B786978DA07384618D5FEF707F990B161
:10C9D0002B78697813F0010313D000233846CDE992
:10C9E00000331A46FEF73EF930B9084B1B68DB07E7
:10C9F00001D500BE00E0002003B0F0BDFDF714FF3C
:10CA0000E5E738461A46FDF72FFFEDE7F0ED00E0C9
:10CA100070B501F1080582B0064628460C46FCF7C1
:10CA20003FFE38B123786178DB07304605D5FEF745
:10CA3000D5F830B9002002B070BDFDF7F5FE002832
:10CA4000F8D0284662886168FCF754FE054690B12C
:10CA5000237862686178D80717D50023CDE90033C1
:10CA600030462B46FEF7FEF8B0B90C4B1B68DB07CF
:10CA7000E0D500BEDFE72078617810F00104304691
:10CA800008D1FDF7E1FE2046D5E730462B46FDF7FD
:10CA9000EBFEE9E7FEF7C8F82846CCE7F0ED00E04A
:10CAA0002DE9F0418A890B7882B00C460646E2B93E
:10CAB000DD07497857D5FEF791F800284FD0227846
:10CAC00063886178D20751D5002B5DD0626800255C
:10CAD0003046CDE90055FEF7C5F800284DD1374B5B
:10CAE0001B68DB073BD500BE3AE003F0020301F10F
:10CAF0000808002B40460CBF40274FF40077304D0C
:10CB000008BF6FF03F05FCF7E3FD874227D8237885
:10CB10006178DB07304634D5FEF760F8F8B140465F
:10CB2000FCF7D6FD874233D805EA000265882378F2
:10CB3000617890B2854228BF0546DA0732D5002DCC
:10CB400037D062680023CDE9003330462B46FEF72C
:10CB500089F80028C3D0284602E0FEF765F80020D7
:10CB600002B0BDE8F081FDF75FFEA6E773B1626831
:10CB70003046FDF779FE0028B1D0608802B0BDE8EC
:10CB8000F081FDF751FEC9E71A46A0E71A46EFE724
:10CB90002078617810F001043046DED1FDF754FEB4
:10CBA0002046DDE73DB1626830462B46FDF75CFE6E
:10CBB000CFE72A46C6E72A46F6E700BFF0ED00E0D9
:10CBC00000FEFFFF0048704780EE3600704700BF50
:10CBD000704700BF704700BF704700BF704700BF7D
:10CBE000704700BF704700BF90ED3C0A704700BF20
:10CBF00090F86B01704700BF90F86C314FF47A6089
:10CC000000FB03F0704700BF90F86301704700BF5E
:10CC10000048704754ED08000048704754ED080084
:10CC200000487047F0E4080000487047F0E408004E
:10CC30000048704768F008000048704768F0080036
:10CC400080F8E810704700BF80F82010704700BFE0
:10CC50006830704760387047704700BFF0B4D0F854
:10CC60009C6E002E14DD07460023184607F5067259
:10CC700015790C78A54202F1A00204D100F69414B3
:10CC8000013047F824300133B342F1D1F0BC704792
:10CC90000020F0BC704700BF084A416E0023C0E985
:10CCA0000E33C0E90C33A0F858305361C1F80C358D
:10CCB000C1F80835C2E90333704700BFFCA9002062
:10CCC00002F6941250F82230002B03DBD0F89C2E91
:10CCD000934200DB704730B403EB830300EB431057
:10CCE000D0F87E42D0F88222D0F88632D0F88A522C
:10CCF000CD600C604A608B60D0F88E42D0F89A52BA
:10CD0000D0F89222D0F896328B61CD610C614A61E5
:10CD100030BC70472DE9F0410F462DED028B4FF4EA
:10CD2000FA610446F0EE408AB0EE608A16469846F4
:10CD30000BF0EAF942F23C6304F51955E05042F277
:10CD40004C6242F24D634EF66021284601FB08F129
:10CD5000C5ED018A01F5FA6180ED028AA7542046EB
:10CD6000E6540BF0D1F904F519542060BDEC028BA8
:10CD7000BDE8F08110B590F83E21044612B9C0F824
:10CD8000E02010BD034901FB02F10BF0BDF9C4F82E
:10CD9000E00010BDC0D4010010B590F83F2104465A
:10CDA00012B9C0F8E42010BD034901FB02F10BF0F9
:10CDB000ABF9C4F8E40010BD80EE360070B50A4C43
:10CDC000C56B86B0D4E9032364690395856B02952E
:10CDD000D0E90C56084601960095049403495CF08E
:10CDE000A7FB06B070BD00BFFCA900203CEE080008
:10CDF0004EF09EB970B5C06D104C036886B01B68CC
:10CE00009847014604A82BF099FB9DF810109DF857
:10CE100012609DF815509DF81100029001F5FA611D
:10CE200003919DF814309DF8132005492046CDE963
:10CE300000565CF07DFB204606B070BD0C7A0020E9
:10CE400070ED0800D0ED507AF5EEC07AF1EE10FAF0
:10CE500021D99FED127AF0EE400AD0B5B0EE670A04
:10CE600077EE600A0C4657F047FD10EE100A5AF0B4
:10CE7000F7FA00220A4B5AF093F9064620460F466D
:10CE80005AF0CCFA02460B46304639465AF040FB7F
:10CE90005AF0EEFDD0BD0020704700BF9A99593F6F
:10CEA0000000F03F70B58B884D880446006D9E11E0
:10CEB00003F03F01026806FB011155FA81F10231CE
:10CEC0009368984707EE900A94ED517A206EF8EE39
:10CED000677A002167EE877ABDE87040FCEEE77A5A
:10CEE00017EE902A02EB820201320CF0C5B900BFA6
:10CEF00070B58B884D880446006D9E1103F03F018C
:10CF0000026806FB011155FA81F1023193689847D6
:10CF100007EE900A94ED567A206EF8EE677A0021BB
:10CF200067EE877ABDE87040FCEEE77A17EE902A4C
:10CF300002EB820201320CF09FB900BF38B502F655
:10CF4000941250F822309DF81420002B03DBD0F807
:10CF50009C1E8B4201DB002038BD03EB83035C0188
:10CF600005462044049900F23E200CF037F92C4489
:10CF700084F83D02E86D03681B689847C4F8A40272
:10CF8000002038BD30B441F2E43541F69A0141F653
:10CF90009402455B002341F644544352855200F508
:10CFA000E851021900F5EA5503511C3141F6945439
:10CFB00053609360D36013615361936129600123CF
:10CFC000035530BC704700BF2DE9F04700F5EC5425
:10CFD00000F518588CB08A4691461C3408F1340884
:10CFE00002E02C34444525D04A46514620465BF0A9
:10CFF00019FA0028F5D101462C2201A85BF045FA68
:10D0000001A80BF089F801AF25460DF1240C3E462E
:10D010000FCE664528606960AA60EB60374605F16F
:10D020001005F4D103CF2C343B782B724445286093
:10D030006960D9D10CB0BDE8F08700BF014811F09C
:10D04000F3BE00BFFCA9002070B52DED028B044695
:10D0500040680368DB6BB0EE608A16460D46984761
:10D06000606803682946D3F8E83098476068036829
:10D07000B0EE480AD3F8E4309847314660680022A1
:10D080001AF01AFF84F82450BDEC028B6068036824
:10D09000082D1B6E8CBF10212021BDE87040184761
:10D0A000024B012258681BF009BA00BFFCA90020FE
:10D0B00001482CF0BDB900BFC4B1002003460022D6
:10D0C00000F59F50D3F8CC1011F02CB800B583B008
:10D0D000D0F8CC20054B009268460A4604490193DB
:10D0E0000FF044FD03B05DF804FB00BFA0E10900B0
:10D0F000FCE40800D0F8CC0001492CF04BBA00BF8A
:10D10000E4E40800406801492CF044BAE4E4080073
:10D11000034600F56A60D3F8CC100FF0A9BB00BF3E
:10D12000034600F6D85059680FF0A2BB10B441F680
:10D130006454021931B100F59F5001235DF8044B8E
:10D1400010F082BB015151609160D1605DF8044BD9
:10D15000704700BF0B7813F0030315D0012B05D0E7
:10D1600000F5EB50002303600020704700F5C35327
:10D170000C331B79DB07F3D400F5C35300F5EB50F8
:10D180000C3303600020704710B50122044600F5FF
:10D190009F5010F085FB04F5EB542060002010BD7B
:10D1A0002DE9F04F02F1FF3E0EEBDE7E4FEA6E0EF0
:10D1B000714594469B4602F0010949DA0F466FF02B
:10D1C00040487D1C6C0004EB080650F8352050F8F0
:10D1D0002660D6F824A000EBC506556A55450AD945
:10D1E000013C744550F8242040F8272000EB8406C9
:10D1F00005DA2746E5E7744540F82720F9DBB9F161
:10D20000000F2BD0651E05EBD5758C424FEA6505E6
:10D210001ADD50F82570DBF824207B6A9A4207D388
:10D2200012E050F82270DBF824307A6A9A420BD967
:10D230006A1E02EBD2725210A94240F8247000EB31
:10D2400085062C461546ECDBC6F800B0BDE8F08F2D
:10D2500000EB8106B9F1000FF6D10C46ACF1020CDF
:10D260000CEBDC7CB4EB6C0FCCD10134640004F12A
:10D270008042013A013C50F82220326000EB8406E3
:10D28000C0E700BF2DE9F04F02F1FF3E0EEBDE7E5E
:10D290004FEA6E0E714594469B4602F0010949DA49
:10D2A0000F466FF040487D1C6C0004EB080650F8F8
:10D2B000352050F82660D6F824A000EBC506556A44
:10D2C00055450AD2013C744550F8242040F82720E7
:10D2D00000EB840605DA2746E5E7744540F8272089
:10D2E000F9DBB9F1000F2BD0651E05EBD5758C422B
:10D2F0004FEA65051ADD50F82570DBF824207B6ABB
:10D300009A4207D812E050F82270DBF824307A6A8B
:10D310009A420BD26A1E02EBD2725210A94240F816
:10D32000247000EB85062C461546ECDBC6F800B0F1
:10D33000BDE8F08F00EB8106B9F1000FF6D10C4685
:10D34000ACF1020C0CEBDC7CB4EB6C0FCCD10134F7
:10D35000640004F18042013A013C50F8222032601E
:10D3600000EB8406C0E700BF02F1FF3C0CEBDC7C65
:10D370004FEA6C0C61452DE9F04F964602F0010A28
:10D380004BDA0F466FF040497D1C6C0004EB090638
:10D3900050F8352050F8266092F928B096F9288088
:10D3A000C34500EBC5060ADD013C644550F8245036
:10D3B00040F8275000EB840605DA2746E4E7644589
:10D3C00040F82720F9DBBAF1000F2CD0651E05EBE1
:10D3D000D5758C424FEA65051CDD50F8257093F930
:10D3E00028C097F92820944508DB13E050F82270F4
:10D3F00093F9282097F928C094450BDD6A1E02EBAB
:10D40000D2725210A94240F8247000EB85062C46D7
:10D410001546EBDB3360BDE8F08F00EB8106BAF117
:10D42000000FF7D10C46AEF1020E0EEBDE7EB4EB30
:10D430006E0FCBD10134640004F18042013A013C0B
:10D4400050F82220326000EB8406BFE702F1FF3C77
:10D450000CEBDC7C4FEA6C0C61452DE9F04F9646F5
:10D4600002F0010A4BDA0F466FF040497D1C6C0058
:10D4700004EB090650F8352050F8266092F928B0E0
:10D4800096F92880C34500EBC5060ADA013C6445DD
:10D4900050F8245040F8275000EB840605DA274660
:10D4A000E4E7644540F82720F9DBBAF1000F2CD0FF
:10D4B000651E05EBD5758C424FEA65051CDD50F8FD
:10D4C000257093F928C097F92820944508DC13E0CB
:10D4D00050F8227093F9282097F928C094450BDA68
:10D4E0006A1E02EBD2725210A94240F8247000EB7F
:10D4F00085062C461546EBDB3360BDE8F08F00EB6C
:10D500008106BAF1000FF7D10C46AEF1020E0EEB18
:10D51000DE7EB4EB6E0FCBD10134640004F18042A7
:10D52000013A013C50F82220326000EB8406BFE74C
:10D530002DE9F84F8E46091A402975DD06469246B8
:10D54000002A7BD0984600F1040BC910736856F886
:10D5500021C05C6ADCF824005EF8049C3268D9F8CB
:10D56000245084420AF1FF3A29D9A8425ED8AC423D
:10D5700029D8C6E900325EF8042C506A596A5C4624
:10D580007346A44625465CF8049BD9F824708F4264
:10D5900013D88842A3F1040304D253F8042D506A2F
:10D5A0008842FAD3A34214D94CF8042CC3F8009053
:10D5B00053F8042C3168506A496A6446E1E7AC428A
:10D5C000D7D8A84232D9C6F800904EF8042C336858
:10D5D000D3E77146434652462046FFF7A9FFA11BF9
:10D5E000402921DDA646BAF1000FAED18C10A71E4E
:10D5F0007F1007F1010806EB880800E0013F58F8AA
:10D60000043D224639463046FFF7CAFD002FF5D1CA
:10D6100055F8043D32682A60AC1BA2100021304648
:10D62000FFF7BEFD042CF3DCBDE8F88FC6F800C0A0
:10D6300046F821205EF8042C33689EE77546D5E74E
:10D640002DE9F84F8E46091A402975DD06469246A7
:10D65000002A7BD0984600F1040BC910736856F875
:10D6600021C05C6ADCF824005EF8049C3268D9F8BA
:10D67000245084420AF1FF3A29D2A8425ED3AC4238
:10D6800029D3C6E900325EF8042C506A596A5C4618
:10D690007346A44625465CF8049BD9F824708F4253
:10D6A00013D38842A3F1040304D953F8042D506A1C
:10D6B0008842FAD8A34214D94CF8042CC3F800903D
:10D6C00053F8042C3168506A496A6446E1E7AC4279
:10D6D000D7D3A84232D2C6F800904EF8042C336853
:10D6E000D3E77146434652462046FFF7A9FFA11BE8
:10D6F000402921DDA646BAF1000FAED18C10A71E3D
:10D700007F1007F1010806EB880800E0013F58F898
:10D71000043D224639463046FFF7B4FD002FF5D1CF
:10D7200055F8043D32682A60AC1BA2100021304637
:10D73000FFF7A8FD042CF3DCBDE8F88FC6F800C0A5
:10D7400046F821205EF8042C33689EE77546D5E73D
:10D750002DE9F84F0646081A402878DD1746002ABA
:10D760007FD0984606F10409C010736856F820E08F
:10D7700093F928509EF9284051F804AC32689AF980
:10D7800028C0A54207F1FF372EDD644561DC654501
:10D790002EDCC6E9003251F8042C92F928B093F936
:10D7A00028C04C460B46A64625465EF804AB9AF9BF
:10D7B0002800604516DCE345A3F1040305DA53F8BD
:10D7C000042D92F928006045F9DBA34216D94EF8E2
:10D7D000042CC3F800A053F8042C306892F928B048
:10D7E00090F928C07446DEE76545D2DC644530DD3B
:10D7F000C6F800A041F8042C3368CEE72046434623
:10D800003A46FFF7A5FFA01B402820DD2146002F48
:10D81000AAD18410A71E7F1007F1010806EB880823
:10D8200000E0013F58F8043D224639463046FFF7F4
:10D830009BFD002FF5D155F8043D32682A60AC1BE2
:10D84000A21000213046FFF78FFD042CF3DCBDE869
:10D85000F88FC6F800E046F8202051F8042C336811
:10D860009BE70D46D5E700BF2DE9F84F0646081A9D
:10D87000402878DD1746002A7FD0984606F1040933
:10D88000C010736856F820E093F928509EF928409C
:10D8900051F804AC32689AF928C0A54207F1FF3765
:10D8A0002EDA644561DB65452EDBC6E9003251F8AE
:10D8B000042C92F928B093F928C04C460B46A64692
:10D8C00025465EF804AB9AF92800604516DBE3456F
:10D8D000A3F1040305DD53F8042D92F928006045F7
:10D8E000F9DCA34216D94EF8042CC3F800A053F873
:10D8F000042C306892F928B090F928C07446DEE70D
:10D900006545D2DB644530DAC6F800A041F8042C46
:10D910003368CEE7204643463A46FFF7A5FFA01BF3
:10D92000402820DD2146002FAAD18410A71E7F1099
:10D9300007F1010806EB880800E0013F58F8043DB4
:10D94000224639463046FFF781FD002FF5D155F8C4
:10D95000043D32682A60AC1BA21000213046FFF75C
:10D9600075FD042CF3DCBDE8F88FC6F800E046F83E
:10D97000202051F8042C33689BE70D46D5E700BF03
:10D980002DE9F0412DED028B0346006D1C69026804
:10D990005D69136ADFF8688084B00E4698470746D1
:10D9A000D8F8040003681B6F9847D8F80400036890
:10D9B000B0EE408A5B6F9847FDEEC87A0E4BA3FB32
:10D9C0000525A3FB043417EE903A10EE100AAD09BA
:10D9D000A409CDE902451CB259F042FD3AB2CDE9A5
:10D9E00000012346304605495BF0A2FD04B0BDECC2
:10D9F000028BBDE8F08100BFD34D6210E8ED080056
:10DA0000FCA90020014811F00FBA00BFFCA90020BA
:10DA100001482BF00DBD00BFC4B100202DE9F84F27
:10DA20008E46091A402975DD06469246002A7BD0AB
:10DA3000984600F1040BC910736856F821C05C6A5F
:10DA4000DCF824005EF8049C3268D9F82450844243
:10DA50000AF1FF3A29D9A8425ED8AC4229D8C6E9D2
:10DA600000325EF8042C506A596A5C467346A4463C
:10DA700025465CF8049BD9F824708F4213D888425D
:10DA8000A3F1040304D253F8042D506A8842FAD358
:10DA9000A34214D94CF8042CC3F8009053F8042C7A
:10DAA0003168506A496A6446E1E7AC42D7D8A84277
:10DAB00032D9C6F800904EF8042C3368D3E771468B
:10DAC000434652462046FFF7A9FFA11B402921DD0E
:10DAD000A646BAF1000FAED18C10A71E7F1007F139
:10DAE000010806EB880800E0013F58F8043D224693
:10DAF00039463046FFF754FB002FF5D155F8043D69
:10DB000032682A60AC1BA21000213046FFF748FBA8
:10DB1000042CF3DCBDE8F88FC6F800C046F82120DD
:10DB20005EF8042C33689EE77546D5E7024B012268
:10DB300058681AF0C3BC00BFFCA90020034600F5DA
:10DB4000985018305968002210F0ECBA00B583B034
:10DB50004268054B009268460A46044901930FF05B
:10DB600005F803B05DF804FBA0E10900FCE408003F
:10DB7000084A0023C2E90433D36050F8642C20F82B
:10DB8000703C40E9243340E92633C2F80C35C2F832
:10DB900008357047FCA9002030B441F21C3541F231
:10DBA000D27141F2CC72455B002341F67C44435272
:10DBB00085520219035141F6784541F6CC4400F5EF
:10DBC000E25153609360D3601361536193611431E8
:10DBD00001234151035530BC704700BF10B4C83811
:10DBE00041F66454021931B100F59F5001235DF8EC
:10DBF000044B0FF029BE015151609160D1605DF876
:10DC0000044B70472DE9F843A0F1C80604462DEDFA
:10DC1000028B884630464FF4FA61F0EE408AB0EE4F
:10DC2000608A174699460AF06FFA42F2745304F577
:10DC30001555E05042F2845242F285534EF660216F
:10DC4000C5ED0F8A01FB09F104F5165585ED008A33
:10DC5000304604F8028001F5FA61E7540AF054FAFC
:10DC600042F27853E050BDEC028BBDE8F88300BF70
:10DC700070B50B4C50F88C5C86B0D4E90323646912
:10DC8000039550F8905C029550E926560846019697
:10DC90000095049403495BF04BFC06B070BD00BFD7
:10DCA000FCA900203CEE08002DE9F0412DED028B8F
:10DCB000034650F8780C53F8B84C026853F8B45C3B
:10DCC000136ADFF8688084B00E4698470746D8F894
:10DCD000040003681B6F9847D8F804000368B0EE8F
:10DCE000408A5B6F9847FDEEC87A0E4BA3FB052573
:10DCF000A3FB043417EE903A10EE100AAD09A40904
:10DD0000CDE902451CB259F0ABFB3AB2CDE90001B6
:10DD10002346304604495BF00BFC04B0BDEC028B9B
:10DD2000BDE8F081D34D6210E8ED0800FCA90020A9
:10DD300090F876300BB983617047054910B501FB47
:10DD400003F10446C8380AF0DFF9A06110BD00BF36
:10DD5000C0D4010090F877300BB9C3617047054912
:10DD600010B501FB03F10446C8380AF0CDF9E061B3
:10DD700010BD00BF80EE36002DE9F04700F5E654F7
:10DD800000F515588CB08A469146143408F12C08D9
:10DD900002E02C34444525D04A46514620465AF0EC
:10DDA00041FB0028F5D101462C2201A85AF06DFB59
:10DDB00001A80AF0B1F901AF25460DF1240C3E4649
:10DDC0000FCE664528606960AA60EB60374605F1B2
:10DDD0001005F4D103CF2C343B782B7244452860D6
:10DDE0006960D9D10CB0BDE8F08700BF2DE9F043E0
:10DDF00090F8443F83B0044683B141F27413C35C8E
:10DE000063B141F27713C356002B03DB002003B04C
:10DE1000BDE8F083B0F8523F002B5FD194F83D315C
:10DE2000002BF3D10B7803F00302012A3DD0002A26
:10DE300050D18A8894F8680102F03F05A842E5D9DC
:10DE4000C3F38303042B59D004F5EB531B68002B59
:10DE5000DCD094F81632002B3CD0012B53D02F4E3F
:10DE60002F48022B14BFB146814696110136F6B2F7
:10DE700001F10A07002D49D068344FF000083846F8
:10DE8000324621465AF0CEFA013D374418B908F11E
:10DE900001005FFA80F815F0FF05F0D119F80600CF
:10DEA000404594BF00200120B1E78A8894F86801BA
:10DEB00002F03F05A842A9D994F86901A842A5D962
:10DEC000C3F38303042B23D004F5EB531B68002B0F
:10DED000BFD19BE7012003B0BDE8F08301914DF075
:10DEE00027F941F26813B4F8525FE2580D4B0199DB
:10DEF000801A03FB05F3984288D28FE794F86A31C1
:10DF0000AB42A1D882E7DFF82090AEE7A846C5E78C
:10DF100094F86A31AB42D7D878E700BF1C61002083
:10DF20002461002080EE3600206100202DE9F043BE
:10DF30008BB004460F461646022102AA00F56A601D
:10DF40000CF0D2F902AA034604F1680120460AF057
:10DF5000B7FB30B105463EB901463A4620460BF0C4
:10DF6000FDF80BB0BDE8F08304F5EB5808F10408A8
:10DF7000404694F8156210F03DFB0136F6B281463A
:10DF800070BB2946404610F08BFB0096ADF80800A8
:10DF90003B4602AA29462046ADF80A900AF02AFD1F
:10DFA00094F8443F002BDCD094F8493F002BD8D0A4
:10DFB00041F25E02B4F8543F0121A154002BD0D0AD
:10DFC00041F264056359002BCBD04DF0B1F8635991
:10DFD00000F56A5018301B1A002BC2DD6051C0E7F3
:10DFE00033463A46294620460AF0D0FCD8E700BF1F
:10DFF000A0F1C800FFF79ABF90F8E83003B9704766
:10E0000070B50446A0B007A816460D460123314A54
:10E01000D4F8CC102BF03CFA07A82BF0ADFE08B9D1
:10E0200020B070BD23682C4A5B6993424DD1E06DEE
:10E0300003681B689847014605A82AF07FFA9DF8F7
:10E0400015009DF814109DF8164002909DF81900D7
:10E050009DF818309DF8172001F5FA610391CDE97C
:10E0600000041E491E485BF063FA1D4907A84BF0E7
:10E070009DFE2B786A881B4801921B4903F003021E
:10E08000023A012A88BF0146C3F383030091324656
:10E09000164907A84CF076F82B78C3F38303082BB6
:10E0A0000AD0022B08D9124907A84CF06BF807A830
:10E0B0002BF036FE20B070BD95F84A3095F84B2015
:10E0C0000C4907A84CF05EF8F1E720469847014656
:10E0D000CCE700BFE4E40800F5CD020070ED0800D5
:10E0E0000C7A00201CF0080018F0080020F008004E
:10E0F00054E4080054F0080090F8E83003B9704781
:10E1000070B50446A0B007A816460D460123274A5D
:10E11000D4F8CC102BF0BCF907A82BF02DFE08B9D1
:10E1200020B070BD2368224A5B69934239D1E06D0B
:10E1300003681B689847014605A82AF0FFF99DF877
:10E1400015009DF814109DF8164002909DF81900D6
:10E150009DF818309DF8172001F5FA610391CDE97B
:10E160000004144914485BF0E3F9134907A84BF085
:10E170001DFE2B786A8801921048114903F00302B2
:10E18000023A012A88BF0146C3F383033246009155
:10E1900007A80C494BF0F6FF07A82BF0C1FD20B0F3
:10E1A00070BD204698470146E0E700BFE4E4080060
:10E1B000F5CD020070ED08000C7A00201CF008007C
:10E1C00018F0080074F0080090F8E83003B97047C0
:10E1D0002DE9F0472DED028B0546A2B009A81746A0
:10E1E0000E460123464AD5F8CC1010EE104A2BF00B
:10E1F0004FF909A82BF0C0FD20B922B0BDEC028B6D
:10E20000BDE8F0872B683F4A5B69934274D1E86DA3
:10E2100003681B689847014607A82AF08FF99DF804
:10E220001D009DF81C109DF81EC002909DF8210055
:10E230009DF820309DF81F2001F5FA610391CDE98A
:10E24000000C314931485BF073F9304909A84BF0B3
:10E25000ADFD286D96F8008001682D4A2D4B896B25
:10E26000B6F802A008F00309A9F10209B9F1010FFB
:10E2700094BF914699468847286D03685B6BB0EE62
:10E28000408A984707EE104ADFED237ACDF80090D8
:10E2900067EE277ABDEEC00AFDEEE77ABDEEC88ACA
:10E2A000C8F383084346CDF804A03A468DED030A2F
:10E2B000CDED047A8DED028A184909A84BF062FF72
:10E2C0003378C3F38303082B0DD0022B0BD91449E9
:10E2D00009A84BF057FF09A82BF022FD22B0BDEC96
:10E2E000028BBDE8F08796F84A3096F84B200D492E
:10E2F00009A84BF047FFEEE7284698470146A5E7F7
:10E30000E4E40800F5CD020070ED08000C7A00206E
:10E3100018F008001CF0080000007A44CCEF080058
:10E3200054E4080054F008002DE9F04F00F5EC53D8
:10E33000064600F51850BBB00F461C33343000249D
:10E340005A6A32B13AAA02EB8402013442F8C83C5C
:10E3500024B22C338342F3D108AD4FEA840905EB94
:10E360000908A8454BD04FEAA902B2FA82F2C2F1DD
:10E370001F0252004FF0000341462846FFF74EFBB4
:10E38000B9F1400F79DC09AB984538D09A464FF087
:10E39000000BA1460FE009ABA3EB0B039D4205D098
:10E3A0005844CBF1040229465AF056F8D045089457
:10E3B000ABF1040B22D05046089B5AF8044B5B6A21
:10E3C000616A9942E7D85AF8083C5A6A9142A5EB2B
:10E3D0000B0C40F2C380504600E0F44640F8043D88
:10E3E0005CF8043C616A5A6A9142ACF1040EF4D8BC
:10E3F000D045CCF80040ABF1040BDCD14C46002CEE
:10E4000040F39780DDF820B0DFF858A1B8464FF010
:10E4100000090422594605A80AF042FFF06D03687E
:10E420001B689847DBF824309BF928200092C31A18
:10E4300005AA514640465BF07BF898F800301BB1C6
:10E4400018F8013F002BFBD109F10109A1450CD0BF
:10E45000A8EB0703852B08DC4FF00A0388F800308F
:10E4600055F829B008F10108D3E7474562D00023E9
:10E4700088F800303BB0BDE8F08F6FF003035B1B02
:10E48000039309A90DF16009A3460FE08D4209D05D
:10E490000AABA3EB0A00039B084403EB0A022946DC
:10E4A00059F0DAFFD1450894514620D08A46089B9E
:10E4B0005AF8044B5B6A606A9842E7D85AF8083CFD
:10E4C0005A6A9042A1F1040C46D9504600E0F44645
:10E4D00040F8043D5CF8043C616A5A6A9142ACF130
:10E4E000040EF4D8D145CCF800405146DED1C845E1
:10E4F0005C4684D00DF15C0EDC46CA46724659F883
:10E50000044B5EF8043B606A596A884222D9CA46C5
:10E5100000E05A464AF8043D52F8043C606A596AE1
:10E520008842A2F1040BF4D8C8451460E5D16446D2
:10E5300065E7B8460A4B18689A889B79C8F80000C6
:10E54000A8F8042008F8063F002388F800303BB004
:10E55000BDE8F08F5246E7E78C46C3E7844647E7BD
:10E56000E0ED0800D4ED0800A0F1C800FFF7DCBE24
:10E570002DE9F04F0C79A4068FB018D10C7814F067
:10E58000030417D1CC88C4B11F46199B1546064613
:10E59000DAB20C4602A818990BF058F89DF8093029
:10E5A0002BB19DF8083003F00F03022B09D00FB0F8
:10E5B000BDE8F08F032CE7D1E4E70C89002CE3D110
:10E5C000F5E706F5EC5A94F9023101930AF11C0AB9
:10E5D00006F51859D34609F134094FF0FF340AE023
:10E5E000DBF82420A24238BFDA460BF12C0B38BFEF
:10E5F0001446D9451FD0202259462846D84659F0FE
:10E6000011FF0028ECD128686968AA68EB684446C5
:10E610000FC42869EB696969AA690FC4C8F820703A
:10E62000F06D03681B6898479DF8043088F828301F
:10E63000C8F82400BBE7D046E5E700BF00000000B3
:10E6400008B50C202DED028B50F04EF8022050F052
:10E6500051F80121062050F053F90121062050F015
:10E66000D3F90A204CF070FD042050F073F808EE46
:10E67000100A0021062050F0C7F9B8EEC88ADFED75
:10E680000C7A68EE277A17EE900A58F0E9FE06A396
:10E69000D3E9002358F03CFF59F012FABDEC028B8D
:10E6A00080B208BDAFF300809A9999999999134067
:10E6B00000803B3F08B50C202DED028B50F014F884
:10E6C000022050F017F80121062050F019F901211D
:10E6D000062050F099F90A204CF036FD042050F045
:10E6E00039F808EE100A0021062050F08DF9B8EE36
:10E6F000C88ADFED0B7A68EE277A17EE900A58F099
:10E70000AFFE05A3D3E9002358F002FF59F0D8F972
:10E71000BDEC028B80B208BD9A99999999991340E2
:10E7200000803B3F2DE9F041034682B05C6D134809
:10E73000B3F85870DD6C0E46FFF7BCFF2368104A33
:10E740001B689342804614D14CF0F2FC04462B68BF
:10E7500028465B6998470B4B0190A3FB0423009765
:10E76000424630469B0908495AF0E2FE02B0BDE835
:10E77000F081204698470446E9E700BFC0A6002084
:10E78000F1CD0200D34D62108CED08002DE9F0416F
:10E79000034682B053F8744C134833F8707C53F836
:10E7A0007C5C0E46FFF786FF2368104A1B68934285
:10E7B000804614D14CF0BCFC04462B6828465B69AB
:10E7C00098470B4B0190A3FB042300974246304629
:10E7D0009B0908495AF0ACFE02B0BDE8F081204622
:10E7E00098470446E9E700BFC0A60020F1CD02002B
:10E7F000D34D62108CED0800F8B543790D2B04461B
:10E8000000F28280604A02EB0312A379072B73D8CF
:10E810005E4D03EB4301890068186E58077A416822
:10E82000457A0346D4ED067A2166F5EEC07A2B20B0
:10E830001021F1EE10FA84F8647084F8655084F8C1
:10E840006600A4F8681063DD3046C4ED177A5AF00C
:10E8500012FF002800F09380431E052B40F29180A8
:10E86000002211468708334653F8045B0132974271
:10E8700081EA0501F8D8C1F30723C1F307424B40F1
:10E88000534020F0030283EA11639042DBB21FD0B1
:10E89000B55C511C884283EA050319D9715C4B4071
:10E8A000911C8142DBB213D2755CD11C884283EA91
:10E8B00005030DD9755C111D884283EA050307D94C
:10E8C000715C0532904283EA010301D9B25C534086
:10E8D0002F48D0E90021D0E902504A406A40424026
:10E8E000C2F307215140C2F30740414081EA12625E
:10E8F000534084F81031F8BD0020244B254E2649A2
:10E90000A07105250B278DE700231F4A43717CE783
:10E91000D2ED017A92ED026AD3ED016A9FED1F7A82
:10E92000196836EE676A66EE876A0A7886EE267A96
:10E9300041F20553BDEEC77A17EE100A0128B8BFA1
:10E94000012032B103EB4313134411F8012F002AC5
:10E95000F8D1B3FBF0F200FB123307EE103AB8EE39
:10E96000C77AB6EE006A37EE067A3046E6EE877A68
:10E97000C4ED177A5AF07FFE00287FF46DAF03468E
:10E98000A6E700231A4683E764D5080004D50800EB
:10E99000F4D40800F0E3080000007A436F12833AD1
:10E9A00010B52DED028BFDEEC08AB0EE408A044614
:10E9B0005AF061FEB8EEE80A9FED0A7A0A4938EE8D
:10E9C000408AF6EE007AE8EE077A204418EE902AA4
:10E9D000BDEC028BFDEEE77ABDE8104017EE903AF1
:10E9E0005AF0A6BD00007A4444D608002DE9F04351
:10E9F000DDB00446002301A8C84A2AF049FD01A859
:10EA00002BF0BAF910B95DB0BDE8F0834FF4847211
:10EA100000211AA859F039FD1AA94FF4847201A8EF
:10EA20002BF008F9054601A82BF07AF9032DEADD51
:10EA3000B5F5847F1A9E0FD0B94B9E4240F0A48258
:10EA40006B1FB3F5827FDED22A461AA9204659F001
:10EA5000F8FCB44B236077E1B24FBE4240F06A81CC
:10EA60002A461AA9204659F0ECFC94F90A10E289CA
:10EA7000B4F86C30A789268A658A1629A8BF1621A2
:10EA8000B2F5FA6F28BF4FF4FA626FF00800B3F5E1
:10EA9000FA6F28BF4FF4FA638142B8BF0146052AD6
:10EAA00038BF0522052B38BF05231E2FA08AA1726F
:10EAB00038BF1E27B6F5167F28BF4FF4167621798A
:10EAC000E281B5F5347F28BF4FF4347594F86A209D
:10EAD000A4F86C30B0F5B46F28BF4FF4B46094F86C
:10EAE0008630A781003118BF012194F89A706582A1
:10EAF000003218BF0122003318BF0123002F14BFBA
:10EB000001250025A0824FF000002682217184F8A3
:10EB10006A2084F8863084F89A5084F8A30000F0C4
:10EB2000D68294F89B30002B00F0D182B4F8983054
:10EB3000B3F5FA6F28BF4FF4FA63052B38BF0523EE
:10EB4000A4F8983094F8BA30002B14BF01220022A8
:10EB50004FF0000384F8BA2084F8C33000F0B38289
:10EB600094F8BB30002B00F0AE82B4F8B830B3F5A7
:10EB7000FA6F28BF4FF4FA63052B38BF0523A4F8BA
:10EB8000B83094F8DA30002B14BF012200224FF085
:10EB9000000384F8DA2084F8E33000F0908294F8DF
:10EBA000DB30002B00F08B82B4F8D830B3F5FA6F6D
:10EBB00028BF4FF4FA63052B38BF0523A4F8D830DB
:10EBC00094F8FA30002B14BF012200224FF000030A
:10EBD00084F8FA2084F8033100F06D8294F8FB3059
:10EBE000002B00F06882B4F8F830B3F5FA6F28BF54
:10EBF0004FF4FA63052B38BF0523A4F8F83094F8D6
:10EC000080306279032B84BF032384F88030002393
:10EC10000D2A84F8853084F85B3096BF424B6371CF
:10EC200003EB0212A37988BF3F4A072B00F25382FD
:10EC30003E4D03EB4301890068186E58077A41681E
:10EC4000457A0346D4ED067A2166F5EEC07A2B208C
:10EC50001021F1EE10FA84F8647084F8655084F89D
:10EC60006600A4F8681040F340823046C4ED177A7D
:10EC70005AF001FD002800F03682431E052B4FF0AC
:10EC800000031A4615D98708314651F8045B013351
:10EC90009F4282EA0502F8D8C2F307235340C2F329
:10ECA00007414B4083EA126320F003029042DBB23B
:10ECB0001FD0B55C511C884283EA050319D9715CE9
:10ECC0004B40911C8842DBB213D9755CD11C884241
:10ECD00083EA05030DD9755C111D884283EA05039B
:10ECE00007D9715C0532904283EA010301D9B25C15
:10ECF00053400F48D0E90021D0E902504A406A4011
:10ED00004240C2F307215140C2F30740414081EA2B
:10ED10001262534084F8103175E600BFE4E3080046
:10ED200041524E3541524E3964D5080004D5080091
:10ED3000F4D40800CD4B9E4240F026812A461AA901
:10ED4000204659F07EFB276000200021C4E91E0107
:10ED5000C4E91C01642300279846A4F86C30994646
:10ED600084F86A70002584F88050002384F881308C
:10ED7000012684F886608022002104F1880059F081
:10ED800084FB002F40F0848194F90A20E389A7894D
:10ED9000268A608AA4F86C80162AA8BF16226FF013
:10EDA0000801B3F5FA6F28BF4FF4FA638A42B8BF7F
:10EDB0000A46052B38BF05231E2FA18AA27238BF31
:10EDC0001E27B6F5167F28BF4FF416762279E38109
:10EDD000B0F5347F28BF4FF43470B1F5B46F28BF5D
:10EDE0004FF4B461131C94F89A20268218BF0123B3
:10EDF000002A18BF01264FF0000208BF0026A78195
:10EE00006082A182237184F89A6084F86A2084F871
:10EE1000A32000F0EF8094F89B30002B00F0EA80F4
:10EE2000B4F89830B3F5FA6F28BF4FF4FA63052BA6
:10EE300038BF0523A4F8983094F8BA30002B14BFDB
:10EE4000012200224FF0000384F8BA2084F8C33076
:10EE500000F0CC8094F8BB30002B00F0C780B4F8F1
:10EE6000B830B3F5FA6F28BF4FF4FA63052B38BFFB
:10EE70000523A4F8B83094F8DA30002B14BF01222F
:10EE800000224FF0000384F8DA2084F8E33000F029
:10EE9000A98094F8DB30002B00F0A480B4F8D830BF
:10EEA000B3F5FA6F28BF4FF4FA63052B38BF05237B
:10EEB000A4F8D83094F8FA30002B14BF01220022B5
:10EEC0004FF0000384F8FA2084F8033100F08680C4
:10EED00094F8FB30002B00F08180B4F8F830B3F5E3
:10EEE000FA6F28BF4FF4FA63052B38BF0523A4F847
:10EEF000F8306279032D84BF032384F88030002327
:10EF00000D2A84F8853084F85B3096BF584B6371C6
:10EF100003EB0212A37988BF554A072B6ED8554DD3
:10EF200003EB4301890068186E58077A4168457AF7
:10EF30000346D4ED067A2166F5EEC07A2B20102127
:10EF4000F1EE10FA84F8647084F8655084F8660075
:10EF5000A4F868105ADD3046C4ED177A5AF08BFBDE
:10EF6000002800F0C080431E052B4FF000031A4616
:10EF70007FF69FAE8708314651F8045B01339F420C
:10EF800082EA0502F8D887E63B4B9E4240F0DD80DE
:10EF90006B1FB3F5827FBFF436AD2A461AA920460F
:10EFA00059F04FFAB4F86C90334B344A2260B9F5FB
:10EFB000FA6FC84628BF4FF4FA68B8F1050F38BF9A
:10EFC0004FF005089E4294F86A703FF4CBAE2C4B8C
:10EFD00094F880509E423FF4CBAEC6E6002384F8FE
:10EFE000FA3086E7002384F8DA3063E7002384F8F8
:10EFF000BA3040E7002384F89A301DE70020214E04
:10F0000021491C4BA07105250B2792E7D2ED017A0F
:10F0100092ED026AD3ED016A9FED1C7A196836EE13
:10F02000676A66EE876A0A7886EE267A41F20553A9
:10F03000BDEEC77A17EE100A0128B8BF012032B121
:10F0400003EB4313134411F8012F002AF8D1B3FB4B
:10F05000F0F200FB123307EE103AB8EEC77AB6EEC4
:10F06000006A37EE067AE7EE267A74E741524E35AB
:10F0700064D5080004D5080041524E3641524E393D
:10F0800041524E38F0E3080000007A436F12833A91
:10F09000D4E91C01D4E91E23C4E92201C4E92423D4
:10F0A00084F89A60A4F8989008222D4904F19B00F6
:10F0B0005AF00FFB68E6002384F8FA309FE500233E
:10F0C00084F8DA307CE5002384F8BA3059E500236F
:10F0D00084F89A3036E50020224E2349234BA07154
:10F0E00005250B27AEE5034603E6D2ED017A92ED46
:10F0F000026AD3ED016A9FED1E7A196836EE676ADF
:10F1000066EE876A0A7886EE267A41F20553BDEEEE
:10F11000C77A17EE100A0128B8BF012032B103EBFD
:10F120004313134411F8012F002AF8D1B3FBF0F276
:10F1300000FB123307EE103AB8EEC77AB6EE006A5B
:10F1400037EE067AE6EE877A8FE503F180739E420A
:10F150003FF41EAF03F180739E423FF419AF52E4B7
:10F16000B8EC0800F0E3080000007A4304D508007A
:10F170006F12833A2DE9F84F00F5EC5808F11C089E
:10F1800000F518572DED028B8146B0EE408A0D46F2
:10F190009246444634374FF0FF3609E0636AB34283
:10F1A00038BFA04604F12C0438BF1E46A74227D022
:10F1B000202221462846A34659F034F90028EDD1F3
:10F1C00028686968AA68EB685C460FC42869EB691F
:10F1D0006969AA690FC4CBF820A0D9F85C0003685C
:10F1E0001B689847F0EE487AFEEECF7ACBF8240001
:10F1F00017EE903A8BF82830BDEC028BBDE8F88F03
:10F20000C346DDE72DE9F041044600F5EB500D461D
:10F21000016888B016461F4609B10B8843B93B46C2
:10F2200032462946204609F0B1FB08B0BDE8F0811E
:10F2300004AA012304F59F500EF006FB0028EEDD22
:10F2400004A80FF0D7F980460028E8D1294604A881
:10F250000FF026FA0097ADF80C00334629462046F9
:10F2600003AAADF80E8009F0C5FB08B0BDE8F08137
:10F270002DE9F84F054640201C46164688460B9F50
:10F280004EF03AFB202183460FF034F92368D04832
:10F290001B68D04AC5F84CB000218342C5E914640C
:10F2A000C5E90021C5E9041140F08F814BF040FF12
:10F2B0000A9AA86100230C98C7492A664FF0010CEE
:10F2C000C64A6866EB61C5E90933A5F858302B6278
:10F2D000C5E91033EF6585F82CC0A9642A6005F1F3
:10F2E000680008F027FFBE4B2B6005F5077AE8336E
:10F2F000C5F8C830544605F5067905F69C662046E3
:10F30000A03408F009FFB442F9D150464FF44862E6
:10F31000002159F0BAF805F1C800B249C5F8A07E3D
:10F320000024C5F8A80EC5F8B01E05F59F5A05F5CE
:10F33000825341F2540E41F2580C41F25C06002017
:10F34000012105F1F007C5F8AC8EC5F8B89EC5F8E7
:10F350009C4EC5F8B4AEC5F8A47E41F25E02C3E986
:10F36000020141F25F0941F2500145F80E4005F5F6
:10F37000835345F80C4041F2640EAC5341F2680CE3
:10F3800041F261060820AC5405F80940FF22685498
:10F3900018461C70214645F80E400C3005F80C400C
:10F3A000AA55282259F071F841F24C1341F2501C31
:10F3B00041F25411D046EC524FF0000A45F80C408F
:10F3C00005F574636C544FF0000B05F58B52404605
:10F3D00041F2741C4FF000084FF0000941F2751122
:10F3E000C3E986ABC3E988ABC2E9028941F2761270
:10F3F00005F80C406C5441F2701C41F27711AC548A
:10F400004FF0FF3245F80C206A5441F2881C05F594
:10F410008D5205F59556C3E98EABC3E990AB1C360A
:10F4200005F80C4041F2B81EC3E994ABC3E996ABB2
:10F4300041F2BC1C147041F2A11141F2BD126C5496
:10F44000C3E99AABC3E99CAB314645F80E4005F8D9
:10F450000C40AC54C6F820410EF094F805F5C450A9
:10F46000314610300EF08EF841F6745105EB010E66
:10F4700041F67C5C41F6885005F5EC530422B42635
:10F480004FF078096C5003F11C08CEF8049045F851
:10F490000C20C3E900462A50444608F69806204648
:10F4A0002C3408F039FEB442F9D105F51850B421D6
:10F4B000343029F021FD41F6985641F6945305F574
:10F4C000195142F23C62002440464FF000094FF0CF
:10F4D0000008AC51C5F8D040C5E93844C5E93689C3
:10F4E0000C6085F8E8402146AC50EC5440F6980298
:10F4F00058F0CBFF214638464FF4947258F0C5FFC0
:10F5000000274FF07C533849C5F844314FF07E5204
:10F51000C5F85811C5F8F02005F1F400C5F84071A0
:10F5200020223249324E0FF0A3F900200021C5E914
:10F530004601C5E94801102205F594702D490FF0E8
:10F5400097F92D48C5F838014FF4A1621623C5F884
:10F550006461A5F86021012685F83C312749C5F88A
:10F5600068114FF4E13342F601704FF4FA72A5F8D6
:10F570003E01A5F86E21C5F8743105F2791085F8C1
:10F58000704185F86D6185F8786110221C490FF093
:10F590006FF941F6645241F68C5C41F69050AB181D
:10F5A00085F88A61C5F88C41C5F8987185F81462B0
:10F5B000022145F80C402C50AC5085F890115C604D
:10F5C0009C60DC602846BDE8F88F204698476FE6CF
:10F5D000F1CD020020F9080080EE3600BCF90800E9
:10F5E000E4F0080030AA00209A99993EACF0080097
:10F5F00000007A42C4F008008D675944404008007A
:10F60000D0F008002DE9F0478AB0044602AA8946E6
:10F6100000F56A6002210AF067FE02AA034604F1BF
:10F620006801204609F04CF8054638B3E06C0368E1
:10F630005B69984704F5EB5704378046384694F8E1
:10F6400015620EF0D7FF0136F6B28246C8B92946D8
:10F6500038460FF025F80096ADF808004B4602AA90
:10F6600029462046ADF80AA009F0C4F9E06C036809
:10F670005B6998474045D4BF002001200AB0BDE82F
:10F68000F08733464A462946204609F07FF9EDE7E0
:10F6900008B5C06C03685B6998470028D4BF002098
:10F6A000012008BD2DE9F8432DED028B0D460968B8
:10F6B0009DF8288009699DF92C7004462846164655
:10F6C0009946B0EE408AF0EE608A884723681F4A68
:10F6D0009B6C934231D160680368B0EE480ADB6BE3
:10F6E0009847606803683146D3F8E8309847606807
:10F6F0000368B0EE680AD3F8E43098474946002220
:10F70000606818F0D9FB606884F824600368082EEC
:10F710001B6E8CBF10212021984741462846442269
:10F7200018F000FC204639460FF07EFBBDEC028B42
:10F730002046BDE8F8430FF07BBB4A463146F0EE69
:10F74000680AB0EE480A20469847E6E749D002002A
:10F75000F8B507681D460E463B6911462A46044621
:10F76000984700B9F8BD236829469B68204698470A
:10F77000FA3045004BF0DCFC074605E023685B6986
:10F780009847A8B94EF000FE4BF0D2FCC31BAB4229
:10F790002046F3D90021304619F024FB23680546A2
:10F7A0009B6920469847002D0ADB07D00220F8BD50
:10F7B000236820469B6998470120F8BD0320F8BDC7
:10F7C0000420F8BD70B50446384816461D4609F0B9
:10F7D00079FF04F5EC53D3E900210A4490424BD25F
:10F7E0005A891989013292B291425A814AD32A78B0
:10F7F00041F2B82302F03F022946E25411F8013BDE
:10F8000041F2B9259B11013304F5935002FB03F239
:10F810006355183058F015FE04F58E5341F2C815A3
:10F820001E60E06D03681B68984741F2C41294F8AB
:10F83000443FA050002262558BB141F27413E35C47
:10F840006BB141F27713E356002B05DB41F2C8128E
:10F850008023A354092070BDB4F8523FA3B994F893
:10F860003D316BB141F2C813E35C43F0800341F2D8
:10F87000C8120920A35470BD012218605A81B6E74E
:10F88000092070BD002070BD4BF052FC41F268139E
:10F89000B4F8521FE258064B801A03FB01F398425A
:10F8A000DDD3635D43F08003E1E700BF24AA0020BD
:10F8B00080EE3600F0B591F84A2002F0F003802B7C
:10F8C0008BB00C4605460BD0902B07D14B88052BEF
:10F8D00004D902F00F02022A00F085800BB0F0BDBF
:10F8E0004B88052BFAD990F8443FC3B141F2741309
:10F8F000C35CA3B141F27713C356002BEEDAB0F824
:10F90000523F63B14BF014FC41F26813B5F8521F3B
:10F91000EA58574B821A03FB01F39A42DED295F85C
:10F920003D31002BDAD1534809F0CCFE41F6745139
:10F930006B186A585E683244904280F091805A8910
:10F940001989013292B291425A81C7D3628894F8E0
:10F950004B30092A03F0040340F28680002BBDD00F
:10F96000236DD5F894219A42B8D32B4694F84A6077
:10F9700053F8681FCDF806109868D9685A68CDF812
:10F980000E00CDF8121098691969CDF80A2016F00A
:10F99000010F5A69CDF81610CDF81E00D969E06C38
:10F9A000CDF81A2094F80241CDF822104FF09203BE
:10F9B000CDF802000CBF26220E22694628468DF89B
:10F9C00001408DF8003008F0CBFF0446002885D0B8
:10F9D0002B680146DB6B2846984721468200284663
:10F9E00009F0BCFB7AE7252B7FF678AF41F68C5601
:10F9F000835923B941F68C530022EA506EE741F651
:10FA00009053C15808F074FB0028F3D1AA59E36C55
:10FA10009A427FF463AF27466E4657F8500F7968D5
:10FA2000BA68FB680FC638697969BA69FB690FC69D
:10FA30006846202205F1680158F0F4FC00283FF4E4
:10FA40004DAF0C4809F03EFE94F9023100EE103A39
:10FA5000024669462846BAEECF0AFFF78BFB3DE720
:10FA6000012268505A8171E7002B3FF437AF7CE7E1
:10FA700080EE360024AA00202DE9F04F0C78C4F364
:10FA8000830485B0072CDDE90E6C02D005B0BDE81B
:10FA9000F08F9846174641F2B8230022D6F800A00E
:10FAA00006F80C20FF22C25496F8049009F1FF33A7
:10FAB0001E2B04460D4640F2BE80043691F800B07D
:10FAC000B9F1000F00F01B8104F59471304659F034
:10FAD00092FD002800F08481304604F5A47159F0AD
:10FAE0008AFD0028D2D106460022414604F5067060
:10FAF00009F0FEFFD0F884309A458146C6D9C0F897
:10FB000084A0E06D03681B68984799F82030C9F815
:10FB1000880023F00303334389F82030386879687C
:10FB2000BA68D7F80CC0C9F86EC0C9F86200C9F845
:10FB30006610C9F86A2038697969BA69D7F81CC0B3
:10FB4000C9F87EC0C9F87200C9F87610C9F87A20E1
:10FB50003EB141F28831204608F0D6FA41F698537A
:10FB6000E0500BF0030BBBF1010F9CBFFF2389F8A2
:10FB70002130D4F85CA0DAF8003050461B68984772
:10FB8000DAF80430984298BF581C04F58E5641F2BA
:10FB9000C4130022CAF804003060E25299F8203001
:10FBA000206E03F00303A3F1030341F2C612B3FA7C
:10FBB00083F35B09A35441F2C71399F82020E25460
:10FBC000036831461B6804220831984741F2CC1380
:10FBD0000222E2540D202B7803F00303012B40F2A4
:10FBE000998041F2B82914F90930002BC0F2FA804B
:10FBF000CDE900603B4642460121204608F070FEF8
:10FC000000283FF443AF41F2B92214F80930A25C56
:10FC100003F03F03013A43EA821304F593524FF491
:10FC200096750146DBB2183220460E9505B0BDE848
:10FC3000F04F08F019BFB9F1010F19D0B9F1020F57
:10FC400000F08680B9F1030F7FF420AF0B7803F04A
:10FC50000303023B012B3FF619AF731D5246414689
:10FC6000FFF7B0FD00283FF411AF04F58E56B2E760
:10FC70000B7803F00303023B012B3FF607AF634809
:10FC800009F020FD04F5EC51D1E90032134498420B
:10FC900080F0B3804B890A8901339BB29A424B8131
:10FCA000FFF4F4AE727941F2B82302F03F02E2545D
:10FCB000737941F2B92C9B110133B11D04F59350B6
:10FCC00004F58E5602FB03F204F80C30183058F09D
:10FCD000B8FBC6F800A0E06D03681B68984741F2C6
:10FCE000C41200233146A05008310093AC220123F6
:10FCF00004F59F500EF07EF90830C0B2B2E7202222
:10FD0000414600F5067009F0D3FE814600287FF4D5
:10FD100028AFD9E603902B7902964FF0010CCDE97C
:10FD2000003C3A46414605F10A03204608F022FD10
:10FD300000283FF4ABAEAB889B1101330146DBB228
:10FD400020464FF4967205B0BDE8F04FFFF75ABA5F
:10FD50000B7803F00303023B012B3FF697AE2B48D1
:10FD600009F0B0FC04F5EC53D3E900210A449042B9
:10FD700047D25A891989013292B291425A81FFF4CD
:10FD800085AE727941F2B82302F03F02E2547379F2
:10FD900041F2B92C9B110133B11D04F5935004F5C8
:10FDA0008E5604F80C3002FB03F2183058F049FB71
:10FDB000C6F800A0E06D03681B68984741F2C413C1
:10FDC0000836E05004F1F40204F5CE7310493046D1
:10FDD00059F0AEFB304659F04EFC0830C0B241E756
:10FDE000032681E6CDE900603B46424601212046DC
:10FDF00008F076FD00289ED148E60860A1F80A9038
:10FE000050E7012218605A81BBE700BF24AA0020F6
:10FE1000CCED0800000000002DE9F04F83462DEDE9
:10FE2000028B00F58E50DDB002601C78012C00F0D2
:10FE30004A81032C0D4600F0E080052C00F08580FF
:10FE4000062C40F08F805D78002D40F084809A79F8
:10FE500099780391202AB3F803905E790BF5185135
:10FE60000BF5EC5328BF202204921C3334315A6A1C
:10FE7000ACB23AB15CAA02EB85050134A4B245F8F4
:10FE8000C83C25B22C338B42F1D1002E00F02C82DD
:10FE9000012E00F07882022E00F0C682032E00F0C0
:10FEA000AE81039B002B00F082834D4540F3868397
:10FEB000049A079409A906918F182AA9531DA5EB46
:10FEC000090001EB89059A4699460590002690465F
:10FED00004952B4606E0059B9E421DD0822A1BDC22
:10FEE000049B9246DBF85C0053F8265002681268C7
:10FEF00090476C6A2946041B4246A7EB080058F05D
:10FF0000A0FA039B95F828103C6001369E42397197
:10FF100009EB0A024F44DED1079C0699B6B20AF1FA
:10FF2000080541F2C41041F2C6132BF800400BF54E
:10FF30008E5052462BF80360083058F082FA28465B
:10FF40005DB0BDEC028BBDE8F08F91F8202002F08F
:10FF50000302032A1FD0002528465DB0BDEC028BAA
:10FF6000BDE8F08F072CF6D10BF58E5404340BF559
:10FF7000CE730093D44AD5490BF1F403204659F0CF
:10FF8000D7FA204659F077FB051D28465DB0BDEC39
:10FF9000028BBDE8F08F5D78002DDCD19F78002FBB
:10FFA000DAD1DBF89C0E0028D8BF0425D4DD04226A
:10FFB00015460BF5077601E0AD2ACDDC931D96F8CA
:10FFC000204005F58E515BFA83F30BEB01050137F9
:10FFD00003F58E535CB130684BF80100B188A980FD
:10FFE00096F8201019700732DBF89C0ED2B28742C7
:10FFF000154606F1A006DFDBAEE70BF518543434E6
:020000023000CC
:1000000020465E7828F08CFF0C204EF06DFB02201D
:100010004EF070FB012106204EF072FC01210620FB
:100020004EF0F2FC0A204BF08FF804204EF092FBC9
:1000300008EE100A002106204EF0E6FCB8EEC88A51
:10004000DFEDA37A68EE277A17EE900A57F008FAE8
:100050009BA3D3E9002357F05BFA57F031FD80B240
:1000600007EE900A9FED9B0AF8EE677A204627EE8E
:10007000800A012128F0F4FF95F82030964813F00B
:1000800003011CBFF143C9B222460FF089FA93481D
:100090000CF018FF0121204628F080FF204628F0B0
:1000A00043FF0546204628F041FF01460BF58E50E0
:1000B0002A46043058F0C5F9043528465DB0BDEC39
:1000C000028BBDE8F08F0C204EF00EFB02204EF0AC
:1000D00011FB214606204EF013FC214606204EF06F
:1000E00093FC0A204BF030F804204EF033FB08EE6E
:1000F000100A002106204EF087FCB8EEC88ADFED1A
:10010000747A774D774E68EE277A36AF17EE900AFD
:1001100057F0A6F96AA3D3E9002357F0F9F957F08D
:10012000CFFCDBF84C30ADF8A8001A6818465369CC
:100130009847DBF85030ADF8AA001A681846136AE1
:1001400098476B68ADF8AC001A681846136F98476B
:10015000D5E90324BDEEC00ADBF810302C9210EE76
:10016000100AA6FB032399094FF47A720023ADF815
:10017000AE002E91DBE936012D9457F06FFEDBE9DE
:100180000C122F903091DBF83800DBF83C106B68D4
:100190003192CDE93201BBF85820ADF8D0201A6871
:1001A0001846536F9847BEEECF0ADBF86420DBF8A1
:1001B000143010EE101AADF8D210D2F80815ADF8C0
:1001C000D410A6FB03136969D2F80C25ADF8D6202C
:1001D0009B09CDE936310BF58E5404342AAE3546F1
:1001E0000FCDBD4220606160A260E3602E4604F145
:1001F0001004F4D103CE3C2520606160ACE60DF123
:10020000A80AAE000AEB0601514505913FF449AE3C
:10021000B210B2FA82F2C2F11F0252004FF0000394
:100220005046FDF721FB402E40F3A1826FF00303FF
:10023000A3EB0A0306932BA90DF1E8080E462A9BAF
:1002400056F8047B93F9283097F92800834240F34D
:100250000D828A4507D02CAB981B069B08449A193F
:10026000514658F0F9F82A9746453146E6D1059BA4
:1002700043453FF416AE0DF1E40E9C46A2464646B9
:10028000724658F8044B5EF8043B94F9281093F931
:100290002800884240F3B082414600E03A4641F8E7
:1002A000043D52F8043C94F9286093F928008642F2
:1002B000A2F10407F2DBC4451460E0D15446F0E536
:1002C0009A9999999999134054ED080048ED0800BE
:1002D00000803B3F6F12833A30AA0020C0A6002066
:1002E000FCA90020D34D62100DF1A80AAF000AEB63
:1002F0000701514505913FF4D4ADBA10B2FA82F22C
:10030000C2F11F0252004FF000035046FDF710F9F2
:10031000402F40F3EB806FF00303A3EB0A03069337
:100320002BA93AAEA0460EE08A4507D02CABD81BCD
:10033000069B0844DA19514658F08EF82A94BE42BA
:10034000394600F00C810F462A9B57F8044B5B6A34
:10035000606A9842E8D857F8083C5A6A9042A1F17E
:10036000040C40F24782384600E0F44640F8043D71
:100370005CF8043C616A5A6A9142ACF1040EF4D80C
:10038000CCF80040DBE70DF1A80AAE000AEB06014D
:10039000514505913FF485ADB210B2FA82F2C2F137
:1003A0001F0252004FF000035046FDF749F9402E5E
:1003B00040F320816FF00303A3EB0A0307932BA9FB
:1003C0003AAE0695A0460EE08A4507D02CABD81B66
:1003D000079B0844DA19514658F03EF82A94BE4269
:1003E000394600F09D810F462A9B57F8044B5B6A03
:1003F000626A9A42E8D357F8080C456AAA42A1F10A
:10040000040380F0FD81BC46069D00E073464CF875
:10041000040D53F8040C616A426A9142A3F1040E80
:10042000F4D306951C60DAE70DF1A80AAE000AEBDA
:100430000601514505913FF434ADB210B2FA82F293
:10044000C2F11F0252004FF000035046FDF780F941
:10045000402E40F325816FF00303A3EB0A030693BC
:100460002BA93AAEA0460F462A9B57F8044B93F9A6
:10047000283094F92800834280F2A280514507D0A9
:100480002CABD81B069B0844DA19514657F0E4FF01
:100490002A94BE423946E6D1059BB34244463FF416
:1004A00000AD0DF1E4089E46A2463746424656F896
:1004B000044B58F8043B94F9281093F9280088421B
:1004C00080F29481314600E0624641F8043D52F8E2
:1004D000043C94F9287093F928008742A2F1040C97
:1004E000F2DCB6451460E0D15446DAE405992BAB52
:1004F00099423FF4D6ACCDE9055498460C461D46CA
:100500000DE0AB1B9A4505D03044C6F104025146BC
:1005100057F0A2FF2A974445A6F1040644D040466E
:100520002A9B58F8047B5B6A796A9942E9D858F8A3
:10053000083C5A6A8A42AAEB060C80F05981404670
:1005400000E0F44640F8043D5CF8043C796A5A6ADD
:100550009142ACF1040EF4D8CCF80070DBE7059BB7
:10056000B34244463FF49DAC0DF1E40C9E46B046C8
:10057000624656F8047B5CF8043B796A586A884204
:1005800010D2B04600E0524648F8043D52F8043C10
:10059000786A596A8842A2F1040AF4D8B64517600D
:1005A000E5D17EE44246F9E7DDE9055479E41E46EB
:1005B00009ABB246082506931946B2E40026F7E7D0
:1005C00057F8082C92F928C08445A1F1040380F261
:1005D0001F81394600E0734641F8042D53F8042C7E
:1005E00094F928C092F928008445A3F1040EF2DCA6
:1005F0001C604EE7059B2BAE1A46B24206963FF4AE
:1006000050AC4FF0000812E0069BA3EB08039A459C
:1006100006D00CEB0800C8F10402514657F01CFF4D
:100620002A97059BB342A8F104083FF43AACB446BC
:100630002A9B56F8047B5B6A796A9942E4D356F8A0
:10064000080C426A8A42AAEB080340F2D780B446FB
:1006500000E073464CF8040D53F8040C796A426AC2
:100660009142A3F1040EF4D31F60DAE756F8082C88
:1006700092F928C08445A1F1040340F3C7803146B4
:1006800000E0734641F8042D53F8042C97F928C074
:1006900092F928008445A3F1040EF2DB1F60E3E524
:1006A000059B2BAE1A46B24206963FF4FAAB4FF0CA
:1006B000000811E0069BA3EB0803534505D0404416
:1006C000C8F10402514657F0C7FE2A97059BB34272
:1006D000A8F104083FF4E5AB30462A9B56F8047BAA
:1006E00093F9283097F928108B42E3DB56F8082C51
:1006F00092F928C08C45AAEB080380F28580314628
:1007000000E0734641F8042D53F8042C97F928C0F3
:1007100092F928008445A3F1040EF2DC1F60D5E7AE
:10072000059B069DB34244463FF4BBAB0DF1E40C80
:100730009E46B046624656F8047B5CF8043B796AF4
:10074000586A884211D9B04600E0524648F8043D44
:1007500052F8043C786A596A8842A2F1040AF4D338
:10076000B6451760E5D1FFF79CBB4246F8E7059B0D
:100770002BAE1A46B24206963FF493AB4FF00008F8
:1007800011E0069BA3EB08039A4505D04044C8F14D
:100790000402514657F060FE2A97059BB342A8F128
:1007A00004083FF47EAB30462A9B56F8047B93F94D
:1007B000283097F928108B42E3DC56F8082C92F980
:1007C00028C08C45AAEB08031CDD314600E07346C7
:1007D00041F8042D53F8042C97F928C092F9280009
:1007E0008445A3F1040EF2DB1F60D6E73A4678E6B3
:1007F0008446B1E68C46C3E532465CE5634633E7A2
:100800000B460FE60346EFE7034687E70B4645E74F
:100810000B46EDE62DE9F0472DED028B044682B044
:100820000D4607F089FE2946C4F8CC5004F56A60ED
:100830000CF048F904F16802D4F8CC1004F5067005
:1008400009F0A4F894F86D5094F86C2094F86E3088
:10085000A76E94F86F80D4F8CCA02D0404F57469C9
:1008600045EA026500214FF48472484645EA0325B3
:1008700057F00BFE0122894984F8C62F4FF0807291
:10088000874BC4F8401FC4F8442F40F201111622D0
:100890008448A4F8481F84F84A2F1E216422C4F813
:1008A0004C3F0023C4F8500FA4F8541FA4F8AC2FF9
:1008B00084F8AA3FA4F8C03F3F227B4904F65C704D
:1008C00058F007FF794AC4F8A02F40F20B502B21B3
:1008D0001022774BA4F8A40F3FBA48F0010884F81F
:1008E000A61FA4F8A82F41F205504C2600EB40109B
:1008F000304413F8016F002EF8D16E4A6E495368E8
:100900000193A1FB001C136801999FED6C7A59407B
:100910000B46D2E902124FEA5C1C5940682303FBE4
:100920001C0007EE900AF8EEE77A4A40F5EE006AFE
:10093000A7EEA67AC2F3072382F00A015940C2F358
:100940000743594041F2500381EA126289ED177A58
:100950005146E2544846FEF749F8594941F24C02E3
:1009600041F24803781E10F1030F88BF0F4645EA95
:100970000805A550E7504AF0DBFB41F2580304F5A7
:100980009F55E0503246D4F8CC1028460CF022FE99
:1009900028460DF0B5F838B104F5EB5201460432A3
:1009A000284601230CF050FF464D94ED4E0A68682E
:1009B00094F86061036894ED598ADB6B94F8617177
:1009C0009847686803683146D3F8E8309847686804
:1009D0000368B0EE480AD3F8E4309847394600225D
:1009E000686817F069FA686885F824600368082E5B
:1009F0001B6E8CBF102120219847284694F93C118A
:100A00000EF012FA94F814126868003118BF012130
:100A1000012217F053FD23682B49D3F898208A420E
:100A200038D194F83E21DAB9C4F8E020D3F89C30EC
:100A3000264A934222D194F83F3113BBC4F8E430E4
:100A400094F88A41224B234A23492448002C18BF9A
:100A50001A4602B0BDEC028BBDE8F0470EF046BE70
:100A60001F49204601FB02F107F04EFB2368C4F842
:100A7000E000D3F89C30154A9342DCD020469847DA
:100A8000DEE71849204601FB03F107F03DFBC4F8FF
:100A9000E400D5E7204690472368C7E741524E3926
:100AA0002C011E000A001400B0EF080000007A4379
:100AB000F0E30800F4D408004FECC44E0088614411
:100AC000EDAFEC0DFCA9002075CD020099CD020020
:100AD000A8EF0800ACEF0800C8EF080030AA00201B
:100AE000C0D4010080EE360010B59AB0D0F8CC101A
:100AF0000E4A01A8002328F0CBFC01A829F03CF9FC
:100B000090B10B4C08E001A828F0EEFD011EC9B21F
:100B1000204606DB49F05CF901A828F0ABFD00286F
:100B2000F1D101A829F0FCF81AB010BDE4E40800E6
:100B3000B065002010B59AB041680F4A01A80023A3
:100B400028F0A6FC01A829F017F990B10B4C08E099
:100B500001A828F0C9FD011EC9B2204606DB49F0F4
:100B600037F901A828F086FD0028F1D101A829F065
:100B7000D7F81AB010BD00BFE4E40800B06500204B
:100B800030B50C469BB00D490546204628F002FDC5
:100B900001A821460123094A28F07AFC01A829F07E
:100BA000EBF840B129464FF4847201A828F00AFD01
:100BB00001A829F0B5F81BB030BD00BFE4E3080080
:100BC0002DE9F04F0E789FB007461546002E00F035
:100BD00083800C4620468249984658F00CFD002838
:100BE0007AD0612E00F010812378642B00F0CB8145
:100BF00007227C49204657F015FC002840F0E7808A
:100C0000E679202E04F1070403D114F8016F202E99
:100C1000FBD02021204658F0E1FC8146002800F05E
:100C2000198316F0DF0F00F04C8363788DF80860AD
:100C3000002B00F0B183202B00F0AE83A2788DF85A
:100C40000930002A00F0AC83202A00F0A983E37861
:100C50008DF80A20002B00F0AB83202B00F0A88336
:100C600022798DF80B30002A00F02A82202A00F029
:100C7000278263798DF80C20002B00F09F83202BB6
:100C800000F09C83A2798DF80D30002A00F09A8341
:100C9000202A00F09783E3798DF80E20002B00F0D6
:100CA0009583202B00F09283227A8DF80F30002A52
:100CB00000F08E83202A00F08B834B4C0FCC2860F1
:100CC0006960AA6007CC2478EB602C7728616961A1
:100CD000AA611FB0BDE8F08F97F89A3097F8BA4034
:100CE0001A1C18BF012204B1013297F8DA0008B1CA
:100CF0000132D2B297F8FA1000294FD0003318BF52
:100D0000012304B1013308B10133DBB209B101336E
:100D1000DBB204220092A021344ADFF8E080DFF841
:100D2000E090DFF8E0A0284658F0CEFB97F9373284
:100D300007F19B04002614F8011CDAB2F0B2D1B11D
:100D4000002B42DB82420CBF52464A4634F8033C39
:100D5000019328212346009205A8424658F0B4FB8F
:100D6000284658F088FC05A9C0F19F02284658F093
:100D70008AFC97F937320136042E04F12004DAD1C7
:100D8000002BA6DB284658F076FC1949C0F19F02DB
:100D900028461FB0BDE8F04F58F075BC002AADD111
:100DA000144E06F1300734460FCCBC42286069600F
:100DB000AA60EB60264605F11005F4D107CE338812
:100DC000AB8128606960AA6083E74A46BEE70A49AA
:100DD00028464C221FB0BDE8F04F57F032BB00BF91
:100DE00064D608004CD80800DCD60800ACD6080051
:100DF000C8D608006CD60800B8D80800BCD60800D1
:100E0000A0E1090050D608006378642B04F10102C8
:100E10007FF4EAAE12F8013F642B7FF4E5AE53781D
:100E2000202B7FF4E1AE2379202B04F1040403D1BD
:100E300014F8013F202BFBD013F0DF0F00F0CA8124
:100E400062788DF80830002A00F09082202A00F0A5
:100E50008D82A3788DF80920002B00F08982202B49
:100E600000F08682E2788DF80A30002A00F0828253
:100E7000202A00F07F8223798DF80B20002B00F0D0
:100E80008582202B00F0828262798DF80C30002A56
:100E900000F08082202A00F07D82A3798DF80D2059
:100EA000002B00F07F82202B00F07C82E2798DF80D
:100EB0000E30002A00F07882202A00F07582237A12
:100EC0008DF80F2013B1202B7FF4F7AE08231EAA54
:100ED0001344002203F8702C97F84832002B00F0DE
:100EE000FF8197F81432002B00F00D8297F89A607A
:100EF00046B102AC214607F19B0058F042FB0028A6
:100F000000F06A8297F8BAA0BAF1000F08D002ACDC
:100F1000214607F1BB0058F034FB002800F0648242
:100F200097F8DA90B9F1000F08D002AC214607F12A
:100F3000DB0058F026FB002800F05C8297F8FAB03E
:100F4000BBF1000F08D002AC214607F1FB0058F0BE
:100F500018FB002800F0FE80002E00F00E82BAF18F
:100F6000000F00F03782B9F1000F00F00582032670
:100F7000BBF1000F00F0018228460423BF4AA021E4
:100F800058F0A2FAA5E66378652B04F101027FF41C
:100F90002FAE12F8013F6C2B7FF42AAE5378202B32
:100FA0007FF426AE2379202B04F1040403D114F836
:100FB000013F202BFBD013F0DF0F00F0738162782C
:100FC0008DF80830002A00F0E381202A00F0E0814B
:100FD000A3788DF80920002B00F0E081202B00F091
:100FE000DD81E2788DF80A30002A00F0DF81202AC6
:100FF00000F0DC8123798DF80B20002B00F0DA81E2
:10100000202B00F0D78162798DF80C30002A00F097
:10101000D381202A00F0D081A3798DF80D20002BF8
:1010200000F0CE81202B00F0CB81E2798DF80E30DC
:10103000002A00F0C981202A00F0C681237A8DF8A9
:101040000F2013B1202B7FF438AE08231EAA1344BF
:10105000002203F8702C97F89A3002AC3BB121467D
:1010600007F19B0058F08DFA002800F0B98197F83D
:10107000BA303BB1214607F1BB0058F082FA002894
:1010800000F0AC8197F8DA303BB1214607F1DB0084
:1010900058F077FA002800F0B28097F8FA3043B1A0
:1010A000214607F1FB0058F06CFA0322002800F0FB
:1010B000A78023462846724AA02158F005FA08E680
:1010C00004231EAA1344002203F8702C97F89A30C8
:1010D00002AC3BB1214607F19B0058F052FA0028C0
:1010E00000F0848197F8BA303BB1214607F1BB008C
:1010F00058F047FA002800F07B8197F8DA303BB1CE
:10110000214607F1DB0058F03CFA002800F06A8124
:1011100097F8FA30002BCCD0214607F1FB0058F0AD
:1011200030FA03260028C4D109F1010057F02DF848
:1011300040F2CB73421F9A42814640F2F380514CF9
:101140000FCC28606960AA6007CCEB6028616961F8
:10115000AA61BEE503264FFA86F97601BA194FF067
:10116000010A82F89AA0D7E98E01C2E9220197ED1F
:10117000907B06F19B0082ED247B2146384458F099
:1011800044FA4149404628F005FA05A8534641462D
:101190003D4A28F07DF905A828F0EEFD40B14FF456
:1011A0008472394605A828F00DFA05A828F0B8FD84
:1011B0003E44364B364AB6F898100191B9F1FF3FDC
:1011C00018BF1A46009223462846324AA02158F0FA
:1011D0007BF97EE5304E06F1300734460FCCBC4239
:1011E00028606960AA60EB60264605F11005F4D11D
:1011F0003068B288B3792860AA80AB7169E50222B1
:1012000007EB42130021A3F89A1097F937321E49D1
:10121000934204BFFF2387F83732404628F0BAF9DB
:1012200005A841460123184A28F032F905A828F0FC
:10123000A3FD40B139464FF4847205A828F0C2F9E5
:1012400005A828F06DFD23462846144AA02158F031
:101250003BF93EE5124E06F1200734460FCCBC4266
:1012600028606960AA60EB60264605F11005F4D19C
:101270002068A3882860AB802BE500BF8CD70800CE
:1012800018D808007CD80800E4E3080054D6080009
:1012900060D60800D0D70800FCD6080034D8080073
:1012A00054D80800544E06F1300734460FCCBC42E7
:1012B00028606960AA60EB60264605F11005F4D14C
:1012C00096E74D4E06F1300734460FCCBC422860FD
:1012D0006960AA60EB60264605F11005F4D187E746
:1012E000464E06F1200734460FCCBC4228606960A8
:1012F000AA60EB60264605F11005F4D12068237939
:1013000028602B71E5E43E4E06F1300734460FCCE1
:10131000BC4228606960AA60EB60264605F11005B2
:10132000F4D1D6E407EB46163649A6F898004046B5
:1013300028F030F905A841460123324A28F0A8F8E0
:1013400005A828F019FD40B139464FF4847205A86C
:1013500028F038F905A828F0E3FCCDF800902346E2
:101360002846294AA02158F0AFF8B2E40123AEE59F
:101370000223ACE50323AAE5022607EB4613642209
:10138000A3F898204FF0FF3902ACE6E604239EE56F
:1013900001235BE605239AE5012392E6022355E645
:1013A00002238EE6062392E5072390E503234DE60C
:1013B000032386E6042349E6052347E6052380E662
:1013C000062343E606237CE607233FE6072378E669
:1013D000082376E60126D0E70646BCE601220FE7A1
:1013E00002460DE702269FE60126B4E606469BE686
:1013F000012699E60226AEE6FCD6080034D708009E
:101400005CD70800E4E3080098D808002DE9F04F05
:101410002DED028B0E78B7B004461746002E61D032
:101420000D462846C349994658F0E5F8002859D09A
:10143000C149284658F0DFF88246002800F028828B
:10144000BE49284658F0D7F8002800F06181BC4911
:10145000284658F0D0F8002800F0C381B949284642
:1014600058F0C9F8002800F0BC810922B649284686
:1014700056F0D8FF002800F04A820A22B3492846D5
:1014800056F0D0FF002840F07F82B14905F10A00F4
:1014900058F077F8B0FA80F0400984F88600AD493A
:1014A000484628F077F81DA849460123A94A27F0A5
:1014B000EFFF1DA828F060FC40B14FF48472214674
:1014C0001DA828F07FF81DA828F02AFC94F8864073
:1014D0009F4BA14AA1493846002C18BF1A4658F024
:1014E00027F8C3E0D4ED177A66799FED9D6ADFF89F
:1014F000B8A294F90AE09B4994F806B0FDEEE76AB9
:10150000B6EE007AF8EEE65A330177EEE57A1293FA
:10151000A7EE867A534419AD93F90CC0FDEEC77A55
:10152000E645764617EE903AA8BF664616EE902A34
:101530004FF0000C28461096C5F804C0CDF864C0E2
:10154000C5F808C0A5F80CC057F0F2FF94F8099050
:10155000B9F1000F00F09080B4F81C81B8F1000FD1
:1015600040F0B1800DF174084B4640467E4A202180
:1015700057F0AAFF0DF15809A38A002B40F089808B
:101580007A4B94F8812093E803000B0C8DF85E30C1
:101590001690ADF85C10D4F80831002A40F0858030
:1015A00014AA1192DBB210460521714A57F08CFF44
:1015B000D4F80831129A94ED067A6E495AF802204E
:1015C000D4ED187A6C4802920BEB4B066B4A51F83B
:1015D000266094F90A100095B5EEC07AF1EE10FA83
:1015E0000396119D94F807C00F95CCBF054615468C
:1015F0000195DFF8B8E1109D614EDFF8B4B13846CF
:10160000277A0E9394F886A0CDF83480A942D8BFEB
:1016100096465C49504BDFF89C81BCF1000F08BF37
:10162000164694F804C00795CDF81890002F0CBF0B
:1016300015465D46BAF1000F0CBF17460F4694F8E9
:1016400064200492FDEEE77A94F880404E4ACDF88B
:1016500020E0BCF1000F18BF4346A021CDE90A6588
:101660000C97CDED057A099457F02EFF012037B085
:10167000BDEC028BBDE8F08F444B93E80300A38AD6
:101680000DF1740888E803000DF15809002B3FF4B0
:1016900077AF3F4A0A21484657F016FF94F8812059
:1016A000D4F80831002A3FF47BAF139314AB1846EB
:1016B000042204F18101119358F00BF800228DF8F7
:1016C0005420139B76E749F033FD94F81E31002B2C
:1016D00072D1D4F818212F4B801A03FB08F3B3FB07
:1016E000F9F9814568D92C4BA9EB0009A3FB092323
:1016F0009B0B3B2B40F23681284B294AA3FB091355
:101700000DF158095B0D48460A2157F0DDFE58E0FF
:10171000014604F59670234C282256F0B6FE0FCCF5
:101720003860A58820687960BA60FB603861BD8246
:101730009CE700BFDCD9080080DA080018DB08004D
:101740003CDB080044DB080074E0080094E008007B
:1017500000040900E4E3080064F30800A0E00800C6
:1017600000007A4444D60800ECD9080020DA0800CA
:1017700030DA080004D5080050D60800A0E10900BE
:1017800010D9080020D9080038DA0800E4D9080088
:1017900028DA080080EE360073B2E745B17C219567
:1017A000FCD9080024DB080064D5080008D908002B
:1017B00018D9080004D908000DF1D8098C4B49F854
:1017C000803D637ACDF804900DF17408B4F81C11D3
:1017D000884A91FBF3F140460091202157F074FEB6
:1017E000CAE68549854848F0C3FB8549834848F0E7
:1017F000BFFB8449814848F0BBFB83497F4848F0E0
:10180000B7FB82497D4848F0B3FB81497B4848F0EB
:10181000AFFB8049794848F0ABFB7F49774848F0F7
:10182000A7FB7E49754848F0A3FB7D49734848F003
:101830009FFB7C49714848F09BFB7B496F4848F00F
:1018400097FB7A496D4848F093FB79496B4848F01B
:101850008FFB7849694848F08BFB7749674848F027
:1018600087FB7649654848F083FB7549634848F033
:101870007FFB7449614848F07BFB38468F227249F0
:1018800056F0DFFD012037B0BDEC028BBDE8F08FD4
:1018900049F04EFC0DF17408D4F84C6105465146F0
:1018A0004046282256F0F1FD5EB1684BAD1BA3FB0C
:1018B00005239B0B3B2B5DD8654A2821404657F0FA
:1018C00003FED4F84811D4F83021D4F82C31CDF8E7
:1018D0002080D4F844010791D4F83C510692D4F802
:1018E00040110593D4F83421D4F838310490CDE96F
:1018F0000032CDE902153846564B574AA02157F021
:10190000E3FD012037B0BDEC028BBDE8F08F5349F9
:1019100005F1090057F035FEB0FA80F04009E0719A
:101920004F49484627F036FE1DA8494601234C4A38
:1019300027F0AEFD1DA828F01FFA40B14FF48472C5
:1019400021461DA827F03EFE1DA828F0E9F9E479FC
:10195000424B444A44493846002C18BF1A4657F0B7
:10196000E7FD83E60DF158094846404A0A2157F041
:10197000ABFD26E73E4B3F4AA3FB05135B0D282139
:10198000404657F0A1FD9CE709223B49284656F006
:1019900049FD002874D1314905F1090057F0F1FDE6
:1019A000B0FA80F0400920722D490DF174084846C4
:1019B00027F0F0FD404649460123294A27F068FDFB
:1019C000404628F0D9F940B14FF484722146404690
:1019D00027F0F8FD404628F0A3F9247A1F4B214A4E
:1019E00026493846002C18BF1A4657F0A1FD3DE69F
:1019F0006E6F77000CDA080048DB0800B065002045
:101A000074DB0800A0DB0800E0DB080010DC080045
:101A100050DC08009CDC0800DCDC080018DD080055
:101A200060DD0800A0DD0800ECDD080028DE08000D
:101A300074DE0800B8DE0800F8DE080038DF0800B1
:101A400074DF0800A0DF0800E4DF080073B2E74598
:101A5000A0DA0800B8DA0800C0DA080000040900BB
:101A6000E4E3080064F3080080E0080004DA0800FA
:101A7000B17C219588DA0800B4E00800C0E00800D5
:101A80009949284657F0B7FD002874D09749284651
:101A900057F0B1FD002800F089809549284657F09D
:101AA000AAFD002800F08E809249284657F0A3FD39
:101AB000002800F09F809049284657F09CFD0028A0
:101AC00000F0FA8007228D49284656F0ABFC00282A
:101AD00040F0A88007352846894957F052FD002874
:101AE00000F027828749284657F04BFD002800F078
:101AF0001D828549284657F044FD002800F0648384
:101B00008249284657F03DFD002800F05A8380495D
:101B1000284657F036FD002800F050837D492846BE
:101B200057F02FFD002800F046837B49284657F0E8
:101B300028FD002800F015822846784957F021FD3D
:101B4000002800F0D981764C04F1200625460FCDFF
:101B5000B54238607960BA60FB602C4607F1100727
:101B6000F4D1234607CB1C889B7838607960BA6033
:101B7000BC81BB737AE501256A492571484627F087
:101B800009FD1DA82B464946664A27F081FC1DA881
:101B900028F0F2F840B121464FF484721DA827F0D6
:101BA00011FD1DA828F0BCF85F4BDBE7207149460A
:101BB0002046FEF7E5FF5D4C0FCC38607960BA60D7
:101BC000FB6053E55A4D012305F1200684F81F31CF
:101BD00084F81E312C460FCCB44238607960BA606C
:101BE000FB60254607F11007F4D128682B7938608F
:101BF0003B713BE54F4B504A504C168803CB1B784A
:101C00003B723860796004F16005384657F033FD67
:101C10003E52431C54F80C1BF81857F0F6FCAC422B
:101C2000F3D123E507224649284656F0FBFB00285E
:101C300000F0968008224349284656F0F3FB00281E
:101C400000F08E8005224049284656F0EBFB064600
:101C5000002840F0FA80053528463C4957F091FCB1
:101C600048B13146284658F093FBB5EE400AF1EEF4
:101C700010FA40F0AC810023A3612046344DFCF7FC
:101C8000BBFD49462046FEF77BFF0FCD2D783D7406
:101C900038607960BA60FB6094ED170A3846FCF74B
:101CA0007FFE384657F0E7FC2A4A03463918106889
:101CB0001279F8500A71D9E4274B1F4A274C16882D
:101CC00003CB1B783B723860796004F1E00538463D
:101CD00057F0D1FC3E52431C54F8101BF81857F033
:101CE00094FCA542F3D1C1E40004090064F30800A8
:101CF000F4E0080024E1080038E108004CE10800A5
:101D0000F0E3080050D9080058D9080064D9080049
:101D100070D908007CD9080088D9080044D9080087
:101D200054E10800E4E30800D4E00800E4E008001F
:101D3000FCE008002CE10800DCE3080004D5080002
:101D400084E108008CE10800C8E10800D0E1080047
:101D5000D8E10800ECE1080040E1080064D5080083
:101D6000722E0CBF07350835C149284657F009FCCB
:101D7000002800F01D82BF49284657F002FC0028C9
:101D800000F01382BC49284657F0FBFB002800F006
:101D90000982BA49284657F0F4FB002800F0FF8179
:101DA000B749284657F0EDFB002800F0F581B5490A
:101DB000284657F0E6FB002800F0EB81B2492846A0
:101DC00057F0DFFB002800F0E181B049284657F0CA
:101DD000D8FB002800F0D781AD49284657F0D1FB49
:101DE000002800F0EB80AB49284657F0CAFB0028DA
:101DF00000F0E180A849284657F0C3FB002800F016
:101E0000D780A649284657F0BCFB002800F0CB80BD
:101E1000A349284657F0B5FB002800F0D580284696
:101E2000A04957F0AEFB002800F0CB809E4C04F197
:101E3000200625460FCDB54238607960BA60FB6058
:101E40002C4607F11007F4D18BE609229749284662
:101E500056F0E8FA002800F0CD8106229449284681
:101E600056F0E0FA002800F0B28105229149284698
:101E700056F0D8FA002800F066810A228E492846DA
:101E800056F0D0FA002800F0418106228B492846FE
:101E900056F0C8FA804600284ED1AB7904F181068D
:101EA000063533B18649284657F06BFB002840F0D1
:101EB000B480002384F8813049462046FEF760FE56
:101EC00094F88120D4F80831002A4DD10DF174081E
:101ED000DBB240467B4A052157F0F6FA94F8815070
:101EE000794B7A4C7A4942463846002D18BF234632
:101EF00057F01EFBFFF7BABB764D07230022A371F4
:101F0000A2612046FCF778FC49462046FEF738FEE1
:101F1000714B18681B7938603B712946781D57F062
:101F200027FB6E4A034610681860B5E601236C4D26
:101F3000E4E703466B4DE1E705226B49284656F07E
:101F400071FA8046D8B1694C0FCC38607960BA60BC
:101F500007CC2488FB60BC8338617961BA61FFF7E4
:101F600085BB0623624DC9E70DF174083146404632
:101F7000042257F0AEFB00238DF87830AEE704F171
:101F80001C06691D3F22304657F0A3FB49462046F8
:101F900084F85B80FEF7F4FD32463846554957F029
:101FA000C7FAFFF763BB3D4D0B2300226371A7E720
:101FB0000A23394DF9E70923364DF6E70823344D56
:101FC000F3E7384D0D23F0E70C23354DEDE72846B8
:101FD000002158F0DDF9DFED487AB4EEE70AF1EEC2
:101FE00010FAB0EE408A06D4DFED447AB4EEE70A88
:101FF000F1EE10FA19DD424D05F120062C460FCC0A
:10200000B44238607960BA60FB60254607F110077A
:10201000F4D120683860FFF729BB294604223046F6
:1020200057F057FB84F8858046E784ED060A204682
:10203000FCF7E2FB20464946FEF7A2FD314B324C4D
:1020400003CB1A889B7879603A81BB723860B0EE16
:10205000480A3846FCF7A4FC384657F00CFB054606
:102060000FCC7C1978516160A260E360FFF7FEBA83
:10207000DC0709009CD90800A4D90800ACD90800E5
:10208000B0D90800B4D90800B8D90800BCD90800F4
:10209000C0D90800C4D90800C8D90800D0D90800A0
:1020A000D4D9080094D9080098E1080034E2080067
:1020B000B0E20800DCE2080008E3080080E3080062
:1020C000D0E1080030DA08003CD90800A0E109009E
:1020D00088E3080044D90800D8E30800E0E30800DA
:1020E00050D90800F0E30800A0E30800B8E30800B6
:1020F00088D90800A8E308000000164300007044D7
:10210000F4E1080018E2080024E2080005F10A00E2
:1021100056F03BF8FF28054600F2D0806072494631
:102120002046FEF72DFD3DBB6F4D05F120062C46E8
:102130000FCCB44238607960BA60FB60254607F185
:102140001007F4D151E5681D56F01FF80328054625
:1021500000F2C88084F8800049462046FEF710FD52
:10216000624A634B6349002D18BF134638462A461E
:1021700057F0DEF9FFF77ABA2A4638465E4957F03B
:10218000D7F9FFF773BA07235C4D0EE706235C4DC2
:102190000BE705235B4D08E704235B4D05E70323AD
:1021A0005A4D02E702235A4DFFE60123594DFCE642
:1021B0000346594DF9E60523584D9FE60423584D33
:1021C0009CE60323574D99E60223574D96E6A81D3A
:1021D00055F0DBFF00F109031F2B054630D9534CA6
:1021E0000FCC3860796003CCBA60FB6038617961EC
:1021F000FFF73CBA05F1090055F0C7FFB0F5B46F21
:10220000054643D8A08238BBC4F82401494620467D
:10221000FEF7B6FC464C04F1200625460FCDB5422C
:1022200038607960BA60FB602C4607F11007F4D182
:102230002868AA88AB793860BA80BB71FFF716BAF4
:10224000A07249462046FEF79BFC2A46384639498B
:1022500057F06EF9FFF70ABA48F06AFFA68A4EF601
:10226000602303FB060644F62161002048F022FFAC
:102270003044C4F8240149462046FEF781FC2A4632
:1022800038462D4957F054F9FFF7F0B92B4C04F1BB
:10229000200625460FCDB54238607960BA60FB60F4
:1022A0002C4607F11007F4D12B4603CB1A889B78F4
:1022B000386079603A81BB72FFF7D8B9204D05F1DB
:1022C00020062C460FCCB44238607960BA60FB60BF
:1022D000254607F11007F4D12288A3783A80BB7015
:1022E000FFF7C4B9174C67E438E30800A0E1090020
:1022F00028D90800F4E2080060E30800BCD908000F
:10230000B8D90800B4D90800B0D90800ACD9080081
:10231000A4D908009CD90800DC0709007CD9080072
:1023200070D9080064D9080058D90800B8E208003C
:1023300088E20800D0E208006CE2080040E20800F1
:1023400014E30800E4E208002DE9F04741F6945553
:102350008946415DAEB0804614461F46002940F0D4
:102360009B801378202B03D114F8013F202BFBD046
:10237000204657F080F9042803D9A3787C2B00F07D
:102380002D810822C349204656F04CF8064628BB4A
:1023900008342046202157F021F9002800F07881E8
:1023A00000F10109A9EB0403402BA8BF402303EB74
:1023B000D3735D1006702246294615A806F0ACFFBF
:1023C000002840F0BA80B44C0FCC24783C743860BC
:1023D0007960BA60FB602EB0BDE8F087B9F1000FFC
:1023E00034D1AE49204657F006F9054670BBAC49DA
:1023F000AC4847F0DDFDD8F89CCEBCF1000F20DDE5
:10240000DFF8C8A2A74EDFF8C89208F5077494F861
:102410002030514630461A46002B00F0CA8147F062
:10242000B1FE21462022304606F05AFF494630468A
:1024300047F0A8FED8F89CCE0135654504F1A0040C
:10244000E5DB00233B702EB0BDE8F08712229649F1
:10245000204655F0E7FF002840F08E80A57C202D17
:1024600004F1120403D114F8015F202DFBD0002DDC
:1024700000F0CF808D4D05F120062C460FCCB442E4
:1024800038607960BA60FB60254607F11007F4D127
:1024900003CD386079609EE710460CF0FBF9002808
:1024A00040F0A2802378202BA14640F07E8114F8D2
:1024B000013F202BFBD0A4EB090909F1FF3A254687
:1024C0002E46013530780BF071F80028F8D13378BA
:1024D0004BB1737830702E461BB904E016F8013FFB
:1024E0000BB1462BFAD1BAF1060FAAD82378002BEC
:1024F000A7D008EB890941F63C5359F80350002D49
:102500009FD008F59F5021460BF034FA08F5C458C7
:102510002A8808F110080546002800F0518121465C
:1025200040462B880BF0ECF800288AD02B790371F9
:1025300009F5EA59C9F8000083E7484655F025FE39
:10254000C0B200902B4615AA08F1680108F5067084
:1025500007F026FB002800F0908041F288314046C9
:1025600005F0D2FD524B41F698511A889B7848F8F5
:1025700001003A80BB702EE708224E49D8F8CC50B3
:10258000204608F5746657F092F828B9237A13F0BC
:10259000DF0F04F1080116D007224749204657F003
:1025A00086F830B9E37913F0DF0F04F1070A00F081
:1025B00093803B462246494608F56A6009F082FB53
:1025C00009E711F8013F202BFBD02B4630463A4655
:1025D000FEF71CFF00287FF4FEAEEAE734F8032B79
:1025E0003A80BB700337CCE608F5C45110314FF484
:1025F000966208F59F5055F024FF41F2EA3200231D
:1026000038F802202D4908F80530384656F090FF7A
:10261000E1E62EAC4FF4906324F8643DD8F86000F6
:10262000036804221B680DF15601984741F68C534C
:10263000DDF8562048F803204EF66021404605F0AC
:1026400063FD41F69053214648F803000A224046B4
:10265000CDF85A5006F084F920B101462A4640468A
:1026600006F07CFD164C0FCC2588A4783860796084
:10267000BA60FB603D82BC74ADE6124C0FCC386092
:10268000257920687960BA60FB6038613D75A2E603
:102690000D4C99E654E5080090E50800A4E5080013
:1026A000ACE50800B0650020BCE50800D0E50800F6
:1026B00074E508000CE60800B8DA08003CE50800FC
:1026C000F8E5080078E5080060E50800B4E50800D2
:1026D00054E408001AF8013F202BFBD0002B7CD0DB
:1026E000A949504656F087FF002876D0A7495046A2
:1026F00056F081FF002800F07781A549504656F03A
:102700007AFF002800F07081A249504656F073FF0E
:10271000002800F0FE81A049504656F06CFF0028CA
:1027200000F026829D49504656F065FF002800F0D3
:102730005B8205229A49504655F074FE002800F04D
:102740003C8207229749504655F06CFE002800F065
:102750009C820C229449504655F064FE002800F0FB
:102760007E8206229149504655F05CFE002800F01A
:102770003E8304228E49504655F054FE002840F016
:1027800007839AF8043013F0DF0F40F0FF820AF15C
:10279000040A51460AF1010A0B78202BF9D02B4686
:1027A0003A463046FEF70CFA15E681464FF0FF3AFE
:1027B00085E60135654504F1A004FFF628AE40E644
:1027C0000346214640460AF09BFF00283FF439AEFD
:1027D0003378463B18BF0123A9E641F2771341F253
:1027E000741418F9033018F80490002BC0F24C81CF
:1027F00006EB431303F19B0415AD2846202200216C
:1028000055F043FEB9F1000F24D041F2701658F88C
:102810000630002B1EDB48F08BFC41F2681241F2BF
:10282000541358F80220DFF8B8E118F803C06149E2
:1028300058F80630821A6048AEFB0262BCF1000F05
:1028400018BF0146920BCDE9001228465B4A2021B1
:1028500056F03AFEB8F8523F002B40F08B80584BB0
:1028600093E803000CAE86E8030098F8DA3F98F886
:10287000FACF1A1C18BF0122BCF1000F00D00132A0
:1028800041F21A0118F8010008B10132D2B241F246
:102890003A0118F80110002955D1002A53D1494BAB
:1028A00093E803000DF13C0A0F90ADF8401041F29F
:1028B000BD130DF1480918F803300022C9F80420AF
:1028C0001292C9F80820002B40F0D88098F8443FB5
:1028D000002B56D041F2741318F80330002B00F08F
:1028E000CB8041F2771318F90330002BC0F2E5805A
:1028F0003549364BCDF8249008F58D50CDF81CA005
:1029000090F800E0DFF8DCC0314A069641F248005A
:10291000BEF1000F18BF6246B8F84CEFB8F84ECFC2
:1029200058F80090B8F8506F0596CDE9015108921B
:1029300000943846CDF82890CDE903EC254AA02133
:1029400056F0C2FD47E5003318BF0123BCF1000F6C
:1029500000D0013308B10133DBB209B10133DBB27E
:102960000DF13C0A0422009250461B4A0A2156F0FF
:10297000ABFD9CE70CAE3046184A0A2156F0A4FD88
:1029800073E70D49044BB5E7DCD908003CDB0800D0
:1029900044DB08000004090064F30800F4E00800C8
:1029A00050EB08004CD80800CCEB080030EC0800D5
:1029B00054D7080020E50800A0E1090018E6080047
:1029C00028E6080038E6080028E5080004D90800D1
:1029D00034E5080050E6080040E6080030E608004C
:1029E00073B2E74560D60800C149C24847F0C0FA53
:1029F000C149C04847F0BCFAC049BE4847F0B8FAE0
:102A0000BF49BC4847F0B4FABE49BA4847F0B0FAEB
:102A1000BD49B84847F0ACFABC49B64847F0A8FAF7
:102A2000BB49B44847F0A4FABA49B24847F0A0FA03
:102A3000B949B04847F09CFAB849AE4847F098FA0F
:102A4000B749AC4847F094FAB649AA4847F090FA1B
:102A5000B549A84847F08CFAB449A64847F088FA27
:102A6000B349A44847F084FAB249384679222EB0D7
:102A7000BDE8F04755F0E5BCAF493AE7AF4A0C2155
:102A8000484656F021FD21E798F8443F002B34D00A
:102A9000B9F1000F5ED0B8F8521F00297BD141F286
:102AA000761318F80340022C00F0C880A44AA54B06
:102AB000012C14BF14461C469EE6B8F8523F002B6A
:102AC000DAD048F035FB41F26813B8F8522F58F8C5
:102AD00003E09D4BDFF860C29C4903FB02F3A0EBCF
:102AE0000E009B4A98F844EF984238BF6146994BD4
:102AF000BEF1000F08BF1346FCE641F2761241F228
:102B0000741318F8024018F80390022CCED1924C9E
:102B100072E60124914988F8444F284626F03AFD90
:102B200015A8234629468D4A26F0B2FC15A827F0A1
:102B300023F940B131464FF4847215A826F042FDC6
:102B400015A827F0EDF8864C0FCC38607960BA6094
:102B5000FB6040E441F2761318F80340022CA5D143
:102B600015AD49462846202255F08FFC7A4C71E677
:102B700088F8440F7949284626F00CFD15A8294607
:102B80000123764A26F084FC15A827F0F5F80028E2
:102B90005BD1744C18E448F0CBFA41F26813B8F8F2
:102BA000521F58F80320684B821A03FB01F39A4224
:102BB000A3D318F804906C4C1EE60AF1050055F0FA
:102BC000E4FA6A4BA0F11E029A42044629D9684CE5
:102BD0000FCC3860796003CC2478BA60FB603C7617
:102BE00038617961FFF7F7BB41F25F0141F25E02A4
:102BF0000123604D08F8013008F8023005F1200685
:102C00002C460FCCB44238607960BA60FB60254630
:102C100007F11007F4D128682B7938603B71FFF772
:102C2000DABBA8F84C0F29463046FDF7A9FF22462B
:102C30003846514956F07CFCFFF7CDBB15AD284610
:102C4000202255F022FC444CDFE531464FF48472DB
:102C500015A826F0B7FC15A827F062F899E70AF145
:102C60000C0055F092FAB0F5167F044625D9434C76
:102C70000FCC38607960BA6007CC2478FB603C7771
:102C800038617961BA61FFF7A6BB0AF1070055F018
:102C90007CFA40F2CB73421F9A4204461AD9384C50
:102CA0000FCCA58838602068A4797960BA60FB6091
:102CB0003861BD82BC75FFF78EBBA8F8500F29465E
:102CC0003046FDF75DFF224638462E4956F030FC6F
:102CD000FFF781BBA8F84E0F29463046FDF750FF9D
:102CE00022463846284956F023FCFFF774BB00BF44
:102CF00090E60800B0650020BCE60800F0E6080099
:102D000038E708007CE70800C0E7080008E808008A
:102D100058E808008CE80800E0E8080008E9080026
:102D20004CE908008CE90800D8E9080024EA08000A
:102D300068EA0800B0EA0800A0E1090048E60800D7
:102D400018E5080034EF080080EE360028E508009A
:102D500064F3080004D9080010E50800E4E3080063
:102D60002CEB08003CEB080004E508006251010070
:102D700058EB0800FCE0080074EB0800DCEB0800EE
:102D800098EB0800FCEB0800B0EB0800354C6FE74F
:102D900004223549504655F045FB0028F6D19AF8F3
:102DA000043013F0DF0FF1D10AF1040A54461AF887
:102DB000013B202BFAD0002B4CD02C49204656F05A
:102DC0001AFC00283ED007222949204655F02AFB4C
:102DD000A0BBE31D15A8274A202156F075FB2B4602
:102DE0003A4615A93046FDF7EBFEFFF7F4BA0AF1B3
:102DF000060055F0CAF9B0F5347F04460FD8A8F89C
:102E0000520F29463046FDF7BBFE0CB91A4CDFE6DF
:102E100022463846194956F08BFBFFF7DCBA184DAD
:102E200005F120062C460FCCB44238607960BA60B8
:102E3000FB60254607F11007F4D1ECE63846422244
:102E4000104914E62B463A4630460F49FDF7B8FEC6
:102E5000FFF7C1BA2B463A4630460C49FDF7B0FEA3
:102E6000FFF7B9BA28ED0800B8EC0800C0EC08007C
:102E70004CD80800D4EC080060EC08007CEC08009A
:102E800038EC0800E4EC0800C8EC0800B4EC0800DA
:102E90002DE9F04F03F69413B5B050F82350002DF0
:102EA00024DBD0F89C3E9D4204461FDA4FEA850A97
:102EB0000AEB05077F0107F1040800F506790E46C5
:102EC000C844B2B93F9B00EB070A1D68DAF8A0328C
:102ED000AB420BD2409B043B00933F9B2A460433FA
:102EE0004146FCF799FF8346002874D135B0BDE810
:102EF000F08F022AFAD1409B052BF7D998F82030A1
:102F000003F00303032BF1D13F9B1B799B10012B93
:102F1000ECDC0693C2193F9BD2F8A0B21B68059364
:102F20009B45E3D8C2F8A032C06D079201680968DA
:102F300088473F9B079A0533C2F8A4020793409A3B
:102F40003F9B00219954069B002B00F09180059B2C
:102F50009B4540F084800DF1D00B00230BF8A33D7E
:102F6000584656F088FB83460028BFD0E36D069391
:102F70001A68184612689047069B5A68904298BF94
:102F8000501C5860059B834208BF01300BF10503BC
:102F90000AA9019300914FF0040C02210A904246C5
:102FA0003E9B8DF82CC0204605F09AFC0146002877
:102FB0009CD00AEB050304EB431393F83D32FF2B3F
:102FC0007ED007F126024FF416754A44204600953C
:102FD00005F04AFD8AE7CAF8A052E06D03681B6855
:102FE0009847CAF8A402337803F00303012B04F5D1
:102FF0008E521AD833790120CDE90030CDE9022B69
:10300000414606F10A033E9A204605F0B3FB00282C
:103010003FF46CAFB3889B1101330146DBB220460D
:103020004FF49672FCF7EEF860E7CDE9002B3E9B7B
:1030300042460121204605F053FC00283FF456AFDC
:103040009AF83D32FF2BE5D007F126024FF4967532
:1030500001464A442046009505F006FD46E70DF17D
:103060002D0B1946079A5B462046FFF76DF977E767
:10307000079856F000FB2022431DCDE90082042171
:103080003F9A0AA806F0CEF934A90A9B41F8AC3D54
:103090000422204605F052FC014600283FF457AFB9
:1030A000A02303FB054393F83D32FF2B12D007F119
:1030B0002602C82000904A44204605F0D5FC46E789
:1030C000B3889B110133DBB220464FF41672FCF734
:1030D00099F80BE7B3889B110133DBB2C822204675
:1030E000FCF790F833E700BF10B5054B044640F8F5
:1030F0002C3B16F051F8204617F0F6F8204610BD8C
:10310000D0D4080010B5074B044640F82C3B16F00D
:1031100043F8204617F0E8F820464AF0F1FB204635
:1031200010BD00BFD0D408002DE9F04F2DED028B6B
:10313000ADF26C4DC4799DF898B41CB9047A002C9A
:1031400000F06D8210930391437990F90A1090ED8D
:10315000178AD0ED188A90F8645090F86580B0F81E
:10316000686090F866708146A04800EB03139246B1
:1031700093F90C4012688C4212695046A8BF0C4665
:10318000904703999A4A0B689B6C934240F0A8863B
:1031900048680368B0EE480ADB6B9847039A5068AA
:1031A00003682946D3F8E8309847039B58680368BA
:1031B000B0EE680AD3F8E4309847039841460022FD
:1031C000406814F079FE0399486881F82450036838
:1031D000082D1B6E8CBF10212021984744223946B0
:1031E000504614F09FFEDAF80030824D1B6E3146D7
:1031F00050469847214603980BF016FE0426DAF84D
:1032000000305046D3F890309847A8B947F090FF67
:10321000074607E0D3F898309847431C04464CD142
:103220004BF0B2F847F084FFC31B312B5046DAF85D
:103230000030EFD91B69984799F88630BBF1000F31
:103240006AD099F8081099F8072039B11099097EC9
:1032500021B199F83612022900F0A186002A00F067
:103260006386DAAD00222A70002B40F0F48101243D
:10327000039803683C219B68984740F6C4133C3090
:10328000B3EB400F80F0FC8599F82831A3422CBFA6
:1032900000235A1CE95C99F81E318DF8541034BF94
:1032A000D2B2012215A80C9089F82821002B00F039
:1032B0007286022343700D933FE0DAF800305046E7
:1032C0001B699847AC42B7D15021002047F0F2FE6D
:1032D000143047F039FF013E91D1D9F830311098C0
:1032E0000133C9F8303190F9331090F8324090F83A
:1032F000313090F83020D0ED0B0A90ED0A0A0191A0
:10330000039800945146FCF7CDF930460DF26C4D10
:10331000BDEC028BBDE8F08F15A901220A808A70EE
:103320000C9199F81E21002B40F08A81002A00F0B0
:103330000E860223CB7004230D93002312930F9368
:10334000CDE906330B93139309930C9B049301234C
:103350000893CB46CDF838A0049A12F8013B032B12
:10336000CDE9042300F07882002B40F07E839BF8A7
:103370000730002B00F0DE80109B1B68002B00F054
:103380007C8519781C4A002908BF13461B4A1DA8D2
:103390002C2156F099F89BF88130DBF80841002B7E
:1033A00040F0938517ADE3B22846154A052156F043
:1033B0008BF8DBF80841134A0DF51E7A23460C21E1
:1033C000504656F081F862A950460C460A9156F0D4
:1033D00052F902460A237F2A80464FF000092370E3
:1033E00040F29385214600240FE000BF64D5080019
:1033F00049D0020042FDFFFFFCE30800DCE40800C6
:1034000030DA080004E408001C464FEAD81343EA07
:1034100049634FEAD91668F07F00002E984608BF2E
:10342000B8F1800FB14601F8010F04F10103EBD2AE
:103430000DF2891103340B440A9F83F80080381978
:103440005146161954F0FDFF1DA856F014F9044614
:103450001223B8197F2CBB5500F1010E22464FF004
:10346000000340F24F857746D1094FEAD31841EA6D
:103470004361434662F07F0C002B0A4608BF802A56
:10348000A7EB000107F801CBEED28E448F1C8EF81B
:1034900000201DA92246384454F0D3FF284656F098
:1034A000EAF83C440A9A344406461A2310197F2E3F
:1034B000135500F1010E32464FF0000340F21F8514
:1034C0007746D1094FEAD31841EA4361434662F097
:1034D0007F0C002B0A4608BF802AA7EB000107F8E3
:1034E00001CBEED28E448F1C29468EF80020384442
:1034F000324654F0A6FFF319DBF80C510A989BF8FA
:103500001021119223446A1C00EB030103F1020411
:103510004FF0280C08BF012200F803C0E62C4FF042
:103520004503DBF808619BF880704B70CBF80C21E9
:1035300040F297800C9A049B9B1A0D9A9A423FF78F
:103540000BAF0B9BDDF838A0D94623B1DBF82C314B
:103550000133CBF82C310F9B2BB11A46B749079B8F
:10356000B74846F00FFE129B2BB11A46B549079B90
:10357000B34846F007FE139B002B00F02484D9F8D3
:103580004831B149AE4801330022C9F8483189F8C1
:103590005021032246F0F6FDDAF80030109A1B693C
:1035A00092ED0A8AD2ED0B8A92F8304092F83150AF
:1035B00092F8326092F9337050469847DAF800304A
:1035C0004FF0FF31D3F88C3050469847039A136878
:1035D000904610461B689847CDE900672B46224667
:1035E000F0EE680AB0EE480A51464046FCF75AF839
:1035F00099F80530954A02EB03135C7B631E622B3E
:1036000040F25584069BA3B10B9B002BD4BF002036
:1036100001200DF26C4DBDEC028BBDE8F08F90F8EF
:103620008640002C7FF48EAD90F81E41002C7FF474
:1036300089AD01200DF26C4DBDEC028BBDE8F08F21
:103640000323CB70002A00F07E8402238DF85830CB
:1036500005230D9371E60221012003232B540C4610
:1036600006E64FF4816212237F2CAAF800208AF824
:10367000023040F2BC838AF803404FF00509012074
:103680009FAB224618700A990AEB090054F0D9FE44
:10369000A1440021DAAC07F0070708465FFA85F875
:1036A00047EA47175FFA86FCC5F3072E0A4668F318
:1036B000070027739DF844706773C6F307236CF304
:1036C00007026EF30F204FF0FF3784F80880C5F330
:1036D000074863F30F222D0E276068F31740C6F3E7
:1036E000074765F31F60360E67F3174284F809E059
:1036F00084F804C066F31F626371E181E57219907A
:1037000033ADE67184F80A8028A8A7711B921A913C
:103710001C914F4E16F012FF2846289615F0BCFD5E
:1037200010224C49299528A816F006FE19A9102246
:1037300028A816F015FE52464B4628A8DEA916F01A
:1037400019FD2846289615F027FD28A809F1100A2A
:1037500016F0CAFD069B01330693089B002B00F070
:103760002182224653460E990398FBF7F1FF044647
:1037700047F0DEFCDBF83431079A0133013207925F
:10378000CBF83431002C3CD1DBF844310133CBF899
:103790004431FF25FE239BF85021FF2A00F00E82C2
:1037A00001320028D2B208BF0120022A8BF8502132
:1037B000CBF84C0101D901221392002C3FF4C1AE89
:1037C000022B02D80F9B01330F93039803685146D5
:1037D0009B689847099B012D0344099307D9042C42
:1037E00005D0129B0133129300230893A2E60B9B92
:1037F00001330B93059B022B00F0D2820023089328
:1038000098E6A31E032CDBB240F0D481DBF8402104
:103810000132CBF84021DBF83C210132CBF83C21CE
:10382000651EEDB2012D00F2C181DBF838210021C7
:103830000132CBF838218BF85011C1E70CE40800B5
:10384000B065002058E408009CE4080064D5080036
:10385000D0D40800F4D408009BF88630002B3FF445
:1038600069AE109B598C586AD3F81CC0002940F0EF
:10387000C98200283FF45EAE02220DF51E7A88460A
:10388000134691465646022400250021374600295A
:103890004FF0280E08BF802807F801EB19D33A46ED
:1038A000C30943EA4163CD0960F07F04002D184647
:1038B00008BF8028A2EB0603294602F8014BEFD28D
:1038C0009D1C05EB08094C461F44E5175FFA89F378
:1038D0004A46BE4938708C4500F2C28262A901276F
:1038E0000A91BC460E46002D4FF0120008BF802CF6
:1038F00037440870C0F07083781E002100E019463C
:10390000E3094FEAD51E43EA4563754664F07F0636
:10391000002D1C4608BF802C00F8016F01F1010347
:10392000EDD202318C440CEB090111911F44E3B23A
:103930000C460A993B7001EB0C00514654F081FD96
:10394000DBF80C61DBF808919BF810819BF8807024
:10395000731C08BF0123CBF80C31119BE62B3FF7FA
:10396000E9AD44F2083212237F2CAAF800208AF82D
:10397000023040F2BF829DF844308AF803300520BF
:1039800001259FAB021911921D70119B0A991033EA
:10399000224650441C460A9354F053FDB4F5807FF0
:1039A0003FF6C8ADDAAC4FF0000C07F007075FFA3E
:1039B00089FE63466246F0B247EA47176EF3070294
:1039C000C6F30721277360F30703C9F307272072A3
:1039D0006172C6F3074061F30F2367F30F22C9F347
:1039E000074161F31742360E4FEA19694FF0FF3570
:1039F00060F31743A4F80EC066F31F6384F804E075
:103A000069F31F62A1712560A07233ADE67284F87C
:103A10000D80677128A884F80790CDF878C0CDF89C
:103A200080C01D931F926A4E16F088FD2846289686
:103A300015F032FC28A810226649299516F07CFC66
:103A40001DA928A8102216F08BFC5246119B28A80D
:103A5000DEA916F08FFB2846289615F09DFB28A8B6
:103A6000DDF828A016F040FC74E6012B00F0B480CD
:103A7000DBF80C819BF81031119318F1010308BF9A
:103A800001230BF11C05CBF80C31284655F0F3FD52
:103A9000E628DBF808919BF8806004463FF64AADC3
:103AA0000DF51E7A4FF4847212237F28AAF80020A5
:103AB0008AF8023040F27E8105238AF803000A93D7
:103AC00001209FAB18700A9B294622460AEB03008F
:103AD00006F0070654F0B5FC46EA461E0A9E002290
:103AE00034190A941546DAAC5FFA88F0C8F3072C4B
:103AF0005FFA89F117469DF84460667360F3070525
:103B00006CF30F25C9F3072361F3070720724FF009
:103B1000FF36C8F3074063F30F2726604FEA1868A3
:103B2000C9F3074660F3174568F31F654FEA196943
:103B300066F3174784F80CE084F809C06371E281EA
:103B4000217169F31F67A0722895A6716DAD84F885
:103B50000B8062A884F8079029922B922A971C4E1A
:103B600016F0ECFC2846629615F096FB62A810222F
:103B70001849639516F0E0FB28A962A8102216F0F8
:103B8000EFFB0A9F52463B4662A8DEA916F0F2FA06
:103B90002846629615F000FB62A807F1100A16F09D
:103BA000A3FBD7E5782047F0CFFADAE5042C3FF401
:103BB0003CAEF0E5022B7FF62EAE31E6002840F059
:103BC0001C810122CBF84C21F5E500BF00105E5F9F
:103BD000D0D40800F4D408009BF80830002B3FF440
:103BE000A9AC109B1B7E002B3FF4A4AC109ED6E921
:103BF0000245DDA3D3E900232046294653F088FC83
:103C000000228046894620462946002353F0F2FED2
:103C100034460022D6E90467E569002840F0DA81DD
:103C2000D34B4046494653F0BDFA53F021FFCEA393
:103C3000D3E9002304463946304653F069FC00229C
:103C40008046894600233046394653F0D3FE002291
:103C5000002840F0BD81C64BCDF8894162AF4FF0DE
:103C6000150C0D2487F805C0404649463C700A975C
:103C700053F098FA53F0FCFEBE4BC7F806009D4285
:103C800040F2698125231220BB7216231193C7F8D5
:103C90000B5002464FF0260A0F23DBF80C519BF81D
:103CA0008040DBF808618DF87B02691C4FF0B80C8E
:103CB00008BF012107F803C03B44CBF80C1139467B
:103CC00001275F7020279F709FA812234FF442772F
:103CD0009BF81081ADF878728DF87A3254F0B1FB10
:103CE00004F007000023DAAC5FFA86FC194640EACC
:103CF00040105FFA85FE6CF307011A46C6F30727EA
:103D000020734FF0FF306EF3070220606771C5F338
:103D1000072067F30F21C6F30747A77160F30F224F
:103D200067F31741C5F30747360E2D0E67F31742A9
:103D300084F804C084F808E0E38166F31F6165F34A
:103D40001F62E671607233AE84F80D8028A8A772F6
:103D5000E5721E9320931F911D92DFF82C9216F0AE
:103D6000EDFB3046CDF8A09015F096FA28A8102269
:103D70008149299616F0E0FA1DA928A8102216F00C
:103D8000EFFA119B9EAA28A8DEA916F0F3F9304697
:103D9000CDF8A09015F000FA28A816F0A5FAD9E4FD
:103DA00000248BF81E4147F0C3F90894CBF81801A2
:103DB000FFF7C0BB04230A93C0B20DF27B2381E658
:103DC00006930B930993109890F9331090F83240B2
:103DD00090F8313090F83020D0ED0B0A90ED0A0ABF
:103DE0000191039800945146FBF75CFC00E4E0B2BB
:103DF0004FF004090DF27B2343E40122CBF84C0180
:103E00001392DAE45D4AA1F6E44382FB034207EE33
:103E1000901ADB17C3EB6203B8EE677A642BDFED11
:103E2000587A0DF51E7AA8BF642323EAE37367EE80
:103E3000277A8AF8013015238AF8023017EE903A73
:103E400008228AF80020CAF80330002862D1494BC2
:103E50009C4540F2AF800722134691460724002577
:103E600062A80D210627C0F801C00A908DF88811BC
:103E70000646BC460DF28D1135E5424BFFF786BA7A
:103E8000013CE4B215AB661C1846294632460C9339
:103E900054F0D7FA99F81E310D96002B3FF44DAA35
:103EA0000C9A02239355E3180D93FFF746BA47F097
:103EB0003FF9099AC4F1640302FB03F2B2FBF4F385
:103EC0000344C9F81431FFF79DBB17AD28460422FF
:103ED0000BF1810155F0FDFB00232B71FFF76BBA4D
:103EE000084642462946F0EE680AB0EE480A98476E
:103EF000FFF774B9E5B204200DF27B2342E50227F7
:103F0000FFF7F2BA0227FFF7C2BA02240DF28913B3
:103F1000FFF792BA092213469146092400250DF2B3
:103F20007F264FF00708B0E483BB99F81E21002AD2
:103F30003FF446AF15AB1A460C93022313700123CE
:103F40000D93FFF7FAB904230D93FFF7F6B9032396
:103F50000D93FFF7F2B911231193204622464FF03B
:103F6000210A0A2399E600BF00000000D012634135
:103F70000000E03F00105E5FF4D40800398EE338A3
:103F80006F12833AFCE30800D0D4080010460121E8
:103F9000DAADFFF762BB01230D93FFF7CEB912BB79
:103FA00001200446DAAD0126AE54002B3FF460A98F
:103FB000FFF753BB62AB19460A9309241223072269
:103FC0000B70119413464FF0020C0DF28917B1E4F7
:103FD000094B41E6084B24E60CF1010C0CEB0904FB
:103FE00011943146A6E4DAAD002208460C462A7048
:103FF00003210122D7E700BF0000E0BF000000005E
:104000002DE9F04F2DED088B8146C3B004F096FAF0
:10401000D9F8E410002940F04284D9F8E0100029D2
:1040200040F0B88442F23C6459F80410002940F092
:10403000FC8309F519542168002940F0C48341F636
:10404000985459F80410002940F0AC83D9F84C007A
:1040500003685B699847002840F3EA8401230C93C6
:10406000634CD4F8AC0009F1F403029330B1036857
:104070009B6998470490002840F0AC8099ED46ABCE
:1040800099ED489B002304939846D9F85C00036897
:104090001B68984782460C2099F83F414AF024FB60
:1040A00002204AF027FB012106204AF029FC0121C9
:1040B00006204AF0A9FC0A2047F046F804204AF0FE
:1040C00049FB002108EE100A06204AF09DFC4FF43F
:1040D0007A72D9E93601002353F0C0FE41F25C0345
:1040E00099ED4EBA29F803400746D9ED598A99F857
:1040F00060B199F8616199F93C51B8EEC88A47F00E
:1041000017F8DFED3C7A029B069068EE277A109351
:1041100017EE900ACDF85CA0ADF860408DED12ABC3
:104120008DED149B8DF8588053F09AF92EA3D3E9A6
:10413000002353F0EDF953F0C3FC12238DF87230D5
:1041400009F574630793049B1997ADF862008DED30
:104150001ABACDED1B8A8DF870B08DF871608DF8AC
:104160007350002B40F05C8141F254129DF8101006
:1041700009F802109DF8583041F2881209F802300F
:1041800043B1DDE91201DDE91423079CC4E98E0186
:10419000C4E9902399F8443F002B00F02B8141F2B1
:1041A000741319F8033083B341F2771419F904201A
:1041B000002A25DB09F583531978002938D101211C
:1041C0001970079B0C490D4803EB42129B3245F0D6
:1041D000D9FF24E094ED02AB94ED049B4FF001086D
:1041E00053E700BFAFF300809A99999999991340CA
:1041F00030AA002000803B3FC0EE0800B0650020E0
:10420000B9F8523F002B41F0998009F583531A7891
:1042100072B100221A707B497B4845F0A9FE99F8DB
:10422000443F2BB941F25F0319F80330002B71D0E2
:1042300046F07EFF41F2540359F80330C01A0028BB
:1042400068DB99F8445F002D00F00B8441F26103B4
:104250009DF858A019F80380BAF1000F40F05C8473
:1042600041F27612534609F802A043452AD041F2A2
:104270006102664909F80230634845F085FD41F264
:10428000761319F80330022B01F0D3806049614A9C
:10429000012B08BF11465C4845F076FD41F27413CE
:1042A00019F8033033B141F2701459F80430002B7F
:1042B00081F29E80544845F073FE99F8445F002DCA
:1042C00000F0A784B9F8543F33B141F2640459F8BF
:1042D0000450002D01F0B68041F25F0299F8445F6E
:1042E00019F80270002B00F0988441F2640359F829
:1042F0000330002B00F0918441F2771219F902206B
:10430000002AC1F28580BAF1000F40F09084002F9E
:1043100040F0318441F2A11319F80330002B43D04F
:1043200041F2B81459F80430002B40F0688441F28F
:10433000A113002209F80320079ED6E99A45D9E97E
:10434000460122462B46D6E99C6753F049FB0028DC
:104350003DD032463B46D9E9480153F041FBB0B36A
:10436000B9F8503F4FF47A7101FB03F14846FBF76F
:1043700049F9002800F03A8341F2BC12002309F801
:104380000230D9F800202449D2F89C2041F2B8101C
:104390008A4249F8003040F0518599F83F31002BAE
:1043A00040F01C84C9F8E43046F0C2FED9E9362357
:1043B000D9F8D010C9F8D000401A141843F10005FC
:1043C000C9E9364543B0BDEC088BBDE8F08FC9E9BB
:1043D0004645C9E94867D9F80030104AD3F8883013
:1043E000934240F0CE84D9F8CC1009F56A6008F009
:1043F0003FFAB5E709F583531A78002A7FF409AF2D
:1044000010E700BFA8EE0800B06500203CEF0800F0
:10441000A0EE080034EF080099CD020011D102008F
:1044200041F24D1319F80330002B40F0228341F282
:104430004C159C4A19F805104E1CA2FB06025208A6
:1044400009EBC1007A3100F5845409EB810100F5D4
:10445000875002EBC20284ED06ABB21A80ED009BDE
:104460000698C1F8400F09F8052041F24D110133BB
:1044700041F25012DBB209F80130069949F80210F6
:1044800041F22812069859F802204EF66021821A4D
:104490008A4240F2268300220892012B40F2AB832D
:1044A00041F22C12069859F802204EF66021821A29
:1044B0008A4212D809F5875109F58552089ED1E93B
:1044C0000245D2E9000142AF07EBC60242E91245BC
:1044D00042E92401721CD2B20892022B00F08B83B5
:1044E00041F23012069859F802204EF66021821AE5
:1044F0008A4200F27D83089C09F5855109F58752AF
:10450000D1E9026742ADD2E9040105EBC4020134EE
:10451000E4B2032B42E92467089442E9120100F057
:10452000938041F23412069859F802204EF6602129
:10453000821A8A4212D809F5855109F58752089ED8
:10454000D1E90445D2E9060142AF07EBC60242E9D0
:10455000244542E91201721CD2B20892042B73D096
:1045600041F23812069859F802204EF66021821A5C
:104570008A4212D809F5855109F58852089ED1E979
:104580000645D2E9000142AF07EBC60242E92445E5
:1045900042E91201721CD2B20892052B54D041F2AA
:1045A0003C12069859F802204EF66021821A8A427F
:1045B00012D809F5885109F58652089ED1E90245BD
:1045C000D2E9000142AF07EBC60242E9124542E9D7
:1045D0002401721CD2B20892062B35D009F58A52FA
:1045E000069812684EF66021821A8A4212D809F59E
:1045F000865109F58852089ED1E90245D2E90401A5
:1046000042AF07EBC60242E9244542E91201721C9F
:10461000D2B20892072B17D041F24412069859F8EB
:1046200002204EF66021821A8A4240F27286082BDE
:104630000AD041F24813069959F803304EF6602229
:10464000CB1A934240F2A386089B022B40F2D382FE
:10465000023BDBB201330A9320AB4FF000089B46CC
:10466000CDF83490BBEC027B4FFA88F5002D8DED30
:10467000027BC0F284831EAB03EBC503D3E9006762
:1046800051EC170B32463B4653F0C8F9002840F076
:10469000768308F1FF3464B204F101091EAB03EB29
:1046A000C90909E0398EE33879E9026732463B46A9
:1046B00053F0B4F960B9544642AB03EBC50522068A
:1046C00045E92267DDE9020104F1FF3A2546EBD511
:1046D00042AB03EBC4049DED027B0A9B08F1010889
:1046E000984504ED227BBDD1089BDDF83490CDF8D0
:1046F0003C905B08DB001EAA0E93D318D3E900237D
:10470000CDE9122332AB0A930023029330AB089316
:10471000CDF834800A9B029CF3E802AB65B2002D11
:104720000A93C0F22A83089B03EBC503D3E9006711
:1047300052465B463046394653F066F9002840F051
:104740001C83013C64B2089B04F1010803EBC80818
:1047500007E078E9026732463B4653F05FF960B9FB
:104760004C4642AB03EBC505230645E910675046AE
:10477000594604F1FF392546EBD542AB03EBC4049F
:10478000029B0D9A01339A42029344E910ABC1D1C6
:104790000E9A089BDDF83C901344D3E90023CDE941
:1047A0001423E1E4484603F0A3FC00283FF44EAC98
:1047B0000022D9F8CC1009F5067005F097FA00230D
:1047C00049F8043042E4484603F092FC00283FF4E4
:1047D00036ACCB4D002668682660036899ED4E0A1A
:1047E000DB6B99F8604199ED598A99F861719847A6
:1047F000686803682146D3F8E8309847686803681A
:10480000B0EE480AD3F8E430984739463246686833
:1048100013F052FB686885F824400368082C1B6E6F
:104820008CBF10212021984709E4484603F060FC22
:1048300000283FF4FEABB24D002649F804606868DA
:10484000026809F5195142F24C6442F24D67D26B8D
:1048500091ED010A19F8044091ED028A19F80770E8
:104860009047686803682146D3F8E830984768683D
:104870000368B0EE480AD3F8E43098473946324628
:10488000686813F019FB686885F824400368082CF1
:104890001B6E8CBF102120219847FFF7CABB4846EA
:1048A00003F026FC00283FF4B8AB30AB1A460221D7
:1048B00009F56A601C46089305F016FD224603467A
:1048C00009F16801484603F0FBFE0546E0B199F89E
:1048D000153209F5EB56043601333046DCB209F0E7
:1048E00089FE0746002840F067852946304609F0D2
:1048F000D7FE0094ADF8C000089AADF8C270294602
:104900003B46484604F076F8D9F800307D49D3F8A4
:104910009C208A4240F0D78599F83F21002A40F038
:10492000B885C9F8E420D3F89830774A934240F02C
:10493000C68599F83E31002B40F0A185C9F8E030DA
:1049400099F8443F002B3FF46DAB99F8493F002B99
:104950003FF468AB41F25E02B9F8543F012109F817
:104960000210002B3FF45EAB41F2640459F80430AE
:10497000002B3FF457AB46F0DBFB59F8043000F551
:104980006A5018301B1A002B7FF74CAB49F8040013
:10499000FFF748BB484603F0ABFB00283FF442ABAF
:1049A00030AB1A46022109F56A601C4605F09CFCF2
:1049B0002246034609F16801484603F081FE20B112
:1049C00001460022484604F0C9FBD9F800304E4A9F
:1049D000D3F89830934240F07C8599F83E31002B13
:1049E00040F06385C9F8E030FFF71CBB41F2BC140E
:1049F00019F804300133DBB2042B09F8043040F21B
:104A0000DA8041F2BD1241F2BC1119F802303F4880
:104A1000FF2B1CBF013309F8023041F2B81200230A
:104A200009F8013049F80230394945F0A1FABBE4F0
:104A3000334C60680368D3F88430984710F0140F43
:104A40007FF40CAB20460AF0FFF900287FF406AB98
:104A500020460AF09FF880F00100C3B20C93FFF7E4
:104A6000FFBA41F25F0319F80370002F40F0838012
:104A700050E441F25010069C59F8002040F6B7313E
:104A8000A21A8A427FF6FCAC41F24C16214A19F870
:104A900006104F1CA2FB075209EBC10452087A31E1
:104AA00004F5845509EB810104F5875402EBC20239
:104AB00085ED06ABBA1A84ED009B082B069CC1F865
:104AC000404F09F806207FF6D0AC41F2281249F891
:104AD000004059F802204EF66021A21A8A4200F2E4
:104AE000528409F5845109F58752D1E90645D2E986
:104AF00000010122CDE91E45CDE930010892CCE448
:104B0000FCA9002099CD020075CD0200B0650020FF
:104B100068EF0800398EE33841F274129DED147B82
:104B200019F802A0DDE912678DED027BBAF1000FE2
:104B300040F09C81079941F2681041F27513C1E978
:104B4000866781ED887B41F26C1541F2701441F269
:104B50007611069E49F8006009F803A04FF601702F
:104B6000012349F805A049F804A029F8010009F833
:104B70000230FFF77ABB0C9B002B7FF4CBAB25B147
:104B800099F8493F002B40F0138500230093B44A65
:104B9000B449079810ABFEF7C7FA002840F012811D
:104BA00046F0C6FA41F2540300F56A50183049F84D
:104BB0000300FFF7AFBB41F2A113012209F8032064
:104BC00046F0B6FA19F8043041F2883141F2B812D1
:104BD00001FB030049F80200FFF7E6BBA249484683
:104BE00001FB03F103F090FAC9F8E400FFF7DCBB26
:104BF000032B7FF496AC00230493FFF7B5BA46F07D
:104C000097FA59F80430C01A0028BFF690ABFFF7A6
:104C1000CBBB41F25F0319F80370BAF1000F3FF408
:104C200076AB41F2771319F90330002B0DDB002F1F
:104C300040F0AB8041F27513012209F80320FFF721
:104C400069BBBAF1000F3FF462AB4FF0000A0C9B56
:104C5000002B7FF45FAB002F40F09B8009F58D5354
:104C60001B78002B00F095809DF85830002B00F049
:104C70009080079C94ED947B8DED027B9DED127BE3
:104C8000DDE9022351EC170B8DED047B52F088FA1D
:104C90006DA3D3E9002352F03BFCDDE90423CDE909
:104CA0000801DDE9020152F07DFA69A3D3E900238E
:104CB00052F02EFC41EC100B4FF032FDD4E996235C
:104CC000DDE914018DED020B52F06AFA5EA3D3E91F
:104CD000002352F01DFC9DED020B53EC102B52F003
:104CE00017FCDDE90823CDE902011046194652F010
:104CF0000FFCDDE90223CDE904011046194652F00C
:104D000007FC02460B46DDE9040152F04BFA41EC88
:104D1000100B50F061F9B9F84E0F8DED040B52F005
:104D20008DFB9DED040B4CA3D3E90023CDE90201DB
:104D300051EC100B52F0ECFB02460B46DDE9020190
:104D400052F058FE28BB41F27513012209F80320E6
:104D5000BAF1000F3FF4DEAA25B199F8493F002BC4
:104D600040F0FF83012300933D4A3E49079810AB72
:104D7000FEF7DAF900284AD112E72C46FDE42C466A
:104D8000A6E448469847FFF7EBBA0C9B002B7FF44C
:104D9000C1AA3DB199F8493F23B141F25E03012216
:104DA00009F80320002300932D4A2E49079810ABE1
:104DB000FEF7BAF900283FF4F3AE41F27513012271
:104DC00009F8032041F25F019DF85820002309F8FB
:104DD0000130E2B1DDE91267DDE914AB079D41F274
:104DE000BC1241F2A11C0121C5E99A67C5E99CAB3F
:104DF00041F2B81009F80C1009F8023009F58D528B
:104E000049F80030C5E99467C5E996AB1170B9F867
:104E1000540F68B146F08CF9B9F8544F4EF6602340
:104E200003FB040444F62161002046F043F92044CA
:104E300041F2640349F80300FFF76CBA4846904713
:104E4000FFF7B2BAAFF30080399D52A246DF913F1F
:104E5000399D52A246DF813F00000000AE4D58410F
:104E600034A80020FCA9002080EE3600079B93EDBB
:104E7000867B5BEC17AB17EE102A5B463046394653
:104E80008DED047B52F08CF9F5A3D3E9002352F0A9
:104E90003FFB324604460D463B465046594652F0CB
:104EA00081F9F1A3D3E9002352F032FB079B93ED84
:104EB000887B41EC100B8DED087B4FF031FCDDE978
:104EC0000823DDE902018DED0A0B52F069F9E4A334
:104ED000D3E9002352F01CFB9DED0A0B53EC102B81
:104EE00052F016FB224682468B462B462046294628
:104EF00052F00EFB524604460D465B46504659465C
:104F000052F006FB02460B462046294652F04AF96B
:104F100041EC100B50F060F8D5A3D3E9002351EC1D
:104F2000100B52F0F5FA0022D34B04460D4652F016
:104F300039F952F09DFD41F2701349F80300B9F8B8
:104F40004E0F52F07BFA22462B4652F053FD0028BA
:104F500040F03A8241F26813B9F84C4F59F80320F7
:104F6000069D4FF47A7341F26C11AA1A03FB04F305
:104F70009A4249F80100C0F0E38241F2751241F211
:104F8000761319F802A0022209F803208AF0010A18
:104F900099F8DA3F002B62D0079BD3E92245DDE97F
:104FA00004232046294652F0FBF8ADA3D3E90023A1
:104FB00052F0AEFA224606460F462B46DDE90401C2
:104FC00052F0F0F8A8A3D3E9002352F0A1FA41EC83
:104FD000100B4FF0A5FB0799DDE90823D1E9240167
:104FE0008DED020B52F0DCF89DA3D3E9002352F0C3
:104FF0008FFA9DED020B53EC102B52F089FA02460A
:105000000B4652F085FA324604460D463B46304682
:10501000394652F07DFA02460B462046294652F0A8
:10502000C1F841EC100B4FF0D7FFB9F8D80F8DED58
:10503000020B52F0F3F99DED020B8DA3D3E900238F
:1050400004460D4651EC100B52F062FA02460B4634
:105050002046294652F0E2FC002840F07E8299F872
:10506000FA3F002B62D0079BD3E92A45DDE90423F0
:105070002046294652F094F879A3D3E9002352F050
:1050800047FA224606460F462B46DDE9040152F058
:1050900089F875A3D3E9002352F03AFA41EC100BDA
:1050A0004FF03EFB0799DDE90823D1E92C018DED96
:1050B000020B52F075F86AA3D3E9002352F028FAE4
:1050C0009DED020B53EC102B52F022FA02460B46D8
:1050D00052F01EFA324604460D463B4630463946EB
:1050E00052F016FA02460B462046294652F05AF86C
:1050F00041EC100B4FF070FFB9F8F80F8DED020B7B
:1051000052F08CF99DED020B59A3D3E9002304461C
:105110000D4651EC100B52F0FBF902460B462046AF
:10512000294652F07BFC002840F0198241F21A0314
:1051300019F80330002B64D0079BD3E93245DDE931
:1051400004232046294652F02BF845A3D3E9002337
:1051500052F0DEF9224606460F462B46DDE90401F1
:1051600052F020F840A3D3E9002352F0D1F941ECEA
:10517000100B4FF0D5FA0799DDE90823D1E9340186
:105180008DED020B52F00CF835A3D3E9002352F059
:10519000BFF99DED020B53EC102B52F0B9F902460A
:1051A0000B4652F0B5F9324604460D463B463046B2
:1051B000394652F0ADF902460B462046294651F0D9
:1051C000F1FF41EC100B4FF007FF41F218038DED9A
:1051D000020B39F8030052F021F99DED020B24A3D4
:1051E000D3E9002304460D4651EC100B52F090F920
:1051F00002460B462046294652F010FC002840F09B
:10520000A88141F23A0319F80330002B78D0079EA9
:10521000D6E93A45DDE904232046294651F0C0FF8E
:105220000FA3D3E9002352F073F922462B46CDE9B0
:105230000201DDE9040151F0B5FF0BA3D3E900231E
:1052400052F066F941EC100B4FF06AFADDE90823E1
:10525000D6E93C018DED040B51F0A2FF0EE000BF3A
:10526000399D52A246DF913F399D52A246DF813FD0
:1052700000000000AE4D58410000E03FDAA3D3E942
:10528000002352F045F99DED040B53EC102B52F026
:105290003FF9DDE9022306460F461046194652F053
:1052A00037F9324604460D463B463046394652F001
:1052B0002FF902460B462046294651F073FF41EC78
:1052C000100B4FF089FE41F238038DED020B39F8D7
:1052D000030052F0A3F89DED020BC5A3D3E9002310
:1052E00004460D4651EC100B52F012F902460B46E3
:1052F0002046294652F092FB0322002840F02A81E2
:1053000002234FF0FF3241F2771109F80120FEF736
:10531000ACBF09F5865109F58852089ED1E90445CC
:10532000D2E9060142AF07EBC60242E9244542E951
:105330001201721CD2B20892FFF779B945F0F8FE5B
:1053400041F26813B9F8525F59F803209E4B09F5F2
:105350008351801A03FB05F398420D7834BF002275
:10536000012295423EF45BAF98420A70FEF453AFBF
:1053700019F90420002ABEF624AF9449944844F059
:10538000F7FDFEF74CBF00220892FFF789B809F538
:10539000865209F58953D2E90645D3E90001089AF6
:1053A00042AE06EBC20343E9244543E91201531C14
:1053B000DBB20893FFF748B9234629460022484646
:1053C00003F0E4FAFFF7A0BA41F26C1359F8032096
:1053D000002A40F09180069849F8030041F27611C6
:1053E000924619F8013043453EF46CAFFEF73FBFDB
:1053F0007849774844F0C8FC59F8041074480A22E8
:1054000044F01AFD7449724844F0BEFCFEF752BFE6
:10541000069AD31A002BFFF614ACBAF1000F7FF4F2
:1054200016AC002F7FF4A7AB0C9B002B7EF472AF61
:1054300092E441F2771419F90430002B4DDA6749F0
:10544000FEF729BF45F074FEB9F8546F4EF660239D
:1054500003FB060644F62161284645F02BFE41F287
:105460005F0399F8445F19F80370304449F8040069
:10547000002D3FF4D2ABB9F8543FFEF733BF584983
:10548000484601FB03F102F03FFEC9F8E000FFF7D8
:1054900057BA4D49484601FB02F102F035FED9F8F2
:1054A0000030C9F8E400FFF73EBA4D49484601FB19
:1054B00003F102F029FEC9F8E000FEF7B3BD48464B
:1054C0009847FFF73DBA48469047D9F80030FFF7B4
:1054D0002ABA48469847FEF7A5BD42493C4844F0E1
:1054E00053FC19F90410079B394803EB41119B3118
:1054F00044F05CFCFEF7D2BE0699A1EB020A43F62B
:10550000972292454CD99DED027B079841F2681590
:1055100041F2751441F27612C0E9866780ED887B0E
:105520004FF601710020069E49F80560824609F891
:10553000040049F8030029F802100123FEF795BE84
:1055400041F27613824619F80330022B7FF4D9AE6C
:105550001EE5022252B20223D5E60022FAE701221A
:10556000F8E741F25C0239F8021000293FF4FAAB87
:10557000002741F25800069C59F80000124A201AF0
:1055800002FB01F2B2FBF3F3834204D841F25E0363
:10559000012209F80320002F3FF4E4ABFFF7F5BA2E
:1055A00041F276134FF0000A19F80330FEF75DBEA2
:1055B00041F25C0239F8021000293FF4E6AA012703
:1055C000D7E700BFAFF3008080EE360000EF0800A1
:1055D000B065002054EF080058EF080010E50800FF
:1055E000C0D4010048EF0800399D52A246DF913F28
:1055F00000000000AE4D58412DE9F0410446012065
:105600002061884616461F4645F092FD00F59C45F0
:1056100020352068E560C4F8148003689B689847CB
:10562000384654F00DF82D21054653F0D7FF08B148
:105630000023037033462A4604F118000249BDE8EE
:10564000F04153F075BF00BF74F3080070B5A0B00F
:10565000044645F06DFDB0F57A6F2068036873D39A
:10566000002211461B6A98472068036801219B6944
:105670009847206803680321DB69984720686169BF
:10568000036804315B6A98472068036814221B6A28
:1056900000219847206803680521DB699847656900
:1056A000A86C51F0DDFE95F87030009302460B4671
:1056B0000CA86F4953F03CFF206803680CA95B6A93
:1056C0009847206803681E221B6A00219847656975
:1056D000686F51F0C5FE95F87130009302460B4695
:1056E0000CA8644953F024FF206803680CA95B6A86
:1056F0009847A56B35B32B79002B00F08E8095F978
:105700003732002BC0F2908005EB431302AD9B3380
:105710002846594A282153F0D7FE20680368002103
:105720001B6A28229847A36B20681A790368002A0D
:1057300014BF03210221DB699847206803682946CA
:105740005B6A984720B070BDDB69042198472068E8
:105750004A4BD0E900210D268025CDE9005680393D
:1057600001EBD171556B49100322A84720680368EB
:105770000121DB6998472068036801219B699847EC
:1057800020683F4903689B6B98472368D3E9002151
:10579000081A00EBD0704110156A18461622A84767
:1057A0002068374903685B6A9847206803680121CD
:1057B000DB6998472068036825469B690121984763
:1057C00055F8180B036829469B6B98472268D2E965
:1057D0000031081A00EBD07041101B6A10462322DA
:1057E00098472068036829465B6A984720682549DE
:1057F00003689B6B98472368D3E90021081A00EBE4
:10580000D0704110156A18463022A84720681D49FB
:1058100003685B6A984720B070BD1B4B93E8070094
:1058200002AD85E8070078E795F834320BB16B8A52
:105830007BB995F83622022A18D0144B1449012A54
:1058400018BF0B4602AD0C4A2846282153F03CFEF7
:1058500063E745F06DFCD5F82822698A0D4B801A64
:1058600003FB01F39842E4D30B4BEBE70B4BE9E767
:1058700034F3080048F3080068F3080038F2080021
:1058800008F308001CF308005CF3080034EF08007C
:10589000A0EE080080EE360004E5080010E50800E0
:1058A00070B5044645F044FC6368984226D22068EF
:1058B00003681B68984700B970BD45F039FCA368C0
:1058C000984210D32068036800215B6998472046FE
:1058D000FFF7BCFE206803681B6D984745F028FC65
:1058E00000F57A70A06045F023FCE3689842E3D9A4
:1058F00020680368BDE87040DB6818472A2049F03B
:105900009FF823698342054601D028B1256145F0FF
:105910000FFCC8306060CAE7206803681B689847BE
:1059200018B9206803689B68984745F001FC00F5AA
:105930009C402030E060E9E733DF704712DF7047BA
:105940006AB138B58D18013D4C1E4FF480710020AE
:1059500045F0B0FB04F8010FAC42F6D138BD7047FA
:1059600010B5074B044603F1E80200F51850236018
:10597000C4F8C820343023F0CBFA204610BD00BF55
:10598000E4F0080030B50B4683B00546694618467A
:105990002C1D03F045FC05F2045502E00834AC422E
:1059A00008D008222146684652F03CFD0028F5D177
:1059B0002060606003B030BDF0B50F4683B006468E
:1059C0006946384603F02CFC341D06F2045501E00C
:1059D000AC421FD021460822684652F023FD08340D
:1059E0000028F5D13B7803F00303023B012B08D9D3
:1059F000D6F80C350133C6F80C350123184603B030
:105A0000F0BDD6F808350133C6F80835012318462D
:105A100003B0F0BDD6F804250C4C6B4603CB06EB67
:105A2000C202002391605060D6F80425013284FB45
:105A30000214D117C1EBA41101EB8101A2EB4112B9
:105A40001846C6F8042503B0F0BD00BF6766666659
:105A500070B5194D194B1A4A1A4919602846002485
:105A600084B0214640F8042B4FF4A0629C63C3E944
:105A7000014452F00AFD0420C5F80445C5F80C4560
:105A8000C5F8084547F038FF0F4E104B104A114C2F
:105A9000019301460092029503460C6030460E4A7F
:105AA0000E49F9F7E5FB0E4A0E49304604B0BDE851
:105AB00070404EF02DBE00BF2C7A0020DC7F00200D
:105AC0009CF30800D4A600201880002024AA0020FF
:105AD0002861002084F30800FCA90020C0A6002053
:105AE000006000206159030070B54FF4E1319AB0B5
:105AF0004B4C4C48F0F752FD4FF47A7045F024FBC4
:105B0000204600F0C5FA201D5A2107F081FA4649C7
:105B1000444844F04BF92169201D07F07FF9014604
:105B2000404844F045FA41480CF0F4FF18B901F040
:105B3000DDFB88B9FEE700213C480CF069FA002241
:105B400011463A480CF022FA394938480CF092FADA
:105B500036480CF021FCEAE7364C374809F05EF98C
:105B600045F0A4FA204629F06DFB344B344A354900
:105B700018A8CDE9184306F0CDFF68B3324C33497D
:105B80002848334E44F012F92022A4F6D861254863
:105B900003F0A6FB234844F003FA2E4B2E480025C1
:105BA0001D7009F06BFEA4F574602249FAF732FE0D
:105BB0002A4B2B4AA4F565613046FFF71DFD2948A5
:105BC000B46309F0CFFF2A46A4F574604FF47A510C
:105BD000F8F7ACF91AB070BD684601F0FBFB184845
:105BE0006946A0F16805602252F02BFC05F16806B9
:105BF0000A2408E001F0EEFB60226946304652F0CC
:105C000020FC013C06D095F86830013BDBB2FD2B4F
:105C10006846EFD818A80A4A0A4906F0A7FFADE778
:105C2000BCA60020B0650020E4F30800D4A6002044
:105C3000F4F30800C4B10020FCA90020A0E1090091
:105C400080800020FCE40800588F002004F4080045
:105C5000DC7F00203C7F002030AA002054ED0800AB
:105C6000F0E40800E0AA002070B5232082B00C46C2
:105C7000012148F0C9FE0121152048F041FE002114
:105C8000152048F0C1FE2046022148F039FE45F0BB
:105C90004FFA42F20F76054608E045F049FA401BFC
:105CA000B0424FF00A0006D845F04EFA204648F0C0
:105CB000C7FE0028F1D01C4B1C4953F824301C4867
:105CC0001F2B86BF03F01F031A4A4FF0A04203F5B3
:105CD000E07342F82310F0F749FB02A8002300F814
:105CE000013DFFF72BFE9DF807208AB94FF0804356
:105CF0000122C3F80025BFF34F8F0F490F4BCA682D
:105D000002F4E0621343CB60BFF34F8F00BFFDE7A7
:105D1000FFF712FE022804D09DF80730002BEAD1CD
:105D2000E4E78DF80730E1E758F808000C000300BD
:105D3000B06500200003005000ED00E00400FA050B
:105D40002DE9F043DFF880815348544DA9B007F0A6
:105D500077F9404653F08FFC4FF00009064608EBF8
:105D600000079E2E71DC2846F0F7C2FA002873D097
:105D70002846F0F7E3FAC4B20A2CF4D03C7021466E
:105D8000284607F8019F44F023F80D2C06F1010680
:105D9000E7D19F2E02D10D2388F89F30013E18F8DD
:105DA00006300D2B5BD03E4809F0EEFE30B13D4C85
:105DB0002368D3B945F0BCF9206001E0394B186085
:105DC000394C2046FEF71CF9384809F031FC3848B8
:105DD000FFF766FD374B986803689B68984794F80F
:105DE000893133BB29B0BDE8F08345F0A1F92368C0
:105DF00040F6B732C01A9042E2D92F4C2F492748BB
:105E000044F0D6F894F860307BB1002120460CF0C5
:105E1000FFF80022114620460CF0B8F82046284929
:105E20000CF028F920460CF0B7FA2A212548FFF794
:105E30001BFF2046F9F72CFC0028D3D10146164859
:105E400006F012FF29B0BDE8F0831448F0F750FACD
:105E500000289ED19F2E9ED0002EA4D09EE70A211E
:105E60000E4843F0B5FF002001466B4608F80600D7
:105E7000154A0D48FCF768FA9DF800301BB900235D
:105E800088F800308FE71149044843F08FFF6946D6
:105E9000024844F08DF8F2E7C0A60020B06500206B
:105EA000E0AA0020B8A600201880002030AA002018
:105EB000DC7F002024AA0020D4A60020ACF3080038
:105EC000D4F30800BCA600203C7F0020A4F3080007
:105ED000002070479FED010A704700BF00000000DE
:105EE000704700BF704700BF704700BF704700BFDA
:105EF0004FF0FF30704700BF00207047704700BF71
:105F000033DF704700797047BFF34F8F0549064B69
:105F1000CA6802F4E0621343CB60BFF34F8F00BF47
:105F2000FDE700BF00ED00E00400FA05C06870471F
:105F3000408A7047007C70470048704718F408009A
:105F40000048704718F4080008B50121232048F0E4
:105F50005BFD0121152048F0D3FC0021152048F0FD
:105F600053FDBDE80840FFF7CBBF00BF08B50121D6
:105F7000232048F049FD0121152048F0C1FC0021F3
:105F8000152048F041FDBDE80840FFF7B9BF00BF4C
:105F90000121232048F038BD0121232048F034BDE1
:105FA0000021232048F030BD0021232048F02CBDE3
:105FB00038B50D4604460121152048F0A1FC00210A
:105FC000152048F021FD0021252048F01DFD4C2D15
:105FD0004FF001014FF0060008D0422D06D048F0E6
:105FE0008FFC0021062048F00FFD0DE048F088FCF2
:105FF0000121062048F008FD236853F80C0C01220B
:106000002044022107F094F8236853F80C0C294629
:106010002044BDE8384007F0EFB800BFF8B503688A
:1060200004460D461520012153F8686C48F068FCC1
:106030000021152048F0E8FC0021252048F0E4FC70
:106040004C2D04EB06074FF001014FF0060008D07D
:10605000422D06D048F054FC0021062048F0D4FC24
:106060000DE048F04DFC0121062048F0CDFCA3597D
:1060700053F80C0C01223844022107F059F8A359B7
:1060800053F80C0C29463844BDE8F84007F0B4B882
:10609000036810B5044653F80C0C204406F0B4FD18
:1060A0000021042048F02CFC0F480CF0B7FF012120
:1060B000232048F025FC0121232048F0A5FC0121E4
:1060C000252048F01DFC2368084953F80C0C204497
:1060D00006F0C0FF2520012148F096FC0A20BDE80B
:1060E000104045F031B800BF90AF002014F4080014
:1060F000036870B553F86C5C4359044653F80C0CB4
:106100006619304406F080FD0021042048F0F8FBB9
:106110000F480CF083FF0121232048F0F1FB0121FF
:10612000232048F071FC0121252048F0E9FB635948
:10613000084953F80C0C304406F08CFF252001214F
:1061400048F062FC0A20BDE8704044F0FDBF00BF8B
:1061500090AF002014F40800704700BFB0F9180099
:10616000704700BF08B540680368D3F8843098478B
:1061700010F0140F14BF0120002008BD4068036810
:106180001B6F1847406803685B6F1847436893F8B4
:106190006C017047007970470020704738B504469D
:1061A00090F83600FF280D4602D0012148F02CFC63
:1061B00094F83500002148F027FC94F83600FF28B9
:1061C00002D0002148F020FC04F1480393E80600C7
:1061D000606C0CF065FD2946606C0CF089FE606C0B
:1061E0000CF0C2FD94F83600FF2802D0012148F0DF
:1061F0000BFC94F835000121BDE8384048F004BCA0
:1062000010B54FF47A7204460023D0E9040151F02E
:1062100025FEA368184410BDD0F88400704700BF65
:10622000D0F88800704700BF90F89030D0F88C000C
:10623000002B08BF0020704790F8A400704700BFF3
:1062400090F88000704700BF704700BF406801228F
:1062500012F034B9A2B1F8B54D1E0746AE187868F1
:106260000368D3F8A43098474FF4807104460020A7
:1062700044F020FF444005F8014FAE42EFD1F8BD95
:10628000704700BF10B5034B0360044609F068FF78
:10629000204610BD9CF7080010B5054A054B02606A
:1062A000044640F80C3F09F05BFF204610BD00BFDC
:1062B000004F09009CF70800D0F8C0305A1C0FD0DE
:1062C00010B500210446184648F09EFB0A2044F011
:1062D0003BFFD4F8C0000121BDE8104048F094BB5A
:1062E000704700BF10B50446D0F8C400421C02D06D
:1062F000002148F089FBD4F8C000431C02D00021E3
:1063000048F082FB94F9BC30ABB1D4F8B820013B23
:1063100084F8BC307AB192F9013063B1013B5BB2D1
:10632000537043B991781078B1FA81F14909BDE809
:10633000104048F069BB10BD828A10B512F0070307
:106340004FF0010118BF0B46044603EBD20390F84F
:10635000360084F8523048F0D3FA94F83500012121
:1063600048F0CEFA94F83600FF2802D0012148F018
:10637000C7FA012194F8340048F0C2FA606C0CF0BE
:1063800043FC606C02210CF005FD012194F83400FF
:1063900048F03AFB012044F0D7FE002194F8340085
:1063A00048F032FB0A2044F0CFFE012194F834007B
:1063B00048F02AFB606C0CF027FC012010BD00BFE8
:1063C00010B5054B0360044609F0CAFE204647F0AD
:1063D00097FA204610BD00BF9CF7080010B5044690
:1063E00047F08EFA204610BD00B583B002AA002304
:1063F00002F8013D40F6AC010123406811F0E8F9D4
:106400009DF80700A0F19600B0FA80F0400903B0B3
:106410005DF804FB4068002110F0DCB84068002102
:1064200011F0A6B82DE91848044644F081FED4E9DD
:106430000423A169A061401A12EB000B43F1000C88
:10644000C4E904BCBDE8188810B5002200238160AF
:10645000C0E90423044644F06BFEA06110BD00BFF8
:1064600030B5446885B00121204611F081F8012241
:106470000021204611F0E2F804AA7F2302F8013D32
:1064800000210123D4F86801CDE9003189210DF004
:10649000F5FBD4F86831186803680521DB69984773
:1064A00044F046FE05460AE044F042FE401B322816
:1064B0000ED8D4F86831186803685B6D9847D4F833
:1064C00068311868D96A03681B6998470028EBD1BE
:1064D00094ED580A204610F0ABF80121204612F046
:1064E000BFFA01222046114611F0E8FF05B030BD89
:1064F00043680A4693F86C1108F0C2BCD0F8C40097
:10650000421C08D008B548F09BFAA0F10100B0FA8F
:1065100080F0400908BD0120704700BFD0F8B400EA
:1065200030F0B4BE10B586B090F8A24090F89F301D
:1065300090F89E20B0F89C10029490F8A14090F83A
:10654000A000CDE9000404A822F0FEF804A822F07F
:1065500047F906B010BD00BF10B504466C3030F0EE
:106560000DFF0123237110BD10B590F8BC30D0F899
:10657000B82001335BB2002B044680F8BC300ADD42
:106580004AB1537801335BB2002B537003DD91782D
:10659000107848F039FAD4F8C400421C02D0012126
:1065A00048F032FAD4F8C000431C04D00121BDE801
:1065B000104048F029BA10BD90F85230002B00F07E
:1065C00025812DE9F04F4FF000084FF6FF7B87B093
:1065D000044647464546D946618A31B3D4E902E6C6
:1065E000002315FB013292B203F1010A1EF80200EA
:1065F00016F802C0844514D09B45B05428BF9B4672
:10660000984538BF9846618AA9451FFA8AF328BF82
:10661000A946AF4238BF2F468B4206D2D4E902E6E4
:10662000DFE701339BB29942DBD847F0ADFE01357D
:1066300094F85230ADB2AB42CED84FF6FF739945C5
:106640000497CDF8149000F0D38094F83600FF281A
:1066500040F0D88004F1480393E80600606C0CF029
:106660001FFB0599049A914200F2B58008F10103DD
:10667000A8EB0B02A3EB0B0301329BB25700019373
:10668000002303930A46BA4693B20293DB009BB2FF
:1066900000930026678AA58A009A94F83500C7F50A
:1066A000A077C5F1F00507EBD77705EBD5750BEBB8
:1066B000670702EB6505019ABBB29F180021013FF5
:1066C00047EA034748F0A0F92A21606C0CF010FC5F
:1066D000012194F8350048F097F9390E606C0CF000
:1066E00007FCC7F30741606C0CF002FCC7F30721FD
:1066F000606C0CF0FDFBF9B2606C0CF0F9FB3544FA
:10670000002194F8350048F07FF9ADB22B21606C80
:1067100045EA05450CF0ECFB012194F8350048F002
:1067200073F9290E606C0CF0E3FBC5F30741606C54
:106730000CF0DEFBC5F30721606C0CF0D9FBE9B26D
:10674000606C0CF0D5FB002194F8350048F05CF942
:106750002C21606C0CF0CCFB012194F8350048F042
:1067600053F9504644F00AFDD84505461CD3029B18
:10677000B4F812E0D4F8089003FB0EFE012303FAEC
:1067800006F15B4609EB0302A3EB0B0712F80E20A0
:106790000A4003F1010C2ED01FFA8CF3B4F85020FC
:1067A00025F817204345EDD9534600222946606C51
:1067B0000CF028FB0136284644F0FAFC082E7FF442
:1067C00069AF039B059A049901331A44039393B26A
:1067D0008B427FF659AF606C0CF0C6FA94F8360025
:1067E000FF2805D0012107B0BDE8F04F48F00CB9F3
:1067F00007B0BDE8F08F1FFA8CF3434525F817204A
:10680000C0D9D1E7002148F0FFF823E7704700BF67
:1068100003680C4ADB6B934210B5044610D1406804
:106820000368D3F88430984710F0140F14BF012088
:10683000002000B110BD2046BDE8104008F004BBA8
:106840009847F6E765610300F0B5044687B000F1AC
:106850006C0508E0D4F8B40003685B699847C1B2DE
:10686000284631F05BF8D4F8B40003681B699847F8
:106870000028EFD123683C4D9B69AB4260D194F86E
:10688000800008B9C4F8CC0044F052FCD4F8C830F9
:10689000984201D807B0F0BD44F04AFC237900F5D6
:1068A0007A70C4F8C8006BB9D4F8B030002B4AD065
:1068B00044F03EFCD4F8D0302C4AC31A934249D954
:1068C000012323712268D4F8CC100229134629DD54
:1068D000D4F8B06036B3D369254A316893424F6823
:1068E0003ED194F8A2C0B4F89C1094F89F3094F86C
:1068F0009E2094F8A100CDF808C094F8A0C0CDF86F
:1069000000C0019004A821F01FFF04A821F068FF37
:1069100001463046B8470023237144F009FC236840
:10692000C4F8D0009B69AB420FD194F880000028D6
:10693000B0D0D4F8CC300133C4F8CC3007B0F0BDBF
:10694000204698479DE72368ECE7204698470028B3
:10695000EFD19FE72268217913460029E2D0B2E700
:10696000204698470146D4E74162030040771B0068
:106970002565030038B50368284A5B6A93420446DC
:1069800047D190F83600FF2802D0012148F03CF8AA
:1069900094F83500002148F037F894F83600FF28C5
:1069A00002D0002148F030F804F1480595E80600CF
:1069B000606C0CF075F93621606C0CF099FA606C23
:1069C0000CF0D2F994F83600FF2802D0012148F0EB
:1069D0001BF8012194F8350048F016F894F83600B9
:1069E000002148F011F895E80600606C0CF058F9A9
:1069F0006021606C0CF07CFA606C0CF0B5F994F8D6
:106A00003600012148F000F80A20BDE8384044F083
:106A10009BBB3621984704F14805DFE79D610300E1
:106A200038B50368284A5B6A9342044647D190F818
:106A30003600FF2802D0012147F0E6FF94F8350028
:106A4000002147F0E1FF94F83600FF2802D0002132
:106A500047F0DAFF04F1480595E80600606C0CF099
:106A60001FF93621606C0CF043FA606C0CF07CF975
:106A700094F83600FF2802D0012147F0C5FF01211C
:106A800094F8350047F0C0FF94F83600002147F035
:106A9000BBFF95E80600606C0CF002F92021606CE9
:106AA0000CF026FA606C0CF05FF994F836000121C6
:106AB00047F0AAFF0A20BDE8384044F045BB362124
:106AC000984704F14805DFE79D61030038B5036886
:106AD000284A5B6A9342044647D190F83600FF2863
:106AE00002D0012147F090FF94F83500002147F0D3
:106AF0008BFF94F83600FF2802D0002147F084FF76
:106B000004F1480595E80600606C0CF0C9F83621E0
:106B1000606C0CF0EDF9606C0CF026F994F836001E
:106B2000FF2802D0012147F06FFF012194F83500C2
:106B300047F06AFF94F83600002147F065FF95E8BA
:106B40000600606C0CF0ACF8A021606C0CF0D0F981
:106B5000606C0CF009F994F83600012147F054FFFD
:106B60000A20BDE8384044F0EFBA3621984704F1D6
:106B70004805DFE79D61030038B50368284A5B6A72
:106B80009342044647D190F83600FF2802D00121F5
:106B900047F03AFF94F83500002147F035FF94F8AC
:106BA0003600FF2802D0002147F02EFF04F14805EF
:106BB00095E80600606C0CF073F83621606C0CF000
:106BC00097F9606C0CF0D0F894F83600FF2802D0EA
:106BD000012147F019FF012194F8350047F014FF17
:106BE00094F83600002147F00FFF95E80600606C2E
:106BF0000CF056F8E021606C0CF07AF9606C0CF047
:106C0000B3F894F83600012147F0FEFE0A20BDE8F3
:106C1000384044F099BA3621984704F14805DFE737
:106C20009D610300036870B55B6AD94EB3420446A8
:106C300040F0298390F83600FF2802D0012147F068
:106C4000E3FE94F83500002147F0DEFE94F83600AC
:106C5000FF2802D0002147F0D7FE04F1480595E84F
:106C60000600606C0CF01CF80121606C0CF040F91F
:106C7000606C0CF079F894F83600FF2802D00121FE
:106C800047F0C2FE012194F8350047F0BDFE962082
:106C900044F05AFA23685B6AB34240F0F08294F8F9
:106CA0003600FF2802D0012147F0AEFE94F83500EF
:106CB000002147F0A9FE94F83600FF2802D00021F9
:106CC00047F0A2FE95E80600606C0BF0E9FF112189
:106CD000606C0CF00DF9606C0CF046F894F836001E
:106CE000FF2802D0012147F08FFE012194F83500E2
:106CF00047F08AFE0A2044F027FA23685B6AB34211
:106D000040F0E18294F83600FF2802D0012147F0DC
:106D10007BFE94F83500002147F076FE94F83600AB
:106D2000FF2802D0002147F06FFE95E80600606C56
:106D30000BF0B6FF3A21606C0CF0DAF8606C0CF0E6
:106D400013F894F83600FF2802D0012147F05CFECA
:106D5000012194F8350047F057FE002194F83600E1
:106D600047F052FE95E80600606C0BF099FF552144
:106D7000606C0CF0BDF8606C0BF0F6FF012194F82C
:106D8000360047F041FE0A2044F0DEF923685B6AD2
:106D9000B34240F0948294F83600FF2802D00121DB
:106DA00047F032FE94F83500002147F02DFE94F8AC
:106DB0003600FF2802D0002147F026FE95E80600A5
:106DC000606C0BF06DFF3621606C0CF091F8606C1C
:106DD0000BF0CAFF94F83600FF2802D0012147F0DB
:106DE00013FE012194F8350047F00EFE002194F8BF
:106DF000360047F009FE95E80600606C0BF050FF86
:106E00006021606C0CF074F8606C0BF0ADFF012138
:106E100094F8360047F0F8FD0A2044F095F923680D
:106E20005B6AB34240F0578294F83600FF2802D0E4
:106E3000012147F0E9FD94F83500002147F0E4FD19
:106E400094F83600FF2802D0002147F0DDFD95E8D8
:106E50000600606C0BF024FF2A21606C0CF048F8EF
:106E6000606C0BF081FF94F83600FF2802D00121FE
:106E700047F0CAFD012194F8350047F0C5FD002117
:106E800094F8360047F0C0FD95E80600606C0BF002
:106E900007FF0021606C0CF02BF8606C0BF064FFB6
:106EA000012194F8360047F0AFFD002194F8360038
:106EB00047F0AAFD95E80600606C0BF0F1FE00219A
:106EC000606C0CF015F8606C0BF04EFF012194F82B
:106ED000360047F099FD002194F8360047F094FD04
:106EE00095E80600606C0BF0DBFE0021606C0BF097
:106EF000FFFF606C0BF038FF012194F8360047F07B
:106F000083FD002194F8360047F07EFD95E80600E9
:106F1000606C0BF0C5FEF021606C0BF0E9FF606C5B
:106F20000BF022FF012194F8360047F06DFD236835
:106F30005B6AB34240F0CB8194F83600FF2802D060
:106F4000012147F061FD94F83500002147F05CFD18
:106F500094F83600FF2802D0002147F055FD95E84F
:106F60000600606C0BF09CFE2B21606C0BF0C0FFE8
:106F7000606C0BF0F9FE94F83600FF2802D0012176
:106F800047F042FD012194F8350047F03DFD01E056
:106F90009D610300002194F8360047F035FD95E827
:106FA0000600606C0BF07CFE0021606C0BF0A0FF13
:106FB000606C0BF0D9FE012194F8360047F024FDF7
:106FC000002194F8360047F01FFD95E80600606C3C
:106FD0000BF066FE0021606C0BF08AFF606C0BF01A
:106FE000C3FE012194F8360047F00EFD002194F80D
:106FF000360047F009FD95E80600606C0BF050FE86
:107000000021606C0BF074FF606C0BF0ADFE012191
:1070100094F8360047F0F8FC002194F8360047F069
:10702000F3FC95E80600606C0BF03AFE8721606C7B
:107030000BF05EFF606C0BF097FE012194F83600B8
:1070400047F0E2FC23685B6AB34240F02C8194F87D
:107050003600FF2802D0012147F0D6FC94F8350015
:10706000002147F0D1FC94F83600FF2802D000211F
:1070700047F0CAFC95E80600606C0BF011FE112188
:10708000606C0BF035FF606C0BF06EFE94F8360010
:10709000FF2802D0012147F0B7FC012194F8350008
:1070A00047F0B2FC0A2044F04FF823685B6AB34211
:1070B00040F0F58094F83600FF2802D0012147F017
:1070C000A3FC94F83500002147F09EFC94F83600AC
:1070D000FF2802D0002147F097FC95E80600606C7D
:1070E0000BF0DEFD1321606C0BF002FF606C0BF007
:1070F0003BFE94F83600FF2802D0012147F084FCC3
:10710000012194F8350047F07FFC0A2044F01CF878
:1071100023685B6AB34240F0CE8094F83600FF28C3
:1071200002D0012147F070FC94F83500002147F0AF
:107130006BFC94F83600FF2802D0002147F064FC75
:1071400095E80600606C0BF0ABFD2921606C0BF03C
:10715000CFFE606C0BF008FE94F83600FF2802D0DA
:10716000012147F051FC012194F8350047F04CFC17
:107170000A2043F0E9FF23685B6AB34240F097803E
:1071800094F83600FF2802D0012147F03DFC94F826
:107190003500002147F038FC94F83600FF2802D073
:1071A000002147F031FC95E80600606C0BF078FD9B
:1071B0002121606C0BF09CFE606C0BF0D5FD94F807
:1071C0003600FF2802D0012147F01EFC012194F86F
:1071D000350047F019FC0A2043F0B6FF2368424906
:1071E000DA6B8A4254D15B6AB34278D194F83600A4
:1071F000FF2802D0012147F007FC94F83500002158
:1072000047F002FC94F83600FF2802D0002147F036
:10721000FBFB95E80600606C0BF042FD3621606CCC
:107220000BF066FE606C0BF09FFD94F83600FF28B3
:1072300002D0012147F0E8FB012194F8350047F026
:10724000E3FB002194F8360047F0DEFB95E80600EA
:10725000606C0BF025FD6021606C0BF049FE606CEA
:107260000BF082FD012194F8360047F0CDFB0A2097
:1072700043F06AFF4EF20703A4F8503070BD1121AD
:107280002046984736E50121984704F14805FEE479
:10729000204690474EF20703A4F8503070BD1321EA
:1072A0002046984731E7112120469847FAE62121E8
:1072B000204698478FE729212046984758E73621EE
:1072C0002046984792E53A212046984745E52B21EC
:1072D000204698475EE62A2120469847CFE536218A
:1072E00020469847ADE700BF7569030070B52E4989
:1072F0002E4884B002F0E4FA1623132217212C48FA
:107300000BF038FD00262A48102516240BF07CFCD3
:107310001223CDE9015600949FED261ADFED260ACF
:107320009FED260A2648052208210DF071FB00F288
:10733000C323012B28D90446D0B9012441F22103EB
:10734000214641F60F5200941D4811F08BF99FED34
:107350001D0A1B4810F00AFE2146194811F080FB57
:1073600022462146164811F0A9F8204604B070BD07
:107370001549164842F01AFD21460A22134842F0E8
:1073800069FE002004B070BDCDE9015600949FED68
:10739000101ADFED090A9FED090A09481223052298
:1073A00008210DF035FBC6E790AF002024AA00208D
:1073B00068AF00206666E63F00007A428D67594458
:1073C00034A8002000000C433CF80800B065002001
:1073D0000000000010B582B0054A064B00926946D5
:1073E0000446019300F0B4FE204602B010BD00BF79
:1073F0002CF7080034A800202DE9F0417149724BA8
:107400004868724A50F80C7C714C8868DC601D46F4
:1074100086B002F188060024D8516E4945F8046F01
:107420004FF0010848201A6004918DF815808DF8FE
:10743000144046F061FA06AB064613E90300664ABB
:10744000664F02AB83E803001123CDE900323046DA
:107450001923142218210CF0DFF8314638460DF0BC
:10746000E1FD5F4B5F4A6049604E3B6038464DF03E
:107470004FF95F4B5F48604A60499D605F60604DB7
:107480001A6083F824400022C3E90344C6E90004DB
:107490000023C6E90423B16043F04AFE594B5A4A1F
:1074A000B0612946C3E9014641F8052B574F85F8DD
:1074B0000480642205F16C001F602FF02FFF26234B
:1074C000184615224146524EC5F8B040C5E9303243
:1074D000C5F8B84085F8BC40C5E93244C5F8D0408D
:1074E000C5F8B46047F00CFAD5F8C000214647F063
:1074F0008BFAD5F8C400431C07D0414647F000FA88
:107500002146D5F8C40047F07FFA424C424ADFF8E2
:1075100028C14249C2F8AC502046802300260027EB
:1075200063604023002540F80CCBC2E90267C2E942
:107530000467C2E90667A36001260223116082F88E
:10754000A430C2F8A05082F8A55082F8A650C2F824
:10755000A86008F0E5FD3248324BE06023654FF645
:10756000FF700B23A4F85C0084F842302E4961655B
:1075700040F602400423A4F8400023772B4AC4F8C5
:107580001E204FF0FF334FF480704FF47F61A4F85A
:1075900058006184C4E91133E3642046114A244948
:1075A00084F86050C4E919554DF0B2F8CDE90056A1
:1075B00033464FF47A722A211E4808F0B9FA06B011
:1075C000BDE8F08104F50800BCA6002020F5080005
:1075D00030F8080080841E0068AF002034A8002026
:1075E00014F60800006000204962030040A7002054
:1075F000FCA90020E4F7080038F70800EF93446680
:1076000060A7002024AA0020F8F7080054FA080018
:1076100040CA0020D4A6002030AA0020040A090095
:107620009CF708007CAF0020005A6202F00087003F
:1076300099620300E0AA0020004F090000212A20DF
:1076400047F05EB9704700BF704700BF704700BF8A
:10765000704700BF002070479FED010A704700BFD0
:10766000000000009FED010A704700BF000000000D
:10767000704700BF704700BF704700BF704700BF32
:1076800000487047A0E109000020704700207047C3
:10769000B7EE000A704700BFC82070474FF47A6009
:1076A000704700BF00000000DFED137A77EEC07A6C
:1076B00070B517EE900A0E464FF0D2FE9FED0C0B00
:1076C00041EC110B4DF0ECFA002251EC100B0B4B7E
:1076D0004FF066FD044630460D464FF09FFE0246D1
:1076E0000B46204629464FF013FF50F0C1F970BDFC
:1076F00000000000000024409A99593F0000F03F2C
:1077000038B50446406D0268002312686363236342
:10771000C4E90E33A4F858309047236821491A6B06
:1077200020628A4222D19B691F4A2048A06493426A
:1077300024D1B6EE007A07EE900AF8EE677A606D13
:107740001B4D036867EE877A1B68FCEEE77AC4ED91
:10775000107A9847236D1A6860641168A94217D19E
:10776000D26A1846904784F82C0038BD20469047CE
:1077700023680D4A9B69A0649342DAD0204698475B
:10778000F7EE007A30EE270AA06C87EE807AD2E717
:1077900018468847236D1A681846D26A904784F8BD
:1077A0002C0038BDC5CB02009176030080EE360078
:1077B00045760300000000002DE9F04304462DED5E
:1077C000028B006D0368C3B05B6802A9FF22984773
:1077D000061E3CDD206D964F036821689A6B4D684C
:1077E000BA4239D15B6B934A9FED938A93423CD165
:1077F000924BDFED910A9D423DD1E06C03681B681E
:107800009847054618B39DF8083003709A0919D1B6
:1078100013F0030336D0032B34D00221C0F8062026
:107820008846012302AAD35CAB809A11032A09D0AF
:1078300003F03F0302FB0333DAB2402A02D890443C
:10784000464529DAE06C036829465B68984743B0EF
:10785000BDEC028BBDE8F0839047206D754A03684C
:107860005B6B9342B0EE408AC2D09847734B9D4207
:10787000F0EE400AC1D0B0EE480A324602A92046D6
:10788000A847BAE7BDF80B30BDF809202B810621C7
:10789000EA8088460523C5E702AB194405F10A00D2
:1078A00050F0CFFDA6EB080292B2B82A6A80C9D880
:1078B00002AB03EB080105F14A0050F0C2FD206D58
:1078C00003689B6BBB4240F0A580002385F8023122
:1078D000D4F85080D8F800309A6BDB68BA4240F098
:1078E00094809FED550A314640469847206D0368C5
:1078F00031469B68B0EE408A98476369226803442A
:10790000636106462846976801F076FC4C4B9F421F
:107910006DD12B78226803F00303012B5CD8A36B95
:10792000D269484901338A42A36367D1DFED467AC1
:1079300077EEC87A17EE900A4FF092FD9FED3A0B62
:1079400041EC110B4DF0ACF9002251EC100B3F4B08
:107950004FF026FC8046304689464FF05FFD0246D8
:107960000B46404649464FF0D3FD50F081F806469D
:10797000312E14DD606DE46C036822681B68576A61
:1079800098472946B6F5FA4FD4BF821900F5FA4256
:107990002046B84743B0BDEC028BBDE8F0832368B6
:1079A00029461B6820469847064600283FF44AAF00
:1079B000012E3FF44CAF606DE46C036822681B68D5
:1079C00097689847320E26F07F43013A03442946D0
:1079D000D2B22046B8473AE7E36B12680133E3635B
:1079E00029462046904706460028E1D12AE702466C
:1079F000B0EE480A29462046B8478AE73146B0EE3D
:107A0000480A204690470646B2E701934046904711
:107A1000019B68E79847F0EE407AFEEECF7ACDED15
:107A2000017A9DF9043051E7000000000000244075
:107A300065760300597603000000000071760300AC
:107A400075760300A97603009A99593F0000F03F2C
:107A5000F0B50446406DE56C03682A681B6816693A
:107A60002DED028BC1B0984701462846B04718B9A2
:107A700041B0BDEC028BF0BD606D944E03681B6895
:107A800098472268636C9169B1420746A0EB0305F1
:107A900040F09180B6EE008A136B8D4A934240F01D
:107AA00083809FED8C7A07EE905AF8EE677A67EE46
:107AB000887AFCEEE77A17EE903A63B128EE078AEF
:107AC000226C6764BCEEC88A1A4418EE103A9A42D7
:107AD00028BF1A462264206D0368FF219B689847DF
:107AE000276C4508AF4244D3606DA56903681B68E5
:107AF0009847401B0028BBDD206D774A03681B6B4D
:107B0000934240F09580E56C606D2A680368D66802
:107B10001B680022E261984701462846B047606032
:107B20000028A5D003788DF80030037813F0030304
:107B30004BD1C2880389ADF80120ADF8033006258A
:107B4000052283880DF8023000F10A0102790DEB5D
:107B5000050001F033FB6668728805445319FF2B5A
:107B600040DDE06C036831465B6898470023636042
:107B70007EE723689B69B3422CD1B0EE008A606D2A
:107B800003681B689847EB1B00EE103AB8EE400AFA
:107B900020EE080ABCEEC00A10EE103A0344A361BE
:107BA00041B0BDEC028BF0BD2046984707EE900A2D
:107BB000B8EE677A77E720468847F7EE007A30EE2E
:107BC000270A226887EE808A66E7032BB1D0022558
:107BD0000122B6E720469847B7EE008A30EE088AC1
:107BE000276CCCE706F14A010DEB050050F029FCAB
:107BF000206D72880368154429469B68984706469D
